:100000000C94F6180C9421190C9421190C942119B4
:100010000C9421190C9421190C9421190C94211978
:100020000C9421190C9421190C9421190C94211968
:100030000C9421190C94A3190C9421190C942119D6
:100040000C9421190C94517F0C9421190C942119B2
:100050000C9421190C9421190C941F880C94021AE9
:100060000C9421190C94C4540C9421190C9421194A
:100070000C9421190C9421190C9421190C94211918
:100080000C9421190C9421190C9421190C94211908
:100090000C9421190C9421190C9421190C94819A17
:1000A0000C9421190C9421190C9421190C942119E8
:1000B0000C9421190C9421190C9421190C942119D8
:1000C0000C9421190C9421190C9421190C942119C8
:1000D0000C9421190C9421190C9421190C942119B8
:1000E0000C942119084AD73B3BCE016E84BCBFFD5E
:1000F000C12F3D6C74319ABD56833DDA3D00C77FF8
:1001000011BED9E4BB4C3E916BAAAABE0000008090
:100110003F05A84CCDB2D44EB93836A9020C50B91F
:10012000918688083CA6AAAA2ABE000000803F0249
:1001300000002100240027002A002D003000330099
:1001400001010000040107010A010000220025004E
:1001500028002B002E0031003400020100000501B0
:1001600008010B01000020002300260029002C00BC
:100170002F003200000100000301060109010505FE
:100180000505070508080808020202020A0A08080D
:10019000040404040101010101010101030303033B
:1001A00003030303040707070C0C0C0C0C0C0C0CCA
:1001B0000202020206060606060606060B0B0B0BDB
:1001C0000B0B0B0B01021020200808102040102000
:1001D000408002010201080402010102040810200B
:1001E0004080804020100804020180040201804009
:1001F0002010080402010804020101020408102072
:10020000408001020408102040800000090A020812
:100210000B0C0D07060304010000000000000000A5
:1002200000000000000000000000000000000000CE
:1002300000000000000011100F000000000000008E
:1002400000000000000000000000000000000000AE
:100250004D383420582059205A2045006563686F76
:100260003A0043616E6E6F7420656E746572207320
:1002700075626469723A20004D3234004D32332089
:100280002573006175746F25692E67004572726F62
:10029000723A006572726F722077726974696E6764
:1002A00020746F2066696C6500436172642065721A
:1002B000726F723A004E6F74205344207072696EF0
:1002C00074696E67002F005344207072696E746900
:1002D0006E67206279746520002E0044656C657439
:1002E000696F6E206661696C65642C2046696C6577
:1002F0003A200046696C652064656C657465643AF3
:10030000002E006F70656E206661696C65642C203C
:1003100046696C653A200057726974696E6720748B
:100320006F2066696C653A20002E006F70656E2044
:100330006661696C65642C2046696C653A20002E04
:10034000006F70656E206661696C65642C2046697B
:100350006C653A200046696C652073656C65637452
:100360006564002053697A653A200046696C65200F
:100370006F70656E65643A20002E006F70656E20A8
:100380006661696C65642C2046696C653A2000538F
:10039000442063617264206F6B006F70656E526FF2
:1003A0006F74206661696C656400766F6C756D654D
:1003B0002E696E6974206661696C6564005344201F
:1003C000696E6974206661696C006563686F3A00E4
:1003D00048617264636F6465642044656661756C2E
:1003E000742053657474696E6773204C6F61646523
:1003F000640053746F7265642073657474696E670A
:10040000732072657472696576656400204400200B
:1004100049002020204D33303120500050494420E5
:1004200073657474696E67733A00205A002059002E
:1004300020204D323036205800486F6D65206F66A1
:100440006673657420286D6D293A00204500205A96
:100450000020580020420020540020204D3230352A
:10046000205300416476616E636564207661726931
:1004700061626C65733A20533D4D696E2066656517
:10048000647261746520286D6D2F73292C20543D92
:100490004D696E2074726176656C20666565647264
:1004A00061746520286D6D2F73292C20423D6D6984
:1004B0006E696D756D207365676D656E7420746906
:1004C0006D6520286D73292C20583D6D6178696D0C
:1004D000756D205859206A65726B20286D6D2F73D9
:1004E000292C20205A3D6D6178696D756D205A2048
:1004F0006A65726B20286D6D2F73292C2020453D75
:100500006D6178696D756D2045206A65726B202874
:100510006D6D2F73290020540020204D323034207F
:100520005300416363656C65726174696F6E3A2054
:10053000533D616363656C65726174696F6E2C20F5
:10054000543D7265747261637420616363656C65A8
:10055000726174696F6E00204500205A00205900B6
:1005600020204D3230312058004D6178696D756D15
:1005700020416363656C65726174696F6E20286DDC
:100580006D2F7332293A00204500205A002059006F
:1005900020204D3230332058004D6178696D756DE3
:1005A0002066656564726174657320286D6D2F73B4
:1005B000293A00204500205A0020590020204D39BA
:1005C0003220580053746570732070657220756E08
:1005D00069743A0053657474696E67732053746F5D
:1005E000726564006563686F3A004572726F723AB3
:1005F000005072696E7465722073746F70706564F8
:100600002064756520746F206572726F72732E207E
:1006100046697820746865206572726F7220616E19
:100620006420757365204D39393920746F207265E7
:1006300073746172742E202854656D7065726174D4
:100640007572652069732072657365742E20536519
:1006500074206974206166746572207265737461B8
:100660007274696E6729005072696E7465722068D1
:10067000616C7465642E206B696C6C282920636141
:100680006C6C656421006F6B00526573656E643A33
:1006900020002200556E6B6E6F776E20636F6D6D5C
:1006A000616E643A20220020423A300020423A3102
:1006B000006F6B20523A002200556E6B6E6F776EA2
:1006C00020636F6D6D616E643A2022007A5F6D6108
:1006D000783A2000795F6D61783A2000785F6D6923
:1006E0006E3A20005A3A00593A0020436F756E74F2
:1006F00020583A2000453A005A3A00593A00583AF0
:10070000004649524D574152455F4E414D453A4D85
:1007100061726C696E2056313B20537072696E7441
:1007200065722F6772626C206D61736875702066E8
:100730006F722067656E36204649524D57415245CB
:100740005F55524C3A687474703A2F2F6669726D17
:10075000776172652E756C74696D616B65722E635D
:100760006F6D2050524F544F434F4C5F564552537C
:10077000494F4E3A312E30204D414348494E455F56
:10078000545950453A556C74696D616B65722045DA
:10079000585452554445525F434F554E543A310ACE
:1007A0000020423A0020453A00543A0020573A00CF
:1007B00020453A00543A002042403A0020403A0096
:1007C000202F0020423A00202F006F6B20543A0067
:1007D0002569206D696E2C202569207365630045AD
:1007E0006E642066696C65206C697374004265678D
:1007F000696E2066696C65206C6973740000000086
:100800000000006643000066430000000000000096
:100810000000000000000066430000664300006620
:10082000430000664300006643000066430000A0EA
:10083000400000A04000004040FF01012569206801
:100840006F757273202569206D696E75746573000C
:10085000446F6E65207072696E74696E6720666998
:100860006C65005072696E7465722073746F70707D
:1008700065642064756520746F206572726F727391
:100880002E2046697820746865206572726F722028
:10089000616E6420757365204D39393920746F207D
:1008A000726573746172742E202854656D70657260
:1008B00061747572652069732072657365742E208A
:1008C0005365742069742061667465722072657363
:1008D00074617274696E6729006F6B004E6F204CF3
:1008E000696E65204E756D62657220776974682047
:1008F000636865636B73756D2C204C617374204C59
:10090000696E653A20004E6F20436865636B7375AE
:100910006D2077697468206C696E65206E756D62F4
:1009200065722C204C617374204C696E653A20000E
:10093000636865636B73756D206D69736D61746356
:10094000682C204C617374204C696E653A20004C11
:10095000696E65204E756D626572206973206E6FD9
:1009600074204C617374204C696E65204E756D6205
:1009700065722B312C204C617374204C696E653A82
:1009800020004D31313000446F6E6520736176690F
:100990006E672066696C652E006F6B004D32390002
:1009A0002020506C616E6E6572427566666572429B
:1009B000797465733A20002046726565204D656D37
:1009C0006F72793A2000446563203136203230312D
:1009D0003300436F6D70696C65643A200056657230
:1009E00073696F6E2031332E313200207C204175C7
:1009F00074686F723A2000446563203136203230CB
:100A000031332031353A30373A353500204C617377
:100A10007420557064617465643A2000312E302E64
:100A200030004D61726C696E200020536F667477E0
:100A30006172652052657365740020576174636844
:100A4000646F67205265736574002042726F776E21
:100A5000206F757420526573657400204578746545
:100A6000726E616C20526573657400506F776572A9
:100A70005570007374617274002200656E71756543
:100A8000696E672022002200656E717565696E6768
:100A90002022006563686F3A0020746F6F206C6FCE
:100AA0006E6720657874727573696F6E20707265F9
:100AB00076656E7465640020636F6C64206578747D
:100AC000727573696F6E2070726576656E74656499
:100AD0000000002110422063308440A550C660E72A
:100AE00070088129914AA16BB18CC1ADD1CEE1EFE3
:100AF000F13112100273325222B5529442F772D67B
:100B000062399318837BB35AA3BDD39CC3FFF3DE32
:100B1000E36224433420040114E664C774A44485CA
:100B2000546AA54BB528850995EEE5CFF5ACC58D82
:100B3000D55336722611163006D776F6669556B41A
:100B4000465BB77AA719973887DFF7FEE79DD7BCD2
:100B5000C7C448E5588668A778400861180228236A
:100B600038CCC9EDD98EE9AFF9488969990AA92B22
:100B7000B9F55AD44AB77A966A711A500A333A12BA
:100B80002AFDDBDCCBBFFB9EEB799B588B3BBB1A72
:100B9000ABA66C877CE44CC55C222C033C600C410A
:100BA0001CAEED8FFDECCDCDDD2AAD0BBD688D49C2
:100BB0009D977EB66ED55EF44E133E322E511E705A
:100BC0000E9FFFBEEFDDDFFCCF1BBF3AAF599F7812
:100BD0008F8891A981CAB1EBA10CD12DC14EF16FC3
:100BE000E18010A100C230E3200450254046706728
:100BF00060B9839893FBA3DAB33DC31CD37FE35E54
:100C0000F3B1029012F322D2323542145277625677
:100C100072EAB5CBA5A89589856EF54FE52CD50D63
:100C2000C5E234C324A014810466744764245405C7
:100C300044DBA7FAB79987B8975FE77EF71DC73CF3
:100C4000D7D326F2369106B0165766767615463417
:100C5000564CD96DC90EF92FE9C899E9898AB9AB03
:100C6000A94458654806782768C018E1088238A367
:100C7000287DCB5CDB3FEB1EFBF98BD89BBBAB9A93
:100C8000BB754A545A376A167AF10AD01AB32A92B7
:100C90003A2EFD0FED6CDD4DCDAABD8BADE89DC9A3
:100CA0008D267C076C645C454CA23C832CE01CC107
:100CB0000C1FEF3EFF5DCF7CDF9BAFBABFD98FF833
:100CC0009F176E367E554E745E932EB23ED10EF057
:100CD0001E7C3C3E5E2B3D3F2F5B5D3B2C2A225C05
:100CE0000045313A200045303A20005A3A20005958
:100CF0003A2000583A20004D53312C4D53322050A9
:100D0000696E730A0024F404D9201BC40C5C0E988D
:100D100004C4095F0265077101F405F900FB04B31F
:100D20000048048700C103690058035500030345C8
:100D300000BE023A008402310053022A0029022533
:100D40000004022000E4011C00C8011900AF0117D3
:100D5000009801140084011300710110006101105A
:100D60000051010E0043010D0036010B002B010B59
:100D70000020010B00150109000C01090003010806
:100D800000FB000800F3000800EB000700E4000689
:100D900000DE000600D8000600D2000600CC0005E8
:100DA00000C7000500C2000500BD000400B9000432
:100DB00000B5000400B1000400AD000400A9000467
:100DC00000A5000300A20003009F0004009B000395
:100DD00000980003009500020093000300900003B8
:100DE000008D0002008B00030088000200860002D4
:100DF0000084000300810002007F0002007D0002E9
:100E0000007B0002007900020077000100760002FA
:100E1000007400020072000100710002006F000205
:100E2000006D0001006C0002006A00010069000210
:100E30000067000100660001006500010064000217
:100E4000006200010061000100600001005F00021B
:100E5000005D0001005C0001005B0001005A000120
:100E60000059000100580001005700010056000120
:100E70000055000100540001005300000053000120
:100E8000005200010051000100500001004F00011C
:100E9000004E0000004E0001004D0001004C00011A
:100EA000004B0000004B0001004A00010049000116
:100EB0000048000000480001004700010046000013
:100EC000004600010045000000450001004400010B
:100ED0000043000000430001004200000042000106
:100EE000004100000041000100400001003F0000FF
:100EF000003F0001003E0000003E0001003D0000F8
:100F0000003D0001003C0000003C0000003C0001EE
:100F1000003B0000003B0001003A0000003A0001E5
:100F200000390000003900010038000000380000DE
:100F300000380001003700000037000100360000D3
:100F400000360000003600010035000000350000CA
:100F500000350001003400000034000000340001BE
:100F600000330000003300000033000100320000B5
:100F700000320000003200010031000000310000AA
:100F8000003100010030000000300000003000019E
:100F9000002F0000002F0000002F0000002F000194
:100FA000002E0000002E0000002E0001002D000089
:100FB000002D0000002D0000002D0001002C00007D
:100FC000002C0000002C0000002C0001002B000071
:100FD000002B0000002B0000002B0001002A000065
:100FE000002A0000002A0000002A00010029000059
:100FF000002900000029000000290000002900014C
:101000000028000000280000002800000028000040
:101010000028000100270000002700000027000032
:101020000027000000270001002600000026000025
:101030000026000000260000002600010025000018
:10104000002500000025000000250000002500000C
:1010500000250001002400000024000000240000FE
:1010600000240000002400010023000000230000F1
:1010700000230000002300000023000000230000E4
:1010800000230001002200000022000000220000D6
:1010900000220000002200000022000100210000C8
:1010A00000210000002100000021000000210000BC
:1010B00000210000002100010020000000200000AD
:1010C00000200000002000000020000000200000A0
:1010D0000020000000200001001F0000001F000091
:1010E000001F0000001F0000001F0000001F000084
:1010F000001F0001001E0000001E0000001E000076
:10110000001E00000024F4D43050C38E20C2A24040
:1011100017828B7011127A910D816CD90AA861E146
:1011200008C7586607615143061E4B5D05C145A7B8
:10113000041A411104093D9803713931034036DB2B
:101140000265339102D4305402802E1D02632CEECE
:1011500001752AC501B028A001102781018F2564DF
:10116000012B244B01E0223401AC211F018D200D05
:1011700001801FFC00841EED00971DDF00B81CD20B
:1011800000E61BC600201BBC00641AB200B219A8FE
:10119000000A19A0006A189900D117910040178B16
:1011A00000B516840031167E00B31579003A157328
:1011B00000C7146F0058146A00EE136600881363AA
:1011C0000025135E00C7125B006C12570015125405
:1011D00000C111510070114F0021114B00D6104970
:1011E000008D1047004610440002104200C00F401E
:1011F00000800F3E00420F3C00060F3B00CB0E3834
:1012000000930E37005C0E3500270E3400F30D32CC
:1012100000C10D3100900D3000600D2E00320D2DFB
:1012200000050D2C00D90C2B00AE0C2900850C29D3
:10123000005C0C2700350C27000E0C2600E80B2460
:1012400000C40B2400A00B23007D0B23005A0B21AC
:1012500000390B2100180B2000F80A1F00D90A1EC4
:1012600000BB0A1E009D0A1D00800A1D00630A1CA7
:1012700000470A1B002C0A1B00110A1A00F7091A62
:1012800000DD091900C4091900AB091900920917FA
:10129000007B091800630917004C0916003609166F
:1012A00000200916000A091500F5081500E00814C9
:1012B00000CC081400B8081400A408140090081307
:1012C000007D0812006B081300580812004608122F
:1012D0000034081100230811001208110001081140
:1012E00000F0071000E0071000D0071000C0071042
:1012F00000B0070F00A107100091070E0083070F31
:101300000074070F0065070E0057070E0049070E0F
:10131000003B070D002E070E0020070D0013070DE0
:101320000006070D00F9060C00ED060D00E0060CA6
:1013300000D4060C00C8060C00BC060C00B0060C5D
:1013400000A4060B0099060C008D060B0082060B0C
:101350000077060B006C060B0061060A0057060BAF
:10136000004C060A0042060A0038060A002E060A49
:101370000024060A001A060A001006090007060AD9
:1013800000FD050900F4050900EB050900E2050967
:1013900000D9050900D0050900C7050900BE0509E7
:1013A00000B5050800AD050800A50509009C050865
:1013B00000940508008C050800840508007C0508D9
:1013C00000740508006C050700650508005D050749
:1013D00000560508004E05070047050700400508B0
:1013E0000038050700310507002A05070023050717
:1013F000001C050600160507000F05070008050676
:101400000002050700FB040600F5040700EE0406D1
:1014100000E8040600E2040700DB040600D5040629
:1014200000CF040600C9040600C3040600BD04067C
:1014300000B7040600B1040500AC040600A60406CB
:1014400000A00405009B0406009504050090040616
:10145000008A04050085040500800406007A04055E
:101460000075040500700405006B040500660405A2
:1014700000610405005C04050057040500520405E2
:10148000004D04050048040500430405003E040423
:10149000003A04050035040500300404002C04055E
:1014A0000027040400230405001E0404001A040499
:1014B0000016040500110404000D040400090405CD
:1014C000000404040000040400FC030400F8030406
:1014D00000F4030400F0030400EC030400E8030438
:1014E00000E4030400E0030400DC030400D8030468
:1014F00000D4030400D0030400CC030400C8030399
:1015000000C50303006563686F3A00205A3A002063
:10151000593A0020583A00656E6473746F707320F6
:101520006869743A20004572726F723A0054656DB2
:101530007065726174757265206865617465642098
:10154000626564207377697463686564206F66669A
:101550002E204D415854454D50207472696767657F
:10156000726564202121003A2045787472756465A3
:1015700072207377697463686564206F66662E20D5
:101580004D494E54454D50207472696767657265C8
:10159000642021003A204578747275646572207366
:1015A00077697463686564206F66662E204D4158C4
:1015B00054454D50207472696767657265642021D7
:1015C00000202D20496E76616C6964206578747204
:1015D00075646572206E756D626572202100000071
:1015E0000000300E0100C00E0A00500F1400D00F92
:1015F0001E0060102800E010320070113C00F01155
:1016000046007012500000135A008013640000144A
:101610006E00901478001015820090158C00101642
:1016200096009016A0001017AA009017B40010188A
:10163000BE009018C8001019D2009019DC00101AD2
:10164000E600801AF000001BFA00801B0401F01B6A
:101650000E01701C1801F01C2201601D2C01E01D00
:101660003601501E4001D01E4A01401F5401B01FD8
:101670005E0130206801A020720110217C019021C0
:101680008601002290016026F401902A5802802EE3
:10169000BC0250322003E03584035039E803803C1B
:1016A0004C04504944204175746F74756E65206612
:1016B000696E69736865642120507574207468656B
:1016C000204B702C204B6920616E64204B6420639A
:1016D0006F6E7374616E747320696E746F20436FE4
:1016E0006E66696775726174696F6E2E6800504925
:1016F00044204175746F74756E65206661696C6510
:1017000064212074696D656F75740020403A006F24
:101710006B20543A006F6B20423A005049442041FC
:1017200075746F74756E65206661696C65642120DF
:1017300054656D706572617475726520746F6F2089
:101740006869676800204B643A2000204B693A20A2
:1017500000204B703A200020436C61736963205075
:10176000494420002054753A2000204B753A20004F
:10177000206D61783A2000206D696E3A2000206467
:101780003A200020626961733A20004D41494E546D
:10179000454E414E4345004D4154455249414C0050
:1017A0005052494E54005072696E74696E672077CA
:1017B000697468205553422E2E2E00737570706F19
:1017C000727440756C74696D616B65722E636F6DB8
:1017D00000436F6E746163743A0053616665747997
:1017E00020636972637569740054656D7020736558
:1017F0006E736F72204245440054656D70207365AE
:101800006E736F72004552524F52202D2053544F29
:101810005050454400801506060606FEFEFEFEFCFE
:1018200000000000000000FCFEFEFEFC0000000EB8
:10183000FEFEFEFE0000E0FCFEFEFCE0E00000001C
:10184000CECECE000000C0C0C0C0C0C0800000002E
:1018500000000080C0C0800000000000008080C048
:10186000C0C0C0C0C0C080800000000006FEFEFEF8
:10187000FE0000000080C0C0C0000000000000802A
:1018800080C0C0C080808000000000C0C0C0C00018
:1018900080C0C0C0C08000000000007FFFFFFFFFCD
:1018A00080000000000080FFFFFFFFFF000000003D
:1018B000FFFFFFFF000000FFFFFFFF000000000030
:1018C000FFFFFF00000081F1FFFF3F0F3FFFFCF033
:1018D000F0FCFF3F0F3FFFFEF880000000C1E1F188
:1018E000F17131010183FFFFFFFC000000FFFFFFEA
:1018F000FF000C3EFFFFF7C301000000FCFEFF8766
:1019000003113131333F3F3F1E000001FFFFFFFF56
:1019100007030101010100000000000001030707A7
:101920000F0F0F0F0F0F0F0707070F0F0600000015
:10193000070F0F07000000070F0F0700000000004F
:101940000F0F0F0000060F0F070100000001070F27
:101950000F070100000001070F0F06000003070F2B
:101960000F0E0E060703070F0F07000000070F0FEB
:101970000700000000030F0F0F0600000003070719
:101980000F0E0E0E0E0E0E06000000000F0F0F0FB2
:10199000000000000000008015090909F90101019B
:1019A0000103FE0000000000FE0301010103FE0030
:1019B0001FF101010101FFF01E030101031E10F0E0
:1019C00000FF313131FF00E020202020202060C0C6
:1019D00080000080C060202060C000000000C04087
:1019E00060202020202020206040C080000FF901CE
:1019F000010101FF0080C060202020E00000008085
:101A0000C04060202020604040C08000E0202020B6
:101A100020E0602020202060C0000000FF80000047
:101A200000007FC0808080C07F0000000000FF00B9
:101A300000FF00000000FF01FF00000000FF0101A7
:101A400000FF000000FF00C37A0E0000C070C0005D
:101A5000030E0E0300C070C00001077CC000E3321B
:101A60001A0A0A8ACAFAC67C00000003FE00FF00B8
:101A7000000000FF73C10000083CE68300FE030184
:101A80000078FCEE4A4E4C404040613F03FE0000AF
:101A90000000F80C06020202030000000003060C1E
:101AA0000818101010101010101808181010190F26
:101AB000000F181010180F000F181010180F00004A
:101AC000001F1010101F0F191010180E0300030E26
:101AD000181010180E0300030E181010190F070C21
:101AE000181010111119080C181010180F000F18E9
:101AF0001010180F0001071C101010190F01070C0F
:101B0000081810111111111111190F00001F1010D8
:101B100010101F0000000000002F40000000000017
:101B200000000000000000808080C0E0FEFF191E61
:101B30009898981818181818189E9F991E38F0E051
:101B40000000000000000000000000000000000095
:101B50000000003CFEFFFF99F1E1C3FFFF000063BE
:101B600063636060606060606363630000FFFF7CCC
:101B700038000000000000000000000080C060B0DD
:101B8000D8D81CFCFF3F0F8FCFC7C7C7C6C6C6C675
:101B9000C6C6C6C6C6C6C6C6C6C6C6C6C7C7C4CCDF
:101BA0000C1CF8F870C00000000EFFF92A2B2B283F
:101BB00028FCFFFF0000FFFFFFFFFFFFFFBFB7177D
:101BC000B5BDB500B5B5F717FFBFBFFFFFFFFF00FD
:101BD00000FFFFFCFF0700C0F0FFFFFDDD1D19192E
:101BE0003FFFFF0000FFFFFFFFFFFFFFFBF1FBFBDD
:101BF000EAEEC0EEEAFAF0FAFAFFFFFFFFFF00009C
:101C0000FFFF0F1FF8E00003070F0F1B1819FBFE63
:101C1000FFFFF0E0C0C1E1F1F1F1F1F1F1F1F1F11B
:101C2000F1F1F9F9F9F9F9F9797979F1F010181F69
:101C3000070603030000000000000000F8FFEFDFCC
:101C4000BF7FFFFFFF404143437F212020217FFFD3
:101C5000FFFF3FB091D1DFD050581F1FF0F00000C0
:101C60000000000000000000000003070F1E3D7B85
:101C700077EED1DEDECF4B4B6969686868603F3F25
:101C8000373737353430101018181A1B0F0600007C
:101C9000000000100FFC0E0FCFCFCFCECCCCCCCCA1
:101CA000CCCCDCC0C007707E7F7F7F7F7F7F7F7F53
:101CB0007F7F7F0F017120FFFFFFFFFFFFFFFFFF0F
:101CC000FFFCE000000000000000000000E0FCFF5E
:101CD000FFFFFFFFFFFFFFFFFF000000000000000D
:101CE00000000000000000000000000000000000F4
:101CF000000000FFFFFFFFFFFFFF000000000000EB
:101D000000000000000000000000000000000000D3
:101D100000000000000000000000000000000000C3
:101D20000000000000000000FFFFFFFFFFFFFF7F3B
:101D3000FFFFFFFFFFF8800000000080F0FFFFFFC3
:101D4000FFFF3FFFFFFFFFFFFFFF00000030F8F83D
:101D5000FCFC7E7E7E3E3E3E3E7E7EFEFEFCFCF831
:101D6000E0800000FFFFFFFFFFFFFF000080C0E0FA
:101D7000F0F8FCFEFE7E3E1E0E06C0E0F0F8FCFC15
:101D8000FE7E3E3E3E3E3E7EFEFCFCF8F0C0800005
:101D900000FEFEFEFEFEFEFEFEFFFFFFFFFFFFFF5A
:101DA00000031FFFFFFFFFFFFCE0E0FCFFFFFFFF62
:101DB000FF1F0100FFFFFFFFFFFFFF0000C0E0F07B
:101DC000F0F8F8FC7C7C3C3C3E1E1E1EFFFFFFFF33
:101DD000FFFFFF0000FFFFFFFFFFFFFFFEFFFFFF12
:101DE000FFFFFFFFF1C080000000FFFFFFFFFFFFCC
:101DF000FF3C3C3C3C3C3C3C3C3C3F3F3F3F3F3F4E
:101E000000000000000000000000FFFFFFFFFFFFD8
:101E1000FF00000000073FFFFFFFFFFFFFFFFF3F46
:101E20000700000000FFFFFFFFFFFFFF00003F7FF4
:101E3000FFFFFFFFFCFCF8F8F87C7C3C3EFFFFFF57
:101E4000FFFFFFFF0000FFFFFFFFFFFFFF03010099
:101E50000003071F7FFFFFFFFEFCF0E38F1F3F3FE4
:101E60007F7FFEFCF8F8F0F0F0F8F8FCFC7E7E3C9A
:101E7000300000FEFEFEFEFEFEFEFE43414E4345E8
:101E80004C002073656300206D696E0020686F75DB
:101E9000720020686F75727300000000000000007F
:101EA0005F00000007000700147F147F14242A7FBE
:101EB0002A12231308646236495522500005030094
:101EC00000001C2241000041221C00082A1C2A0894
:101ED00008083E08080050300000080808080800FC
:101EE0006060000020100804023E5149453E004257
:101EF0007F400042615149462141454B311814123F
:101F00007F1027454545393C4A494930017109054B
:101F1000033649494936064949291E00363600002C
:101F20000056360000000814224114141414144101
:101F3000221408000201510906324979413E7E11FE
:101F400011117E7F494949363E414141227F41413D
:101F5000221C7F494949417F090901013E41415104
:101F6000327F0808087F00417F41002040413F0147
:101F70007F081422417F404040407F0204027F7F5F
:101F80000408107F3E4141413E7F090909063E4158
:101F900051215E7F09192946464949493101017F8E
:101FA00001013F4040403F1F2040201F7F2018205C
:101FB0007F631408146303047804036151494543A3
:101FC00000007F4141020408102041417F000004CD
:101FD000020102044040404040000102040020543D
:101FE0005454787F48444438384444442038444466
:101FF000487F3854545418087E0901020814545478
:102000003C7F0804047800447D40002040443D00AB
:10201000007F10284400417F40007C041804787C35
:102020000804047838444444387C14141408081410
:1020300014187C7C080404084854545420043F4479
:1020400040203C4040207C1C2040201C3C40304034
:102050003C44281028440C5050503C4464544C4498
:10206000000836410000007F0000004136080008EB
:10207000082A1C08081C2A08086275696C64706CC0
:102080006174652E006F662061646A757374696E91
:102090006720796F75720074726F75676874207449
:1020A00068652070726F6365737300492077696C8F
:1020B0006C20677569646520796F7500434F4E54D5
:1020C000494E554500473120462569205A2569204B
:1020D0005825692059256900473238205A30205840
:1020E000302059300066726F6D207468652062750B
:1020F000696C64706C6174652E0061206D696C6C34
:10210000696D65746572206177617900756E7469B7
:102110006C20746865206E6F7A7A6C652069730034
:10212000526F746174652074686520627574746F91
:102130006E00342F323100434F4E54494E55450006
:10214000434F4E54494E554500473120462569209E
:102150005A300047312046256920582569205925E5
:102160006900473120462569205A350066726F6D37
:1021700020746865206275696C64706C6174652E8A
:102180000069732061206D696C6C696D657465729E
:1021900020617761790073637265772074696C6C74
:1021A00020746865206E6F7A7A6C65005475726E63
:1021B000206C656674206275696C64706C6174650E
:1021C00000352F323100434F4E54494E554500479C
:1021D0003120462569205A300047312046256920A4
:1021E0005825692059256900473120462569205A1C
:1021F000350066726F6D20746865206275696C6465
:10220000706C6174652E0069732061206D696C6C5F
:10221000696D6574657220617761790073637265B9
:10222000772074696C6C20746865206E6F7A7A6CA4
:1022300065005475726E20726967687420627569F2
:102240006C64706C61746500362F323100434F4E00
:1022500054494E554500746865206275696C647018
:102260006C617465206C6576656C2E0070617065BC
:102270007220746F2066696E652D74756E65006ED0
:102280006F77207573652061207368656574206FB2
:102290006600526570656174207468697320737498
:1022A00065702C2062757400372F323100434F4E19
:1022B00054494E554500473120462569205A300083
:1022C000473120462569205825692059256900474E
:1022D0003120462569205A35006269742072657381
:1022E000697374616E63652E00756E74696C207914
:1022F0006F75206665656C2061006275696C64703D
:102300006C61746520616E64206E6F7A7A6C650012
:10231000536C69646520612070617065722062652C
:10232000747765656E00382F323100434F4E544943
:102330004E554500434F4E54494E5545007468650F
:10234000206C65667420636F726E65722E2E2E008F
:10235000526570656174207468697320666F7200DD
:10236000392F323100434F4E54494E554500746861
:102370006520726967687420636F726E65722E2EB5
:102380002E00526570656174207468697320666FF1
:10239000720031302F323100434F4E54494E554573
:1023A00000444F4E4500746F20696E73657274204F
:1023B0006D6174657269616C2E00746865206E656C
:1023C0007874207374657020697300746865206286
:1023D00075696C64706C617465004E6F7720746809
:1023E0006174207765206C6576656C6564003131B9
:1023F0002F323100434F4E54494E5545004731204E
:102400004631323030302058313130205930006D73
:102410006174657269616C206C6F6164696E6700DC
:102420007072696E74686561642068656174696E54
:102430006720666F7200506C656173652077616913
:10244000742C0031322F32310061626F7665207456
:102450006865206172726F772E00796F75722055F2
:102460006C74696D616B6572322C0066726F6D20E1
:102470007468652072656172206F6600496E7365CD
:102480007274206E6577206D6174657269616C008D
:1024900031332F323100434F4E54494E5545004C95
:1024A0006F6164696E67206D6174657269616C2E1D
:1024B0002E2E0031342F32310066726F6D206E6F18
:1024C0007A7A6C652E2E2E006D6174657269616C6E
:1024D0002065786974730050757368206275747430
:1024E0006F6E207768656E0031352F323100434FB3
:1024F0004E54494E554500556C74696D616B65725B
:10250000322E00696E73657274656420696E207482
:10251000686520006D6174657269616C20796F7502
:102520002068617665004E6578742C2073656C6553
:102530006374207468650031362F32310052454192
:1025400044590031372F32310041425300504C4141
:1025500000697320746869732072696768743F004A
:10256000414253206173206D6174657269616C2C06
:1025700000596F7520686176652063686F73656EBA
:102580000031382F3231004E4F00594553006974E5
:10259000206973207573696E672E006F66206D6108
:1025A00074657269616C006B6E6F77732077686118
:1025B00074206B696E64004E6F7720796F7572209E
:1025C000556C74696D616B6572320031392F32312F
:1025D00000434F4E54494E5545006D616B65206177
:1025E000203344205072696E74210049276D207297
:1025F00065616479206C657427730032302F323145
:102600000041524520594F552052454144593F0001
:10261000746F207072696E742069742100616E6439
:102620002070726573732074686520627574746FAE
:102630006E006F6E207468652053442D6361726470
:102640000053656C6563742061207072696E74203C
:1026500066696C650032312F3231004C4554275386
:10266000205052494E540052656164696E67206380
:102670006172642E2E2E0032312F323100796F7547
:102680007220556C74696D616B6572322E2E2E004E
:10269000746861742063616D6520776974680050A7
:1026A0006C6561736520696E736572742053442D87
:1026B000636172640032312F3231006973207468B3
:1026C00069732072696768743F00504C41206173E0
:1026D000206D6174657269616C2C00596F7520689A
:1026E0006176652063686F73656E0031382F323113
:1026F000004E4F0059455300473238205A3000628F
:102700007574746F6E20746F20636F6E74696E756C
:102710006500556C74696D616B657221205072653E
:102720007373207468650073746172747570206FC0
:102730006620796F75720057656C636F6D652074E4
:102740006F2074686520666972737400312F3231AE
:1027500000434F4E54494E554500612066697273DF
:10276000742072756E2077697A6172642E007761C9
:102770006C6B20796F75207468726F75676800667E
:102780006972737420737461727475702049207754
:10279000696C6C0042656361757365207468697368
:1027A0002069732074686500322F323100434F4E28
:1027B00054494E554500473120462569205A256920
:1027C00000473238205A3000676F696E6720746F97
:1027D00020646F2074686174206E6F772E006164CE
:1027E0006A7573746D656E74732C207765206172E1
:1027F00065007765206E65656420746F20646F20C6
:10280000736F6D65004166746572207472616E73DA
:10281000706F72746174696F6E00332F32310043D0
:102820004F4E54494E554500473120462569205AA0
:1028300025692058256920592569004732382058D4
:1028400030205930004300432F00436C69636B20F4
:10285000746F2072657475726E004275696C647075
:102860006C6174652074656D702E3A005245545544
:10287000524E00414456414E434544004255494C56
:10288000442D7C504C415445004731205A3430008F
:10289000473238205A3000473238205A3000473209
:1028A0003820583020593000414456414E43454469
:1028B00000746F2064656661756C743F00526573C7
:1028C00065742065766572797468696E67004E4F2D
:1028D000005945530056657273696F6E2031332E6F
:1028E00031320044656320313620323031332031BB
:1028F000353A30383A30300052657475726E006D7A
:102900006D2F736563004D61782073706565642079
:102910005A006D6D2F736563004D6178207370658B
:1029200065642059006D6D2F736563004D617820DB
:1029300073706565642058006D6D2F736563005872
:102940002F59204A65726B0030306D6D2F736563AF
:102950005E3200416363656C65726174696F6E001D
:102960004D4F54494F4E006D6D2F736563006D6D73
:102970002F736563006D6D2F736563006D6D2F732D
:102980006563006D6D2F7365635E32003F3F3F00EE
:102990004D6178207370656564205A004D61782020
:1029A00073706565642059004D61782073706565AA
:1029B00064205800582F59204A65726B00416363A8
:1029C000656C65726174696F6E003C2052455455A8
:1029D000524E006D6D2F73656300526574726163B2
:1029E00074207370656564006D6D0052657472616A
:1029F0006374206C656E677468005245545241439D
:102A000054494F4E006D6D2F736563006D6D003F2F
:102A10003F3F005265747261637420737065656432
:102A20000052657472616374206C656E677468002F
:102A30003C2052455455524E004300432F00436CF6
:102A400069636B20746F2072657475726E00526FCB
:102A50007461746520746F206578747275646500A4
:102A60004E6F7A7A6C652074656D706572617475ED
:102A700072653A004300432F00436C69636B207416
:102A80006F2072657475726E004E6F7A7A6C652075
:102A900074656D70657261747572653A00250042E7
:102AA00072696768746E657373004C454400250055
:102AB0003F3F3F0020476C6F77207768656E20644A
:102AC0006F6E6500204F6E207768696C65207072AC
:102AD000696E74696E670020416C77617973204F6D
:102AE00066660020416C77617973204F6E004272F8
:102AF000696768746E657373003C20524554555283
:102B00004E003F3F3F00466163746F7279207265EB
:102B10007365740056657273696F6E004D6F7469EA
:102B20006F6E2073657474696E677300526574729A
:102B3000616374696F6E2073657474696E67730086
:102B40004D6F7665206D6174657269616C005261CC
:102B5000697365206275696C64706C617465004CA2
:102B60006F776572206275696C64706C6174650062
:102B7000486F6D65206865616400486561747570B3
:102B8000206275696C64706C61746500486561747D
:102B90007570206E6F7A7A6C65004C4544207365C1
:102BA0007474696E6773003C2052455455524E0050
:102BB00041425300504C410052455455524E00532F
:102BC000455454494E4753004348414E4745004DF4
:102BD0004154455249414C0053656C6563746564CA
:102BE000206D6174657269616C3A004F4B0025007D
:102BF0004D6174657269616C20666C6F77002500A9
:102C000046616E207370656564006D6D004D617482
:102C1000657269616C204469616D65746572004319
:102C2000004275696C64706C6174652054656D70E8
:102C30002E00430054656D70657261747572650095
:102C40004D4154455249414C00505245534554530F
:102C5000004E657720707265736574003C205245A4
:102C60005455524E00250025006D6D004300430071
:102C70003F3F3F0053746F7265206173207072652F
:102C800073657400466C6F7720250046616E0044C2
:102C900069616D6574657200486561746564206280
:102CA00075696C64706C6174650054656D706572F3
:102CB0006174757265003C2052455455524E004D6A
:102CC0006F64696679207468652073657474696ED1
:102CD000677300250046616E3A20004300430025DB
:102CE00000466C6F773A006D6D00437573746F6DBD
:102CF000697A65003C2052455455524E00666F7209
:102D0000206D6174657269616C2072656D6F7661AA
:102D10006C0048656174696E67207072696E7468D2
:102D200065616400473238205830205930005265C0
:102D300076657273696E67206D6174657269616C26
:102D40000052656D6F7665206D6174657269616CA6
:102D50000043414E43454C005245414459004731E0
:102D600020462569205825692059256900473238B1
:102D70002058302059300061626F76652074686594
:102D8000206172726F772E00796F7572206D6163AA
:102D900068696E652C0066726F6D207468652062CC
:102DA00061636B73696465206F6600496E73657259
:102DB00074206E6577206D6174657269616C004383
:102DC000414E43454C00524541445900466F72778D
:102DD000617264696E67206D6174657269616C000F
:102DE000636F6D6573206F757420746865206E6FF6
:102DF0007A7A6C6500576169742074696C6C206D17
:102E00006174657269616C0043414E43454C0052E8
:102E100045414459004300432F00436C69636B20D4
:102E2000746F2072657475726E004E6F7A7A6C657D
:102E30002074656D70657261747572653A005344F3
:102E40002043415244004731204631323030302057
:102E500058352059313000473238003B464C4156F6
:102E60004F523A556C746947436F6465003B464C5A
:102E700041564F523A556C746947436F6465004E32
:102E80006F2066696C657320666F756E6421004FF4
:102E90004B004F4B0052656164696E67206361723D
:102EA000642E2E2E00506C6561736520696E73650B
:102EB00072742063617264004E6F2053442D43414D
:102EC000524421003C204241434B003C2052455497
:102ED00055524E0066726F6D2074686520736C6980
:102EE0006365722E0073657474696E672077697408
:102EF000682073657474696E67006F7665727269B5
:102F00006465206D616368696E650054686973204B
:102F100066696C652077696C6C0043414E43454C93
:102F200000434F4E54494E55450047323800473113
:102F30002046313530302045300047393220452594
:102F40006900436F64653A0053442D6361726421E4
:102F50000072656164696E67004572726F722077F6
:102F600068696C650052455455524E20544F204DAF
:102F700041494E00746865207072696E742E005964
:102F80006F752063616E2072656D6F76650050729B
:102F9000696E742066696E697368656400430050E9
:102FA00072696E74657220636F6F6C696E672064FE
:102FB0006F776E004241434B20544F204D454E5594
:102FC0000054696D65206C6566740054696D6520F8
:102FD0006C65667420756E6B6E6F776E0043004390
:102FE0000048656174696E67206275696C64706C15
:102FF000617465004300430048656174696E670051
:103000005072696E74696E673A0041424F525400C3
:1030100054554E450041626F72742074686520708B
:1030200072696E743F004E4F0059455300250042AF
:1030300072696768746E6573730025004D6174650D
:103040007269616C20666C6F7700250046616E20A6
:1030500073706565640025005072696E742073702A
:103060006565640054554E45006D6D2F73656300B2
:1030700052657472616374207370656564006D6D70
:103080000052657472616374206C656E67746800C9
:1030900052455452414354494F4E006D6D2F736554
:1030A00063006D6D003F3F3F005265747261637451
:1030B0002073706565640052657472616374206C7E
:1030C000656E677468003C2052455455524E002589
:1030D0000025002500430043004300430025004C29
:1030E0004544204272696768746E65737300526567
:1030F0007472616374696F6E004D617465726961A9
:103100006C20666C6F770046616E20737065656435
:10311000004275696C64706C6174652074656D70D3
:103120002E0054656D706572617475726500537020
:10313000656564003C2052455455524E00507265FE
:10314000706172696E6720746F207072696E743A74
:103150000048656174696E672075702E2E2E0041DF
:10316000424F52540054554E45004E6F20696E66D2
:103170006F20617661696C61626C65006D006D0045
:103180004D6174657269616C3A200054696D653AED
:1031900020003B4D4154455249414C3A003B544973
:1031A0004D453A00466F6C64657200494E46494E83
:1031B0004954594E414ECDCCCC3D0AD7233C17B78C
:1031C000D13877CC2B329595E6241FB14F0A0000F9
:1031D00020410000C84200401C4620BCBE4CCA1B17
:1031E0000E5AAEC59D74D32F5455CE2F11241FBE39
:1031F000CFEFD1E2DEBFCDBF00E00CBF14E0A0E016
:10320000B2E0E2EEF9EB01E00BBF02C007900D92D5
:10321000A232B107D9F715E1A2E2B4E001C01D92D4
:10322000A53DB107E1F711E3CAEED1E304C022974F
:10323000FE010E94E1DCC63ED107C9F704D00C9420
:10324000D4D30C940000CF93DF9332D10E94465226
:10325000C0E0D0E00E94BD512097E1F30E94000041
:10326000F9CFCF92DF92EF92FF920F931F93CF93FC
:10327000DF937C016B018A01C0E0D0E00FC0D60172
:103280006D916D01D701ED91FC910190F081E02DE0
:10329000C7011995C80FD91F01501040011511051C
:1032A00071F7CE01DF91CF911F910F91FF90EF90B9
:1032B000DF90CF9008958230B9F0833028F48823CE
:1032C00051F0813051F50AC0843011F18430E8F0BA
:1032D000853019F520C010926E00089580916F001E
:1032E0008D7F80936F000895809170008D7F809313
:1032F000700081E08093B0008091B100887F84608D
:103300008093B1001092B300089510927100089557
:103310001092720008951092730008951F93182F51
:1033200080913B03811711F09FEF06C0EFE2F1E0BF
:1033300094918FEF80933B03892FBDDF812F60E055
:10334000AAD21F9108951F920F920FB60F920BB63B
:103350000F9211242F933F934F935F936F937F931B
:103360008F939F93AF93BF93EF93FF93809122042A
:1033700090912304A0912404B09125040097A10505
:10338000B10551F1E0912604F091270480819091DC
:103390002804892780838091220490912304A0919E
:1033A0002404B0912504181619061A061B06BCF44D
:1033B0008091220490912304A0912404B0912504CB
:1033C0000197A109B1098093220490932304A0934B
:1033D0002404B093250403C080913B039FDFFF9139
:1033E000EF91BF91AF919F918F917F916F915F917D
:1033F0004F913F912F910F900BBE0F900FBE0F90EA
:103400001F9018951F920F920FB60F9211242F93B1
:103410003F938F939F93AF93BF9380912D0490918F
:103420002E04A0912F04B091300430913104019604
:10343000A11DB11D232F2D5F2D3720F02D57019693
:10344000A11DB11D2093310480932D0490932E046F
:10345000A0932F04B09330048091290490912A0402
:10346000A0912B04B0912C040196A11DB11D809355
:10347000290490932A04A0932B04B0932C04BF91A9
:10348000AF919F918F913F912F910F900FBE0F9011
:103490001F9018958FB7F89420912D0430912E0429
:1034A00040912F04509130048FBFB901CA01089593
:1034B000789484B5826084BD84B5816084BD85B50F
:1034C000826085BD85B5816085BDEEE6F0E08081D6
:1034D00081608083E1E8F0E01082808182608083F7
:1034E000808181608083E0E8F0E08081816080837A
:1034F000E1EBF0E0808184608083E0EBF0E08081AC
:1035000081608083E1E9F0E0808182608083808156
:1035100081608083E0E9F0E0808181608083E1EA7E
:10352000F0E0808182608083808181608083E0EA36
:10353000F0E0808181608083E1E2F1E0808182605F
:103540008083808181608083E0E2F1E0808181601E
:103550008083EAE7F0E080818460808380818260FC
:1035600080838081816080838081806880831092E5
:10357000C10008951F93CF93DF93182FEB0161E0F3
:10358000D7D0209709F4CAC0CF3FD10509F4C9C0EC
:10359000E12FF0E0E65FFD4F8491893009F466C0C9
:1035A0008A30B0F48430F1F1853040F4823059F142
:1035B000833070F5813009F0AEC020C0873009F447
:1035C00043C0883008F048C0863009F0A4C034C039
:1035D0008D3009F478C08E3038F48B3009F45AC03D
:1035E0008C3008F066C04CC0803109F480C0813155
:1035F00009F487C08F3009F08EC06FC084B5806831
:1036000084BDC7BD91C084B5806284BDC8BD8CC077
:1036100080918000806880938000D0938900C0935F
:10362000880082C080918000806280938000D09367
:103630008B00C0938A0078C08091B000806880932E
:10364000B000C093B30070C08091B00080628093DE
:10365000B000C093B40068C08091900080688093EF
:103660009000D0939900C09398005EC08091900024
:10367000806280939000D0939B00C0939A0054C0C6
:1036800080919000886080939000D0939D00C093BB
:103690009C004AC08091A00080688093A000809127
:1036A000A0008F7B8093A000D093A900C093A800B6
:1036B0003BC08091A00080628093A000D093AB00BB
:1036C000C093AA0031C08091A00088608093A000C0
:1036D000D093AD00C093AC0027C0809120018068DA
:1036E00080932001D0932901C09328011DC08091AF
:1036F0002001806280932001D0932B01C0932A0186
:1037000013C080912001886080932001D0932D0107
:10371000C0932C0109C0C038D1051CF4812F60E092
:1037200002C0812F61E0B7D0DF91CF911F91089542
:10373000CF93DF93482F50E0CA018C539E4FFC017A
:10374000349142585E4FFA018491882369F190E0E8
:10375000880F991FFC01E05DFE4FA591B491FC011B
:10376000E65BFE4FC591D491662351F42FB7F894D0
:103770008C91932F909589238C93888189230BC0FA
:10378000623061F42FB7F8948C91932F9095892330
:103790008C938881832B88832FBF06C09FB7F894B2
:1037A0008C91832B8C939FBFDF91CF9108958930AB
:1037B00009F449C08A30A0F4843051F1853040F4D6
:1037C000823079F1833000F5813009F063C026C082
:1037D000873079F1883098F5863009F05BC025C0D4
:1037E0008D3009F442C08E3028F48B30B1F18C302A
:1037F000C0F52DC0803109F442C0813109F445C0C3
:103800008F3009F047C037C0809180008F7703C0A8
:10381000809180008F7D80938000089584B58F779C
:1038200002C084B58F7D84BD08958091B0008F77EC
:1038300003C08091B0008F7D8093B0000895809187
:1038400090008F7707C0809190008F7D03C080919A
:103850009000877F8093900008958091A0008F77DB
:1038600007C08091A0008F7D03C08091A000877F5A
:103870008093A0000895809120018F7703C08091EC
:1038800020018F7D80932001089580912001877F02
:10389000809320010895FF920F931F93F62E482FD7
:1038A00050E0CA01865F9D4FFC012491CA018C53F0
:1038B0009E4FFC01149142585E4FFA01049100237F
:1038C000C1F0222311F0822F72DFE02FF0E0EE0F23
:1038D000FF1FE65BFE4FA591B4919FB7F894FF20C0
:1038E00021F48C911095812302C08C91812B8C93B3
:1038F0009FBF1F910F91FF900895AC01DB01FA016A
:1039000090E02EE28C91803229F0983009F42193D6
:103910008C9181939F5F11969B30A1F71082CA0111
:103920000895FC01128217A60895FC0187A588233B
:1039300011F081E082830895FC018281811112825D
:103940000895CF93DF93EC01FC01EA55FE4F80818F
:10395000882309F461C081508083DE01AB5ABF4FD8
:10396000FE01EC58FF4F8BE101900D928150E1F781
:10397000FE01ED5AFF4FCE58DF4F88819981C25723
:10398000D0409183808330E0BE016A557E4F3FC0B6
:10399000832F90E0AC014F5F5F4FDC01E5E0AA0FA1
:1039A000BB1FEA95E1F7A81BB90BAC0FBD1FFA01CD
:1039B00025E0EE0FFF1F2A95E1F7E41BF50BEC0F56
:1039C000FD1FAC58BF4FEC58FF4F2BE101900D92FB
:1039D0002150E1F7FC0125E0EE0FFF1F2A95E1F7EA
:1039E000E81BF90BEC0FFD1FEE58FF4FDA0185E0E5
:1039F000AA0FBB1F8A95E1F7A41BB50BAC0FBD1F27
:103A0000AE58BF4F8D919C91918380833F5FFB01A6
:103A10008081381708F4BCCFDF91CF910895FC0165
:103A20008AE194E0918380838781882321F0CF010C
:103A300004960C94CA7008950F931F938C010E94F2
:103A40003D7F0E94397EC80181539E4F0E94CA70FB
:103A5000F801128280E592E00E94D2531F910F91EB
:103A60000895CF92DF92EF92FF920F931F93DF930F
:103A7000CF93CDB7DEB76F970FB6F894DEBF0FBE0A
:103A8000CDBF8C016B01085A1F4FD8018C9108558E
:103A90001040882321F480E3E82EF12C03C0B1E527
:103AA000EB2EF12CE00EF11E8AE194E09A838983DB
:103AB0001C821B8218861D82B7016C5F7F4FCE016E
:103AC0000596A60121E00E940378882391F5ECE594
:103AD000F2E0949108C08091C00085FFFCCF9093E4
:103AE000C600319694919923B1F7E2E6F2E0949101
:103AF00008C08091C00085FFFCCF9093C60031962E
:103B000094919923B1F709C08091C00085FFFCCF43
:103B10000894C11CD11C9093C600F6019081992392
:103B200099F78091C00085FFFCCF8AE08093C600A2
:103B300056C0F801EA55FE4F80818A3008F03EC039
:103B40008F5F8083282F30E0C9010197FC01A5E039
:103B5000EE0FFF1FAA95E1F7E81BF90BEC58FF4F9A
:103B6000E00FF11F21503040AF01415E5F4FBF01B8
:103B70008BE1DB010D90BD01DA010D92AD018150A9
:103B8000C1F7929182913296968F858F7F972115FA
:103B9000310541F7D801AC58BF4FF70134968BE19E
:103BA00001900D928150E1F70E581F4FF70182816D
:103BB0009381D8018D939C9302571040D801AB5A42
:103BC000BF4FFE0135968BE101900D928150E1F7D8
:103BD0000D5A1F4F8B819C81F80191838083CE0108
:103BE00001961DDF6F960FB6F894DEBF0FBECDBFF6
:103BF000CF91DF911F910F91FF90EF90DF90CF90C9
:103C00000895EF92FF920F931F938C019FECE92E82
:103C100091E0F92EE00EF11EC7010E947B70C701F2
:103C20000E94CA70F801108211821F910F91FF90BB
:103C3000EF900895CF92DF92EF92FF920F931F9330
:103C4000CF93DF937C016B01DB010D900020E9F73E
:103C50008D0101501040061B170BEFECF1E0EE0E4A
:103C6000FF1ED7011C92E1E3FEEFEE0EFF1ECB011B
:103C70006EE470E00E947BD4EC01009731F4F8010F
:103C80003197EC0DFD1D86010EC060E270E00E94D0
:103C90007BD48C010F5F1F4FCE016AE270E00E945F
:103CA0007BD4FC0131978DE081838AE0828313828B
:103CB000C70185539E4FB8010E94FD788FEC91E0BB
:103CC000E80EF91ED7018C91882319F1ECE8F2E097
:103CD000949108C08091C00085FFFCCF9093C600EE
:103CE000319694919923B1F7E3E9F2E0949108C0F9
:103CF0008091C00085FFFCCF9093C60031969491CF
:103D00009923B1F78091C00085FFFCCF8AE08093B2
:103D1000C600DF91CF911F910F91FF90EF90DF9040
:103D2000CF900895CF93DF93EC018FA5882309F4FA
:103D30003DC0E7ECF2E0949108C08091C00085FF9F
:103D4000FCCF9093C600319694919923B1F7CE5051
:103D5000DE4F488159816A817B81C25FD14080EC0E
:103D600098E02AE030E00E94EB55E5ECF2E0949117
:103D700008C08091C00085FFFCCF9093C6003196AB
:103D800094919923B1F7C651DE4F488159816A81D8
:103D90007B81CA5ED14080EC98E02AE030E00E944E
:103DA000EB558091C00085FFFCCF12C0E5EBF2E03F
:103DB000949108C08091C00085FFFCCF9093C6000D
:103DC000319694919923B1F78091C00085FFFCCF83
:103DD0008AE08093C600C755DE4F68816623E1F014
:103DE000E9EAF2E0949108C08091C00085FFFCCF21
:103DF0009093C600319694919923B1F780EC98E0A6
:103E000070E04AE050E00E943A568091C00085FF81
:103E1000FCCF8AE08093C600DF91CF9108952F9266
:103E20003F924F925F926F927F928F929F92AF924A
:103E3000BF92CF92DF92EF92FF920F931F93DF9387
:103E4000CF93CDB7DEB7AD970FB6F894DEBF0FBEF8
:103E5000CDBF5C014B014DA7FC0187A5882309F468
:103E6000E1C13FEC432E31E0532E4A0C5B1CC201F2
:103E70000E94CA70F50112821A8A1D8A198A188A4C
:103E80008AE194E09F878E872FE4C22ED12CCA0C42
:103E9000DB1C80E390E0A80EB91EF601B182A0827F
:103EA00080ED9FEFA80EB91EF40180818F3209F0DA
:103EB0008DC0C4016FE270E00E947BD47C01089445
:103EC000E11CF11C3E010894611C711C160178C0B4
:103ED000C7016FE270E00E947BD46C01009709F487
:103EE00083C0E816F90608F07FC08C010E191F097F
:103EF000C301B701A8010E949BD4060D171DF8014C
:103F00001082F30107C08091C00085FFFCCF31967D
:103F10009093C60090819923B1F78091C00085FFEE
:103F2000FCCFFAE0F093C600F10160817181611568
:103F3000710519F460E070E002C06C5F7F4FCE0144
:103F40004296A30121E00E940378882371F5EBE7F4
:103F5000F3E0949108C08091C00085FFFCCF90935E
:103F6000C600319694919923B1F7FE01319607C0AE
:103F70008091C00085FFFCCF31969093C600908160
:103F80009923B1F7E9E7F3E0949108C08091C0006C
:103F900085FFFCCF9093C600319694919923B1F799
:103FA0008091C00085FFFCCF37C18EE090E08C0F80
:103FB0009D1FF1019183808376010894E11CF11C1F
:103FC00092E0E916F10408F083CF0BC0E1E5F0E0E0
:103FD000AE0EBF1EF601B182A0828FEA9FEFA80E3F
:103FE000B91E082DF92C01C00E2DF501E15BFF4F24
:103FF0009DA5992309F4ADC060817181611571059A
:1040000019F460E070E002C06C5F7F4FC201402F86
:104010005F2D21E00E940378882309F46AC0E0EE56
:10402000F1E0AE0EBF1EF5014081518162817381C6
:104030008AE090E0A80EB91EF501408351836283A7
:10404000738386E19EEFA80EB91EEBE6F3E0949130
:1040500008C08091C00085FFFCCF9093C6003196C8
:1040600094919923B1F7802F9F2D9C01F90107C0EE
:104070008091C00085FFFCCF31969093C60090815F
:104080009923B1F7E3E6F3E0949108C08091C00072
:1040900085FFFCCF9093C600319694919923B1F798
:1040A00080EC98E02AE030E00E94EB558091C0005F
:1040B00085FFFCCF8AE08093C600E2EFF1E0AE0E10
:1040C000BF1EF5011082118212821382E5E5F3E032
:1040D000949108C08091C00085FFFCCF9093C600EA
:1040E000319694919923B1F78091C00085FFFCCF60
:1040F00093C0E1E4F3E0949108C08091C00085FF93
:10410000FCCF9093C600319694919923B1F7802FFC
:104110009F2D9C01F90107C08091C00085FFFCCF55
:1041200031969093C60090819923B1F7EFE3F3E0C5
:10413000949108C08091C00085FFFCCF9093C60089
:10414000319694919923B1F78091C00085FFFCCFFF
:1041500063C0608171816115710519F460E070E0E0
:1041600002C06C5F7F4FC201402F5F2D26E50E9489
:104170000378882381F5EBE2F3E0949108C0809105
:10418000C00085FFFCCF9093C6003196949199238F
:10419000B1F7802F9F2D9C01F90107C08091C000CD
:1041A00085FFFCCF31969093C60090819923B1F79B
:1041B000E9E2F3E0949108C08091C00085FFFCCF54
:1041C0009093C600319694919923B1F78091C000E5
:1041D00085FFFCCF21C081E0F5018083E7E1F3E0BA
:1041E000949108C08091C00085FFFCCF9093C600D9
:1041F000319694919923B1F7F40107C08091C000E2
:1042000085FFFCCF31969093C60090819923B1F73A
:104210008091C00085FFFCCF8AE08093C600CE016C
:104220000E96FDDBAD960FB6F894DEBF0FBECDBF88
:10423000CF91DF911F910F91FF90EF90DF90CF9082
:10424000BF90AF909F908F907F906F905F904F90B6
:104250003F902F900895FC0181E08183CF0140E0E1
:10426000DECD2F923F924F925F926F927F928F920C
:104270009F92AF92BF92CF92DF92EF92FF920F93F5
:104280001F93DF93CF93CDB7DEB7AC970FB6F894FB
:10429000DEBF0FBECDBF5C014B01FC0187A58823AB
:1042A00009F437C1C50181539E4F0E94CA70F501C0
:1042B00012821A8A1D8A198A188A8AE194E09F87D5
:1042C0008E875FE4C52ED12CCA0CDB1C20E330E0C6
:1042D000A20EB31EF601B182A08220ED3FEFA20E26
:1042E000B31EF40180818F3209F090C0C4016FE2E7
:1042F00070E00E947BD47C010894E11CF11C3E011B
:104300000894611C711C260142E1242E312C2C0ED4
:104310003D1E77C0C7016FE270E00E947BD46C0144
:10432000009709F481C0E816F90608F07DC08C01F9
:104330000E191F09C301B701A8010E949BD4060DE5
:10434000171DF8011082F30107C08091C00085FF9E
:10435000FCCF31969093C60090819923B1F780915C
:10436000C00085FFFCCFFAE0F093C600F201608147
:1043700071816115710519F460E070E002C06C5F35
:104380007F4FC101A30121E00E940378882371F5CA
:10439000E3E0F3E0949108C08091C00085FFFCCF7A
:1043A0009093C600319694919923B1F7FE0131960E
:1043B00007C08091C00085FFFCCF31969093C60066
:1043C00090819923B1F7E1E0F3E0949108C08091E6
:1043D000C00085FFFCCF9093C6003196949199233D
:1043E000B1F78091C00085FFFCCF8DC02EE030E09A
:1043F0002C0F3D1FF2013183208376010894E11CCC
:10440000F11CE114F10409F085CF0BC081E590E0C7
:10441000A80EB91EF601B182A0822FEA3FEFA20ECC
:10442000B31ED82C092D02C0DE2C0F2D8FE490E096
:10443000A80EB91EF5018081918121EB3FEFA20EFC
:10444000B31E009719F480E090E001C004966D2D32
:10445000702F0E94CF78882339F1E3EFF2E0949136
:1044600008C08091C00085FFFCCF9093C6003196B4
:1044700094919923B1F78D2D902F9C01F90107C0DC
:104480008091C00085FFFCCF31969093C60090814B
:104490009923B1F782EF91E0A80EB91EF5011082C1
:1044A00011821282138232C0EBEDF2E0949108C0C7
:1044B0008091C00085FFFCCF9093C6003196949107
:1044C0009923B1F78D2D902F9C01F90107C08091A0
:1044D000C00085FFFCCF31969093C6009081992350
:1044E000B1F7E9EDF2E0949108C08091C00085FF3A
:1044F000FCCF9093C600319694919923B1F78091A7
:10450000C00085FFFCCF8AE08093C600CE010E96E6
:1045100086DAAC960FB6F894DEBF0FBECDBFCF9152
:10452000DF911F910F91FF90EF90DF90CF90BF90A0
:10453000AF909F908F907F906F905F904F903F9043
:104540002F900895EF92FF920F931F93CF93DF93D5
:104550008C01FC0117A687A9882321F0C801C49605
:104560000E94CA7068EAE62E61E0F62EE00EF11EA7
:10457000C70160E045E30E949E6E882309F5ECE5E3
:10458000F2E0949108C08091C00085FFFCCF909329
:10459000C600319694919923B1F7EDEBF3E0949135
:1045A00008C08091C00085FFFCCF9093C600319673
:1045B00094919923B1F78091C00085FFFCCF7DC015
:1045C000E801C355DE4FCE01B70141E00E949A7960
:1045D000882341F5CE01B70140E00E949A798823F3
:1045E00009F5ECE8F2E0949108C08091C00085FFE5
:1045F000FCCF9093C600319694919923B1F7EAEAE3
:10460000F3E0949108C08091C00085FFFCCF9093A7
:10461000C600319694919923B1F78091C00085FF2F
:10462000FCCF4BC0C801C496BE010E94A173882371
:1046300009F5ECE8F2E0949108C08091C00085FF94
:10464000FCCF9093C600319694919923B1F7EAE993
:10465000F3E0949108C08091C00085FFFCCF909357
:10466000C600319694919923B1F78091C00085FFDF
:10467000FCCF23C081E0F80187A7ECE5F2E094913C
:1046800008C08091C00085FFFCCF9093C600319692
:1046900094919923B1F7EFE8F3E0949108C08091E9
:1046A000C00085FFFCCF9093C6003196949199236A
:1046B000B1F78091C00085FFFCCF8AE08093C600EF
:1046C000D801AB5ABF4FF801F4968BE101900D92DF
:1046D0008150E1F7F80182A993A90D5A1F4FF80103
:1046E0009183808303551040C801C096015B1F4F22
:1046F000F80191838083DF91CF911F910F91FF90FB
:10470000EF9008952F923F924F925F926F927F9217
:104710009F92AF92BF92CF92DF92EF92FF920F9350
:104720001F93DF93CF93CDB7DEB7CC55D0400FB6F4
:10473000F894DEBF0FBECDBF6C01662311F526EFE6
:1047400031E0C20ED31ED6018C91EAE0FEEFCE0E10
:10475000DF1E882309F4E7C02EEE31E0C20ED31E1F
:10476000D601ED90FD900D911C91E2E1FEEFCE0E91
:10477000DF1E0E944A1AE616F7060807190708F412
:10478000D2C026EF31E0C20ED31ED6011C92EAE061
:10479000FEEFCE0EDF1ED6019F968C91882339F452
:1047A000C601D0DEF60187A5882309F4BCC000D07D
:1047B00000D0EDB7FEB731967E010894E11CF11CE4
:1047C000ADB7BEB71296FC92EE92119783E892E0D5
:1047D00093838283D6019D968D919C919E9795831C
:1047E00084830E94CAD48701EDB7FEB736960FB610
:1047F000F894FEBF0FBEEDBF570108C0D8018C91E1
:1048000090E00E94DFD3F80181938F01F5010190C0
:104810000020E9F73197EA19FB09802F8E198E17CE
:104820006CF3A4E3AA2EB12CAC0CBD1CC50140E076
:1048300050E060E070E00E94B16F9924FDE3EF2E3C
:10484000F12CEC0EFD1E2E010894411C511CEFE1D1
:104850006E2E712C6C0E7D1E7CE7272E72E0372E9B
:1048600042C0D8018C9190E00E94DFD3F80181937F
:104870008F01F70101900020E9F73197EE19FF0948
:10488000802F8E198E176CF327968FAD27978E3752
:1048900051F1C701B20145E050E00E948DD400976C
:1048A00011F500D000D0EDB7FEB73196ADB7BEB769
:1048B00012967C926E9211973382228255824482A4
:1048C0000E94CAD4EDB7FEB736960FB6F894FEBF75
:1048D0000FBEEDBFC3010E944B5488E792E00E94D7
:1048E000D25399249394C501B70140E050E00E944F
:1048F000C072181614F48701BCCF992041F48FEFD1
:104900009FEFD6019E969C938E939D9706C0F601CD
:1049100085A596A5019696A785A729EA31E0C20E3E
:10492000D31ED6011C92C45ADF4F0FB6F894DEBFD7
:104930000FBECDBFCF91DF911F910F91FF90EF90F0
:10494000DF90CF90BF90AF909F907F906F905F90DF
:104950004F903F902F9008952F923F924F925F92E9
:104960006F927F928F929F92AF92BF92CF92DF927F
:10497000EF92FF920F931F93DF93CF93CDB7DEB7E4
:10498000CD58D0400FB6F894DEBF0FBECDBF8C011E
:104990003B016A0184E090E0C80ED91EF8017196CF
:1049A000C757DF4FF983E883C958D040C801049640
:1049B000C957DF4F99838883C758D040CA57DF4F04
:1049C0001882C658D04036E6E32EF12CEC0EFD1EC0
:1049D00027EF822E21E0922E800E911E98EFA92EB5
:1049E00091E0B92EA00EB11E8EE0282E312C2C0E97
:1049F0003D1EB7E44B2E512C4C0E5D1EF201349639
:104A0000C557DF4FF983E883CB58D040ECE5F2E09F
:104A10008491C357DF4F8883CD58D04021C1F7011F
:104A20008385282F30E0A90148715070403151052D
:104A300009F024C1F4019081913009F41FC1923032
:104A400009F41CC1CE010196B7010E947D1C1E868F
:104A5000F3018081882329F4C10160E072E00E94A3
:104A600070D4C101B3010E9470D4C101BE016F5F57
:104A70007F4F0E9470D4C10160E072E00E9470D448
:104A80001CA61FA61BA61AA68AE194E099A788A7D0
:104A9000CE018C96B601AE014F5F5F4F21E00E94C0
:104AA0000378882309F03EC0F40180818823D1F582
:104AB000C357DF4F9881CD58D040ECE5F2E008C0F5
:104AC0008091C00085FFFCCF9093C60031969491F1
:104AD0009923B1F7E2E0F2E007C08091C00085FFC2
:104AE000FCCF31969093C60090819923B1F78091C5
:104AF000C00085FFFCCFFAE0F093C600FE013196BE
:104B000007C08091C00085FFFCCF31969093C6000E
:104B100090819923B1F78091C00085FFFCCF8AE096
:104B20008093C600C557DF4FA881B981CB58D040CC
:104B3000FE01BC968BE101900D928150E1F78AA5B0
:104B40009BA5F201938382838AE194E09183808321
:104B5000C801B101A20100DFC2010E940F1DCE01F8
:104B600088960E940F1D7CC0953E09F479C09E3244
:104B700009F476C09F3509F473C0F801918999232F
:104B800031F09E3209F46CC09F3509F469C023FDF1
:104B900067C080E04031510509F481E0F80184A745
:104BA000882349F4F7018085873409F059C081854D
:104BB0008E3709F455C0C957DF4F88819981C7588E
:104BC000D040B7010E947D1CF4018081882329F523
:104BD000F30107C08091C00085FFFCCF3196909310
:104BE000C60090819923B1F7C957DF4FE881F98159
:104BF000C758D04007C08091C00085FFFCCF3196D8
:104C00009093C60090819923B1F78091C00085FFF1
:104C1000FCCFFAE0F093C60023C0813039F4F501EF
:104C2000808191810196918380831AC08230C1F482
:104C3000CA57DF4FF881C658D0402F2F30E0F5011A
:104C40008081918128173907F1F0CA57DF4FF88129
:104C5000C658D040FF5FCA57DF4FF883C658D040D0
:104C6000C601B701C757DF4F48815981C958D040A5
:104C70000E94C07218160CF4D2CE05C0F7019081C4
:104C8000992309F071CFC357DF4F0FB6F894DEBFF9
:104C90000FBECDBFCF91DF911F910F91FF90EF908D
:104CA000DF90CF90BF90AF909F908F907F906F904C
:104CB0005F904F903F902F900895EF92FF920F9347
:104CC0001F93DF93CF93CDB7DEB76F970FB6F894EE
:104CD000DEBF0FBECDBF7C018C01015B1F4F8F5A21
:104CE0009F4FF8019183808327EF31E0E20EF31E9E
:104CF00021E0F70121937F011182108228E03EEF2D
:104D0000E20EF31E049640E050E060E070E00E9486
:104D1000B16FF80120813181DE011596F9013496D9
:104D20008BE101900D928150E1F7F901828193812D
:104D30009C838B838AE194E09A838983C70165E130
:104D400072E08E010F5F1F4FA80106DEC8010E94AE
:104D50000F1DF701E850FE4F808191816F960FB6CD
:104D6000F894DEBF0FBECDBFCF91DF911F910F91A1
:104D7000FF90EF900895EF92FF920F931F93DF93B0
:104D8000CF93CDB7DEB76F970FB6F894DEBF0FBEE7
:104D9000CDBF7C018C01015B1F4F8F5A9F4FF801E3
:104DA0009183808327EF31E0E20EF31E22E0F701CA
:104DB000208329E03EEFE20EF31EF701E850FE4F9C
:104DC00060831182049640E050E060E070E00E9451
:104DD000B16FF80120813181DE011596F901349619
:104DE0008BE101900D928150E1F7F901828193816D
:104DF0009C838B838AE194E09A838983C70165E170
:104E000072E08E010F5F1F4FA801A6DDC8010E944E
:104E10000F1D6F960FB6F894DEBF0FBECDBFCF91BA
:104E2000DF911F910F91FF90EF900895EF92FF9205
:104E30000F931F93DF93CF93CDB7DEB76F970FB666
:104E4000F894DEBF0FBECDBF7C0187EF91E0E80E86
:104E5000F91EF701108289E09EEFE80EF91E870126
:104E60000C5C1F4FC80140E050E060E070E00E9421
:104E7000B16FDE011596F8018BE101900D92815022
:104E8000E1F7F70182A993A99C838B838AE194E0DF
:104E90009A838983C70165E172E08E010F5F1F4F1E
:104EA000A8015ADDC8010E940F1D6F960FB6F89435
:104EB000DEBF0FBECDBFCF91DF911F910F91FF904D
:104EC000EF9008950F931F93CF93DF93DC01D49657
:104ED0001C92D497D7961C92D797D3961C921E9269
:104EE000D2978AE194E0D1969C938E93D097AB5A57
:104EF000BF4F1C9213961C92A855B040FD01EF5A6B
:104F0000FF4FAD5ABF4F11961C921E92A355B04051
:104F100091838083ED01C059DF4FFE0120E030E036
:104F2000482F148217821382128240839183215E5C
:104F30003F4F7F9681E02633380799F7A755BE4F3C
:104F400089E18C9313961C9258961C921B961C9286
:104F500013961C92A25DB140FD01E553FE4FA35391
:104F6000BE4F11961C921E92408391835D961D92B6
:104F70001D921D921C92139718961D921D921D92C0
:104F80001C921397A25FB14012961C9212979F96A3
:104F90001C929F971C9211961C9211978D010251A1
:104FA0001E4FF8011082118212821382AA55BE4F41
:104FB0001C92FE01C90111920197E9F7A05BBF4F56
:104FC00081E08C93A65FB1409E961C921E929D97A5
:104FD0000E944A1A68577C4E8F4F9F4FF80160839A
:104FE000718382839383DF91CF911F910F910895F5
:104FF000DF93CF93CDB7DEB7E0970FB6F894DEBF5F
:105000000FBECDBFDE011196EAECF3E080E1019026
:105010000D928150E1F7DE015196EAEBF3E080E179
:1050200001900D928150E1F7DE019196EAEAF3E0FA
:1050300080E101900D928150E1F789819A81AB81E5
:10504000BC818093D5089093D608A093D708B093DD
:10505000D80889899A89AB89BC898093C5089093BF
:10506000C608A093C708B093C80889A19AA1ABA1AC
:10507000BCA18093E9089093EA08A093EB08B09351
:10508000EC088D819E81AF81B8858093D90890937B
:10509000DA08A093DB08B093DC088D899E89AF897C
:1050A000B88D8093C9089093CA08A093CB08B09399
:1050B000CC088DA19EA1AFA1B8A58093ED089093D7
:1050C000EE08A093EF08B093F00889859A85AB8528
:1050D000BC858093DD089093DE08A093DF08B09331
:1050E000E008898D9A8DAB8DBC8D8093CD0890930F
:1050F000CE08A093CF08B093D00889A59AA5ABA5F8
:10510000BCA58093F1089093F208A093F308B093A4
:10511000F4088D859E85AF85B8898093E1089093CA
:10512000E208A093E308B093E4088D8D9E8DAF8DC7
:10513000B8A18093D1089093D208A093D308B093DC
:10514000D4088DA59EA5AFA5B8A98093F508909326
:10515000F608A093F708B093F8080E949C5A80E0E4
:1051600090E4ACE9B5E48093FD089093FE08A09329
:10517000FF08B09300098093010990930209A0935E
:105180000309B093040920E030E040E050E02093B0
:10519000F9083093FA084093FB085093FC0880E22A
:1051A0009EE4A0E0B0E08093C1089093C208A09371
:1051B000C308B093C4082093110930931209409397
:1051C00013095093140980E090E0A0EAB1E48093C1
:1051D000050990930609A0930709B09308098DEC7F
:1051E0009CECACECBEE38093090990930A09A09370
:1051F0000B09B0930C0980E090E0A0EAB0E4809342
:105200000D0990930E09A0930F09B09310092093F4
:105210004C0630934D0640934E0650934F06209314
:1052200048063093490640934A0650934B06209314
:10523000440630934506409346065093470686E65B
:1052400096E6A2E4B1E48093850390938603A0934D
:105250008703B093880360E070E080E89FE30E94DA
:1052600060876093890370938A0380938B03909384
:105270008C036BE774E184E192E40E946C87609395
:105280008D0370938E0380938F03909390030E94FD
:10529000548680E090E0A0E8BFE380939103909370
:1052A0009203A0939303B093940384E195E09093C9
:1052B0007B0380937A0390937D0380937C0382EE3B
:1052C00094E090937F0380937E0384E68093A90308
:1052D0001092E410EAECF3E0949108C08091C000D1
:1052E00085FFFCCF9093C600319694919923B1F736
:1052F000E0EDF3E0949108C08091C00085FFFCCF01
:105300009093C600319694919923B1F78091C00093
:1053100085FFFCCF8AE08093C600E0960FB6F89434
:10532000DEBF0FBECDBFCF91DF910895CF93DF9346
:10533000CAECD3E0FE01949108C08091C00085FFC3
:10534000FCCF9093C600319694919923B1F7E4EC89
:10535000F5E0949108C08091C00085FFFCCF909348
:10536000C600319694919923B1F78091C00085FFD2
:10537000FCCF8AE08093C600FE019491EAECF3E052
:1053800008C08091C00085FFFCCF9093C600319685
:1053900094919923B1F74091D5085091D608609126
:1053A000D7087091D8088CEB95E00E9407344091A3
:1053B000D9085091DA086091DB087091DC0889EB1C
:1053C00095E00E9407344091DD085091DE0860911D
:1053D000DF087091E00886EB95E00E940734409169
:1053E000E1085091E2086091E3087091E40883EBD2
:1053F00095E00E940734E6E1F2E007C08091C0002A
:1054000085FFFCCF31969093C60090819923B1F728
:105410008091C00085FFFCCF8AE08093C600FE012A
:105420009491EAECF3E008C08091C00085FFFCCFC6
:105430009093C600319694919923B1F7E9E9F5E08C
:10544000949108C08091C00085FFFCCF9093C60066
:10545000319694919923B1F78091C00085FFFCCFDC
:105460008AE08093C600FE019491EAECF3E008C064
:105470008091C00085FFFCCF9093C6003196949137
:105480009923B1F74091C5085091C6086091C708AB
:105490007091C80880E995E00E9407344091C908DE
:1054A0005091CA086091CB087091CC088DE895E0C6
:1054B0000E9407344091CD085091CE086091CF08EA
:1054C0007091D0088AE895E00E9407344091D10895
:1054D0005091D2086091D3087091D40887E895E084
:1054E0000E940734E6E1F2E007C08091C00085FF2A
:1054F000FCCF31969093C60090819923B1F78091AB
:10550000C00085FFFCCF8AE08093C600FE01949125
:10551000EAECF3E008C08091C00085FFFCCF9093D7
:10552000C600319694919923B1F7E9E6F5E094919C
:1055300008C08091C00085FFFCCF9093C6003196D3
:1055400094919923B1F78091C00085FFFCCF8AE048
:105550008093C600FE019491EAECF3E008C08091CC
:10556000C00085FFFCCF9093C6003196949199239B
:10557000B1F74091E9085091EA086091EB08709109
:10558000EC0880E695E00E941A344091ED085091B5
:10559000EE086091EF087091F0088DE595E00E94AB
:1055A0001A344091F1085091F2086091F30870911B
:1055B000F4088AE595E00E941A344091F50850916C
:1055C000F6086091F7087091F80887E595E00E9469
:1055D0001A34E6E1F2E007C08091C00085FFFCCFFD
:1055E00031969093C60090819923B1F78091C000C5
:1055F00085FFFCCF8AE08093C600FE019491EAEC1F
:10560000F3E008C08091C00085FFFCCF9093C600F6
:10561000319694919923B1F7E2E2F5E0949108C0B4
:105620008091C00085FFFCCF9093C6003196949185
:105630009923B1F78091C00085FFFCCF8AE0809369
:10564000C600FE019491EAECF3E008C08091C0002E
:1056500085FFFCCF9093C600319694919923B1F7C2
:105660004091FD085091FE086091FF08709100097B
:1056700089E195E00E9407344091010950910209A7
:10568000609103097091040986E195E00E94073456
:10569000E6E1F2E007C08091C00085FFFCCF3196C3
:1056A0009093C60090819923B1F78091C00085FF47
:1056B000FCCF8AE08093C600FE019491EAECF3E00F
:1056C00008C08091C00085FFFCCF9093C600319642
:1056D00094919923B1F7E3E6F4E0949108C08091A6
:1056E000C00085FFFCCF9093C6003196949199231A
:1056F000B1F78091C00085FFFCCF8AE08093C6009F
:10570000FE019491EAECF3E008C08091C00085FFAF
:10571000FCCF9093C600319694919923B1F74091B4
:10572000F9085091FA086091FB087091FC088AE52D
:1057300094E00E9407344091110950911209609140
:1057400013097091140987E594E00E940734409191
:10575000C1085091C2086091C3087091C40884E5E3
:1057600094E00E941A344091050950910609609115
:1057700007097091080981E594E00E94073440917F
:10578000090950910A0960910B0970910C098EE486
:1057900094E00E94073440910D0950910E096091E8
:1057A0000F09709110098BE494E00E940734E6E140
:1057B000F2E007C08091C00085FFFCCF3196909346
:1057C000C60090819923B1F78091C00085FFFCCF7E
:1057D0008AE08093C600FE019491EAECF3E008C0F1
:1057E0008091C00085FFFCCF9093C60031969491C4
:1057F0009923B1F7E9E3F4E0949108C08091C000E7
:1058000085FFFCCF9093C600319694919923B1F710
:105810008091C00085FFFCCF8AE08093C600FE0126
:105820009491EAECF3E008C08091C00085FFFCCFC2
:105830009093C600319694919923B1F74091440614
:1058400050914506609146067091470680E394E0CA
:10585000DED7409148065091490660914A06709102
:105860004B068DE294E0D3D740914C0650914D0603
:1058700060914E0670914F068AE294E0C8D7E6E147
:10588000F2E007C08091C00085FFFCCF3196909375
:10589000C60090819923B1F78091C00085FFFCCFAD
:1058A0008AE08093C600FE019491EAECF3E008C020
:1058B0008091C00085FFFCCF9093C60031969491F3
:1058C0009923B1F7ECE1F4E0949108C08091C00015
:1058D00085FFFCCF9093C600319694919923B1F740
:1058E0008091C00085FFFCCF8AE08093C600FE0156
:1058F0009491EAECF3E008C08091C00085FFFCCFF2
:105900009093C600319694919923B1F74091850305
:1059100050918603609187037091880382E194E03F
:1059200076D76091890370918A0380918B0390915F
:105930008C030E946687AB01BC018FE094E067D7BF
:1059400060918D0370918E0380918F0390919003ED
:105950000E947287AB01BC018CE094E058D7E6E16D
:10596000F2E007C08091C00085FFFCCF3196909394
:10597000C60090819923B1F78091C00085FFFCCFCC
:105980008AE08093C600DF91CF910895EF92FF9255
:105990001F93CF93DF93EC017B01142F88819981B2
:1059A0000E9464DBF70181937F01888199810196D0
:1059B00099838883115091F7DF91CF911F91FF90C8
:1059C000EF900895EF92FF920F931F93DF93CF9381
:1059D000CDB7DEB766970FB6F894DEBF0FBECDBF6A
:1059E00084E690E09A83898380911702909118024F
:1059F000A0911902B0911A028B8B9C8BAD8BBE8B40
:105A00008E01015F1F4F7E010894E11CF11CC7014C
:105A1000B80144E0BBDFCE014396B80143E050E05B
:105A20000E948DD4009709F0A6C0C70165ED78E00B
:105A300040E1ACDFC70165EC78E040E1A7DFC701DA
:105A400069EE78E040E1A2DF0E949C5AC7016DEF49
:105A500078E044E09BDFC70161E079E044E096DF55
:105A6000C70169EF78E044E091DFC70161E179E0C7
:105A700044E08CDFC70161EC78E044E087DFC701D8
:105A800065E079E044E082DFC70169E079E044E065
:105A90007DDFC7016DE079E044E078DFC70164E4B1
:105AA00076E04CE073DFC701BE016D5F7F4F42E0DF
:105AB0006DDFC701BE016B5F7F4F42E067DFC7014B
:105AC000BE01695F7F4F42E061DFC701BE01675FD2
:105AD0007F4F42E05BDFC701BE01655F7F4F42E061
:105AE00055DFC701BE01635F7F4F42E04FDFC70153
:105AF00065E873E044E04ADFC70169E873E044E029
:105B000045DFC7016DE873E044E040DFC7016AE7A5
:105B100073E046E03BDFC70169EA73E041E036DF4E
:105B2000C70164EE70E141E031DF0E945486EAEC87
:105B3000F3E0949108C08091C00085FFFCCF909362
:105B4000C600319694919923B1F7E2EFF3E0949176
:105B500008C08091C00085FFFCCF9093C6003196AD
:105B600094919923B1F78091C00085FFFCCF8AE022
:105B70008093C60001C03CDAD9DB66960FB6F89474
:105B8000DEBF0FBECDBFCF91DF911F910F91FF9070
:105B9000EF900895EF92FF921F93CF93DF93EC0164
:105BA0007B01142F88819981F70161917F010E9407
:105BB0007FDB88819981019699838883115091F7C1
:105BC000DF91CF911F91FF90EF900895EF92FF9298
:105BD0000F931F93DF93CF93CDB7DEB766970FB6C2
:105BE000F894DEBF0FBECDBF80911B0290911C02C6
:105BF000A0911D02B0911E028F87988BA98BBA8B42
:105C000084E6E82EF12CFA82E9828E010F5F1F4FA5
:105C1000C801BE01615F7F4F44E0BCDFC80165ED94
:105C200078E040E1B7DFC80165EC78E040E1B2DF41
:105C3000C80169EE78E040E1ADDFC8016DEF78E0C2
:105C400044E0A8DFC80161E079E044E0A3DFC801D7
:105C500069EF78E044E09EDFC80161E179E044E06B
:105C600099DFC80161EC78E044E094DFC80165E0A9
:105C700079E044E08FDFC80169E079E044E08ADF41
:105C8000C8016DE079E044E085DFC80164E476E0B6
:105C90004CE080DF84EB90E09C838B8386E490E093
:105CA0009E838D8318861F8280EF90E09A87898774
:105CB000FC86EB861E861D86C801BE016D5F7F4F88
:105CC00042E068DFC801BE016B5F7F4F42E062DFE8
:105CD000C801BE01695F7F4F42E05CDFC801BE01C1
:105CE000675F7F4F42E056DFC801BE01655F7F4FAF
:105CF00042E050DFC801BE01635F7F4F42E04ADFF0
:105D0000C80165E873E044E045DFC80169E873E075
:105D100044E040DFC8016DE873E044E03BDFC801C8
:105D20006AE773E046E036DFC80169EA73E041E004
:105D300031DFC80164EE70E141E02CDF8091170291
:105D400090911802A0911902B0911A028B8B9C8B32
:105D5000AD8BBE8BFA82E982C801BE016D5E7F4FBA
:105D600044E018DFEAECF3E0949108C08091C000B1
:105D700085FFFCCF9093C600319694919923B1F79B
:105D8000E4EDF5E0949108C08091C00085FFFCCF60
:105D90009093C600319694919923B1F78091C000F9
:105DA00085FFFCCF8AE08093C60066960FB6F89414
:105DB000DEBF0FBECDBFCF91DF911F910F91FF903E
:105DC000EF900895DF93CF930F920F92CDB7DEB788
:105DD0002091CF153091D015CE01019621153105B6
:105DE00019F4855D954102C0821B930B9A838983C8
:105DF00089819A810F900F90CF91DF91089520E0D3
:105E00008091360890913708181619060CF421E095
:105E1000822F0895EF92FF920F931F93CF93DF93FA
:105E2000EC01E0905006F09051060091520610915E
:105E30005306688179818A819B81A80197010E941C
:105E4000D4D5882324F4E882F9820A831B83E09066
:105E50005406F090550600915606109157066C8135
:105E60007D818E819F81A80197010E94D4D58823CE
:105E700024F4EC82FD820E831F83E0905806F0909C
:105E8000590600915A0610915B06688579858A85C6
:105E90009B85A80197010E94D4D5882324F4E88625
:105EA000F9860A871B87E0905003F0905103009118
:105EB000520310915303688179818A819B81A801E3
:105EC00097010E94D7D7181624F4E882F9820A8332
:105ED0001B83E0905403F0905503009156031091FA
:105EE00057036C817D818E819F81A80197010E945B
:105EF000D7D7181624F4EC82FD820E831F83E0901E
:105F00005803F090590300915A0310915B03688580
:105F100079858A859B85A80197010E94D7D7181695
:105F200024F4E886F9860A871B87DF91CF911F91B9
:105F30000F91FF90EF90089580916D06811181E09F
:105F4000089580916D060895CF93DF938130910578
:105F500041F46F5F7F4FF9F482E394E00E9462277F
:105F60001AC0892BC1F46F5F7F4FA9F48DEF95E0C4
:105F70000E940F1DC9EBD5E0CE010E940F1D6F9747
:105F800084E0C338D807C1F7CE010E940F1DCE01AF
:105F900081970E940F1DDF91CF91089580E090E0DE
:105FA0006FEF7FEFD1CF81E090E06FEF7FEFCCCF4D
:105FB0001F93182F0E943D8780916D06882309F05A
:105FC00035C010936D0680916F0690917006A09178
:105FD0007106B09172068093730690937406A09335
:105FE0007506B0937606EAEEF5E0949108C08091CC
:105FF000C00085FFFCCF9093C60031969491992301
:10600000B1F7E1EFF5E0949108C08091C00085FF01
:10601000FCCF9093C600319694919923B1F780916B
:10602000C00085FFFCCF8AE08093C6001F910895D1
:10603000F8940E943D87159A469A439A409A8CE0BC
:1060400060E00E94981BEAEEF5E0949108C0809110
:10605000C00085FFFCCF9093C600319694919923A0
:10606000B1F7E7E6F6E0949108C08091C00085FFA3
:10607000FCCF9093C600319694919923B1F780910B
:10608000C00085FFFCCF8AE08093C600FFCF0E944E
:106090004A1A6093770670937806809379069093F6
:1060A0007A06E091A006F091A106EE55F94F8081A5
:1060B0008823A9F4E6E8F6E0949108C08091C00036
:1060C00085FFFCCF9093C600319694919923B1F748
:1060D0008091C00085FFFCCF8AE08093C6000895C0
:1060E000EF92FF920F931F930E944A1AE0907B0653
:1060F000F0907C0600917D0610917E062091770637
:10610000309178064091790650917A06621B730BA4
:10611000840B950BE616F7060807190730F4E1140F
:10612000F1040105110509F083DF80916D03909161
:106130006E03A0916F03B09170030097A105B105A4
:10614000F9F00E944A1A2091770630917806409122
:10615000790650917A06621B730B840B950B209184
:106160006D0330916E0340916F03509170032617B9
:1061700037074807590720F48091050E8091060ED5
:10618000069B02C08AE014DF0E94275D1F910F91D9
:10619000FF90EF9008956F927F928F929F92AF92AF
:1061A000BF92CF92DF92EF92FF920F931F93F82E40
:1061B00060917F06709180068091810690918206A1
:1061C0002091830630918406409185065091860681
:1061D0000E94E4D73B014C0100D000D00DB71EB7A0
:1061E0000F5F1F4F60914C0370914D03882777FD1F
:1061F0008095982F0E9476D620917103309172037A
:1062000040917303509174030E94A9D820E030E0BC
:1062100040E752E40E94DBD520E030E048EC52E455
:106220000E94DBD55B016C01F80160827182828281
:106230009382F48280915C06858384E396E06BE828
:1062400076E04FE756E020E001E032E0E32E0E94E6
:106250000F5780918B0690918C06A0918D06B0917E
:106260008E068093340690933506A0933606B0933D
:10627000370680918F0690919006A0919106B0917B
:1062800092068093380690933906A0933A06B0930D
:106290003B068091930690919406A0919506B0914B
:1062A000960680933C0690933D06A0933E06B093DD
:1062B0003F068091970690919806A0919906B0911B
:1062C0009A068093400690934106A0934206B093AD
:1062D00043068DB79EB706960FB6F8949EBF0FBEC5
:1062E0008DBF0E944A1A6093770670937806809358
:1062F000790690937A061F910F91FF90EF90DF90AF
:10630000CF90BF90AF909F908F907F906F900895A7
:10631000CF92DF92EF92FF920F931F938BE896E05C
:1063200079DD0E944A1A609377067093780680930D
:10633000790690937A0660913406709135068091C3
:1063400036069091370620918B0630918C0640914D
:106350008D0650918E060E94D4D5882309F07AC00C
:10636000609138067091390680913A0690913B060B
:1063700020918F063091900640919106509192069F
:106380000E94D4D5882309F065C060917103709193
:106390007203809173039091740320E030E040E732
:1063A00052E40E94DBD57B018C018BE896E06FE81C
:1063B00076E043E956E027E936E0ECE5CE2EE6E06C
:1063C000DE2E0E94506080918B0690918C06A091E9
:1063D0008D06B0918E068093340690933506A09377
:1063E0003606B093370680918F0690919006A09163
:1063F0009106B09192068093380690933906A09347
:106400003A06B0933B068091930690919406A09132
:106410009506B091960680933C0690933D06A09316
:106420003E06B0933F068091970690919806A09102
:106430009906B0919A068093400690934106A093E6
:106440004206B09343061F910F91FF90EF90DF90AB
:10645000CF90089560914C0370914D03882777FD8C
:106460008095982F0E9476D6209171033091720307
:1064700040917303509174030E94A9D820E030E04A
:1064800040E752E40E94DBD520E030E048EC52E4E3
:1064900088CF80EC98E00E944B55E9E8F6E09491B3
:1064A00008C08091C00085FFFCCF9093C600319654
:1064B00094919923B1F740916F06509170066091C5
:1064C0007106709172064F5F5F4F6F4F7F4F80EC88
:1064D00098E02AE030E00E9407568091C00085FFD6
:1064E000FCCF8AE08093C600D2CD2F923F924F928C
:1064F0005F926F927F928F929F92AF92BF92CF9254
:10650000DF92EF92FF920F931F93DF93CF9300D010
:1065100000D0CDB7DEB78C018330910508F040C1C3
:106520003C01660C771C660C771C93012C5C394F80
:106530003A83298380E090E0A0E0B0E0F901808315
:106540009183A283B38384E396E068E376E04CE32F
:1065500056E020E436E00E94F35AF301EF5DF74F76
:106560006591759185919491075C174FF801E490BE
:1065700093012557394F3E832D8320E030E040ECD6
:106580005FE30E94A9D85B016C01FF24E7FCF09453
:106590000F2D1F2DC801B7010E9476D61B012C01BB
:1065A000C601B501A20191010E94A9D8AD81BE81A9
:1065B0006D937D938D939C931397F301E45CFC4F53
:1065C000FC83EB836081718182819381609371038D
:1065D00070937203809373039093740320E030E010
:1065E00040E752E40E94DBD57B018C018BE896E00A
:1065F0006FE876E043E956E027E936E0FCE5CF2E88
:10660000F6E0DF2E0E9450600E943D7F80E090E027
:10661000A0E0B0E0E981FA8180839183A283B38313
:1066200084E396E068E376E04CE356E020E436E06D
:106630000E94F35AF301E35DF74F85909590A59082
:10664000B490C501B4019058A20191010E94A9D84B
:10665000AD81BE816D937D938D939C9313976091D3
:10666000710370917203809173039091740320E021
:1066700030E040E752E40E94DBD57B018C018BE8DF
:1066800096E06FE876E043E956E027E936E00E94BD
:1066900050600E943D7FC501B401A50194010E9494
:1066A000FBD4A20191010E94A9D8ED81FE816083F3
:1066B000718382839383AB81BC816D917D918D9138
:1066C0009C9120E030E040E450E40E94DBD56093F0
:1066D000710370937203809373039093740320E0AB
:1066E00030E040E752E40E94DBD57B018C018BE86F
:1066F00096E06FE876E043E956E027E936E00E944D
:1067000050600E943D7FF301E350F84F6591759111
:1067100085919491F301EC5BF94F208131814281A5
:1067200053810E94FBD49B01AC01E981FA81208353
:10673000318342835383F301E75FF74F259135910E
:1067400045915491F301E05BF94F208331834283FB
:106750005383F301EB5EF74F2591359145915491A9
:10676000A0E5B3E06A0E7B1EF301208331834283F0
:106770005383AC01CB01DA01ED81FE8180839183EB
:10678000A283B38380E090E0A0E0B0E08093710347
:1067900090937203A0937303B09374030E94CC7D13
:1067A00026960FB6F894DEBF0FBECDBFCF91DF9116
:1067B0001F910F91FF90EF90DF90CF90BF90AF901F
:1067C0009F908F907F906F905F904F903F902F9011
:1067D0000895682F2091A0063091A10680E690E0F0
:1067E000AC01249FC001259F900D349F900D112472
:1067F0008455994F70E00E947BD49C019093AB0626
:106800008093AA0680E0232B09F081E00895FC0123
:10681000949108C08091C00085FFFCCF9093C60082
:10682000319694919923B1F780EC98E022E030E022
:106830000C940D57FC01949108C08091C00085FF15
:10684000FCCF9093C600319694919923B1F780ECD8
:1068500098E02AE030E00C94EB558091AA069091E4
:10686000AB06019660E070E04AE050E00C9480D204
:106870008091AA069091AB06019660E070E00C94BE
:106880001AD1CF93DF93EC0180915C0680936E0662
:1068900084E59FDF882309F46EC0EADF0E9448D6B2
:1068A000262F60936E06662309F465C0E4EEF5E0DA
:1068B000949108C08091C00085FFFCCF9093C600E2
:1068C000319694919923B1F7C936D10599F0CA361A
:1068D000D10524F4C836D105F1F50FC0CD36D10568
:1068E00031F0CA3DD105B9F5EFE1F2E031C0E6E3A0
:1068F000F2E023C0EDE4F2E015C0E4E6F2E007C008
:106900008091C00085FFFCCF31969093C6009081A6
:106910009923B1F720C08091C00085FFFCCF31964C
:106920009093C60090819923B1F715C08091C00063
:1069300085FFFCCF31969093C60090819923B1F7E3
:106940000AC08091C00085FFFCCF31969093C600AD
:1069500090819923B1F780EC98E0622F40E050E0FD
:106960000E94F6558091C00085FFFCCF8AE080939D
:10697000C60081E001C080E0DF91CF9108955F9271
:106980006F927F928F929F92AF92BF92CF92DF923F
:10699000EF92FF920F931F93DF93CF9300D00F924C
:1069A000CDB7DEB719821A821B821C8214E3C12E76
:1069B00016E0D12EBBE8EB2EB6E0FB2E00E010E097
:1069C0003E010894611C711C55245394F801E65251
:1069D000FC4F8081FEDE882359F14ADF4B015C01C8
:1069E000F801E25DF94F8081882311F061E002C077
:1069F00060919B0670E0882777FD8095982F0E9414
:106A000076D6F60120813181428153810E94A9D836
:106A10009B01AC01C501B4010E94FBD4F701608366
:106A2000718382839383F301E00FF11F50820AC0C8
:106A3000F60180819181A281B381F70180839183E6
:106A4000A283B3830F5F1F4F84E090E0C80ED91E6E
:106A5000E80EF91E0430110509F0B8CF86E4B9DE5E
:106A60008823D9F005DF7B018C0160939C0670932D
:106A70009D0680939E0690939F0620E030E040E0C4
:106A800050E00E94D7D7181644F4E0927103F092B8
:106A90007203009373031093740380915E0688233E
:106AA00009F4C1C08981882309F0BDC08A81882387
:106AB00009F0B9C08B81882309F0B5C08C81882387
:106AC00009F4B1C0A0904006B0904106C0904206C3
:106AD000D090430660919706709198068091990630
:106AE00090919A06A60195010E94FAD47B018C012F
:106AF0002DEC3CEC4CEC5DEB0E94D4D588230CF0E3
:106B00004EC080915F06882309F08DC06091930686
:106B10007091940680919506909196062091650358
:106B20003091660340916703509168030E94FBD443
:106B300060939306709394068093950690939606BF
:106B4000C801B701905820915D0330915E034091D8
:106B50005F03509160030E94FAD49B01AC01C6010F
:106B6000B5010E94FAD46093400670934106809369
:106B70004206909343068091610390916203A09135
:106B80006303B09164038093710390937203A093A5
:106B90007303B093740381E080935F0644C0C8011F
:106BA000B7012DEC3CEC4CEC5DE30E94D7D71816F6
:106BB000D4F580915F068823B1F160915D037091F7
:106BC0005E0380915F0390916003A80197010E948A
:106BD000FAD420916006309161064091620650918E
:106BE00063060E94FBD49B01AC01C601B5010E9463
:106BF000FBD46093400670934106809342069093C5
:106C000043068091690390916A03A0916B03B09150
:106C10006C038093710390937203A0937303B093FA
:106C2000740310925F060F900F900F900F90CF910A
:106C3000DF911F910F91FF90EF90DF90CF90BF9069
:106C4000AF909F908F907F906F905F90089597DEA8
:106C500089E4BFDD882351F00BDE60937F067093DB
:106C6000800680938106909382060CC080E090E0BD
:106C7000A0E0B0E080937F0690938006A093810609
:106C8000B09382068AE4A5DD882351F0F1DD60939C
:106C900083067093840680938506909386060895F4
:106CA00080E090E0A0E0B0E08093830690938406BB
:106CB000A0938506B093860608952F923F924F9237
:106CC0005F926F927F928F929F92AF92BF92CF927C
:106CD000DF92EF92FF920F931F93DF93CF93CDB785
:106CE000DEB76E970FB6F894DEBF0FBECDBF109221
:106CF000640687E46EDD882309F44DC6B9DD0E9481
:106D000043D66A30710509F48BC06B3071059CF471
:106D10006230710599F16330710524F4772334F5FD
:106D20000C94FB4C6330710581F16430710511F0F6
:106D30000C94FB4C33C06A35710509F4D7C56B352B
:106D4000710554F46B30710509F405C16C3171059E
:106D500011F00C94FB4C74C16B35710509F4CAC574
:106D60006C35710511F00C94FB4CC9C580916D0612
:106D7000882321F404DECCDA0C941E4D80916D063C
:106D8000882319F464DF81E006C080916D068823B2
:106D900029F45DDF80E0FFD90C941E4D80E519DDFC
:106DA000882321F4EE24FF24870105C061DD0E94C1
:106DB00048D67B018C0183E50CDD882359F058DD32
:106DC00020E030E04AE754E40E94A9D80E9448D667
:106DD0007B018C010E943D7F0E944A1A5B016C017D
:106DE000AE0CBF1CC01ED11E0E944A1A60937706CB
:106DF000709378068093790690937A0681E0809369
:106E0000640605C00E946D8B6BD90E94BF940E94DE
:106E10004A1A6A157B058C059D05A0F30C94FB4C62
:106E200080915F06882311F00C94FB4C809134060E
:106E300090913506A0913606B091370680938B0667
:106E400090938C06A0938D06B0938E0680913806A1
:106E500090913906A0913A06B0913B0680938F0637
:106E600090939006A0939106B093920680913C0671
:106E700090913D06A0913E06B0913F068093930607
:106E800090939406A0939506B0939606E0915C06C5
:106E9000F0E0EE0FFF1FEE0FFF1FEB51F74F609179
:106EA0005D0370915E0380915F0390916003208188
:106EB0003181428153810E94DBD59B01AC016091FD
:106EC00040067091410680914206909143060E94CF
:106ED000FAD49B01AC016093970670939806809357
:106EE000990690939A06E0907103F09072030091D6
:106EF0007303109174038091610390916203A091D8
:106F00006303B09164038093710390937203A09321
:106F10007303B093740360914006709141068091B1
:106F20004206909143060E94FAD4609360067093E3
:106F30006106809362069093630681E080935F060A
:106F4000E7D9E0927103F0927203009373031093F8
:106F500074030C94FB4C80915F06882311F40C940D
:106F6000FB4C8091340690913506A0913606B09185
:106F7000370680938B0690938C06A0938D06B09372
:106F80008E068091380690913906A0913A06B0910C
:106F90003B0680938F0690939006A0939106B09342
:106FA000920680913C0690913D06A0913E06B091DC
:106FB0003F068093930690939406A0939506B09312
:106FC000960660914006709141068091420690912C
:106FD000430620916006309161064091620650910F
:106FE00063060E94FBD46093970670939806809383
:106FF000990690939A06E0907103F09072030091C5
:107000007303109174038091690390916A03A091B6
:107010006B03B0916C038093710390937203A09300
:107020007303B093740310925F0672D9E0927103F8
:10703000F092720300937303109374030C94FB4C4F
:1070400085E0809364068091710390917203A09112
:107050007303B09174038093A6069093A706A09340
:10706000A806B093A90680914C0390914D0390938C
:1070700033068093320684E690E090934D0380932C
:107080004C030E944A1A60937706709378068093A7
:10709000790690937A0681E00E94D37D8091340630
:1070A00090913506A0913606B091370680938B06F5
:1070B00090938C06A0938D06B0938E06809138062F
:1070C00090913906A0913A06B0913B0680938F06C5
:1070D00090939006A0939106B093920680913C06FF
:1070E00090913D06A0913E06B0913F068093930695
:1070F00090939406A0939506B093960680914006CF
:1071000090914106A0914206B09143068093970664
:1071100090939806A0939906B0939A0680E090E029
:10712000A0E0B0E08093710390937203A093730387
:10713000B093740388E54DDB882351F489E549DB7E
:10714000882331F48AE545DB882311F481E001C00E
:1071500080E080937503882309F4A2C10F2EF0E02C
:107160008F2EF0E09F2EF0E0AF2EF0E0BF2EF02D3E
:107170008092340690923506A0923606B092370679
:107180008092380690923906A0923A06B0923B0659
:1071900080923C0690923D06A0923E06B0923F0639
:1071A00084E396E068E376E04CE356E020E436E0E2
:1071B0000E94F35A80E090E8ACEAB3EC80938B062F
:1071C00090938C06A0938D06B0938E0680E090E895
:1071D000ACEAB3E480938F0690939006A093910657
:1071E000B09392068093930690939406A09395068D
:1071F000B093960660913C0370913D0380913E03ED
:1072000090913F03609371037093720380937303B3
:107210009093740320E030E040E752E40E94DBD515
:107220007B018C018BE896E06FE876E043E956E05D
:1072300027E936E0FCE5CF2EF6E0DF2E0E94506015
:107240000E943D7F0E94CC7DEDEFF7E06591759146
:1072500085919491209144063091450640914606CF
:10726000509147060E94FBD4609334067093350614
:107270008093360690933706E9E0F8E08591959182
:10728000A591B4918093500690935106A093520615
:10729000B0935306E5E1F8E085919591A591B491FD
:1072A0008093500390935103A0935203B0935303E0
:1072B000E1E0F8E0659175918591949120914806FF
:1072C0003091490640914A0650914B060E94FBD4EA
:1072D000609338067093390680933A0690933B0684
:1072E000EDE0F8E085919591A591B49180935406D5
:1072F00090935506A0935606B0935706E9E1F8E03F
:1073000085919591A591B4918093540390935503E1
:10731000A0935603B0935703E5E0F8E065917591AB
:107320008591949120914C0630914D0640914E06E6
:1073300050914F060E94FBD460933C0670933D062B
:1073400080933E0690933F06E1E1F8E085919591A8
:10735000A591B4918093580690935906A0935A062C
:10736000B0935B06EDE1F8E085919591A591B4911C
:107370008093580390935903A0935A03B0935B03EF
:1073800084E396E068E376E04CE356E020E436E000
:107390000E94F35A8091340690913506A0913606EA
:1073A000B091370680938B0690938C06A0938D0640
:1073B000B0938E068091380690913906A0913A06D6
:1073C000B0913B0680938F0690939006A093910610
:1073D000B093920680913C0690913D06A0913E06A6
:1073E000B0913F068093930690939406A0939506E0
:1073F000B09396066091710370917203809173034C
:107400009091740320E030E040E752E40E94DBD525
:107410007B018C018BE896E06FE876E043E956E06B
:1074200027E936E00E9450608092710390927203C7
:10743000A0927303B09274030E943D7F0E94CC7DA2
:1074400080918B0690918C06A0918D06B0918E064E
:107450008093340690933506A0933606B093370692
:1074600080918F0690919006A0919106B09192061E
:107470008093380690933906A0933A06B0933B0662
:107480008091930690919406A0919506B0919606EE
:1074900080933C0690933D06A0933E06B0933F0632
:1074A00080917503882321F48AE593D9882319F004
:1074B00082E090E01AD880917503882351F488E522
:1074C00088D9882309F46DC189E583D9882309F413
:1074D00068C180E090E0A0E0B0E080933406909333
:1074E0003506A0933606B0933706809338069093FE
:1074F0003906A0933A06B0933B0684E396E068E32E
:1075000076E04CE356E020E436E00E94F35A80E057
:1075100090E8ACEAB3EC80938B0690938C06A09332
:107520008D06B0938E0680E090E8ACEAB3E48093D9
:107530008F0690939006A0939106B09392062091A7
:107540003C0330913D0340913E0350913F03209313
:107550007103309372034093730350937403E0906C
:107560004003F09041030091420310914303C8018E
:10757000B7010E94D4D5882344F4E0927103F092BD
:1075800072030093730310937403609171037091FD
:107590007203809173039091740320E030E040E720
:1075A00052E40E94DBD57B018C018BE896E06FE80A
:1075B00076E043E956E027E936E0ECE5CE2EE6E05A
:1075C000DE2E0E9450600E943D7FEDEFF7E0659156
:1075D0007591859194912091440630914506409192
:1075E0004606509147060E94FBD460933406709380
:1075F00035068093360690933706E9E0F8E08591EA
:107600009591A591B4918093500690935106A093C3
:107610005206B0935306E5E1F8E085919591A59166
:10762000B4918093500390935103A0935203B0936D
:107630005303E1E0F8E06591759185919491209173
:1076400048063091490640914A0650914B060E94E7
:10765000FBD4609338067093390680933A06909372
:107660003B06EDE0F8E085919591A591B49180936A
:10767000540690935506A0935606B0935706E9E139
:10768000F8E085919591A591B491809354039093DE
:107690005503A0935603B093570384E396E068E341
:1076A00076E04CE356E020E436E00E94F35A809105
:1076B000340690913506A0913606B0913706809336
:1076C0008B0690938C06A0938D06B0938E068091C6
:1076D000380690913906A0913A06B0913B06809306
:1076E0008F0690939006A0939106B09392066091B6
:1076F000710370917203809173039091740320E081
:1077000030E040E752E40E94DBD57B018C018BE83E
:1077100096E06FE876E043E956E027E936E00E941C
:10772000506080E090E0A0E0B0E08093710390931F
:107730007203A0937303B09374030E943D7F0E9471
:10774000CC7D80918B0690918C06A0918D06B09196
:107750008E068093340690933506A0933606B09338
:10776000370680918F0690919006A0919106B09176
:1077700092068093380690933906A0933A06B09308
:107780003B068091930690919406A0919506B09146
:10779000960680933C0690933D06A0933E06B093D8
:1077A0003F0680917503882321F488E512D8882349
:1077B00021F080E090E00E9475328091750388236B
:1077C00021F489E506D8882321F081E090E00E9429
:1077D000753288E50E94E9338823C9F03ED86115E7
:1077E00071058105910599F043D8209144063091A7
:1077F000450640914606509147060E94FBD460938F
:10780000340670933506809336069093370689E5E3
:107810000E94E9338823C9F020D8611571058105DC
:10782000910599F025D8209148063091490640915C
:107830004A0650914B060E94FBD460933806709321
:10784000390680933A0690933B068AE50E94E93315
:107850008823C9F002D8611571058105910599F059
:1078600007D820914C0630914D0640914E0650911C
:107870004F060E94FBD460933C0670933D068093B4
:107880003E0690933F0684E396E068E376E04CE39F
:1078900056E020E436E00E94F35A80E00E94D37D57
:1078A0008091A6069091A706A091A806B091A9067E
:1078B0008093710390937203A0937303B093740346
:1078C000809132069091330690934D0380934C0340
:1078D0000E944A1A6093770670937806809379061F
:1078E00090937A060E94CC7D0C94FB4C10929B06E0
:1078F0000C94FB4C81E080939B060C94FB4C85E43C
:107900000E94E933882311F40E943D7F44E3E42E72
:1079100046E0F42E34E4C32E36E0D32E00E010E02F
:10792000F801E652FC4F80810E94E933882331F14F
:10793000033061F40E943834F701608371838283DD
:10794000938380E496E00E94C75A18C00E9438349E
:10795000F60120813181428153810E94FBD4F701DD
:10796000608371838283938384E396E068E376E0A7
:107970004CE356E020E436E00E94F35A0F5F1F4FBD
:1079800024E030E0E20EF31EC20ED31E04301105D7
:1079900039F60C94FB4C8DE40E94E933882311F4F2
:1079A0000C941D4C0E9438340E9443D669377105EF
:1079B00011F40C948D466A3771050CF09CC061354A
:1079C000710509F495C7623571050CF048C069313D
:1079D000710509F4D1C16A317105F4F4653171059D
:1079E00009F493C16631710574F46231710509F4CB
:1079F0008CC76431710509F458C16131710511F00A
:107A00000C94FB4C4CC16731710509F48AC1683193
:107A100071050CF0A1C17FC16E31710509F419C265
:107A20006F31710574F46B31710509F4D0C16B319C
:107A300071050CF4A7C16C31710511F00C94FB4C6D
:107A4000CCC16A32710509F434C36035710509F49B
:107A50004BC76F31710511F00C94FB4CA9C26A360B
:107A6000710509F4C4C66B367105F4F4653571050A
:107A700009F49CC7663571054CF46335710509F44A
:107A80003FC7643571050CF040C736C768367105CD
:107A900009F457C3693671050CF084C36C35710560
:107AA00011F00C94FB4C9DC76337710511F40C94D5
:107AB0007645643771057CF46D36710509F441C46F
:107AC0006237710511F40C9495456B36710511F010
:107AD0000C94FB4C05C76737710509F4DCC06837A7
:107AE000710514F00C9489466537710511F00C94FA
:107AF000FB4C0C94854531E06033730711F40C9412
:107B0000A74941E0613374070CF057C06F3C710521
:107B100011F40C94F447603D71051CF56B3C710544
:107B200011F40C943A476C3C71057CF46E3B710582
:107B300009F49AC5693C710511F40C9418476C3826
:107B4000710511F00C94FB4C1CC36D3C710511F4D4
:107B50000C9478476E3C710514F00C94D6470C9445
:107B600058476D3D710511F40C94B9486E3D71058F
:107B70008CF4613D710511F40C944348613D71052D
:107B800014F40C9423486C3D710511F00C94FB4CDB
:107B90000C94AA4851E06E32750711F40C94554AC2
:107BA00081E06F32780714F00C94644A6D52714092
:107BB00011F00C94FB4C0C94CF48E3E0603A7E0744
:107BC00009F4BBC1F3E0613A7F077CF521E0663F31
:107BD000720711F40C94AD4A31E0673F73079CF4CF
:107BE00041E0643F740711F40C94A74A51E0653FEB
:107BF000750714F00C94AA4A6059714011F00C9466
:107C0000FB4C0C94A44A93E06B38790711F40C9464
:107C1000B34AE3E06B397E0709F466C1675F7140E0
:107C200011F00C94FB4C0C94B04A27E262317207BD
:107C300011F40C941F4B37E2633173079CF447E255
:107C40006031740711F40C94F74A57E261317507FB
:107C500014F00C94FA4A675E734011F00C94FB4CDC
:107C60000C94E24A97E26431790711F40C94744B56
:107C7000E7E264317E0714F40C94444BF7E265317B
:107C80007F0711F40C94A44B6A51774211F00C94C5
:107C9000FB4C0C94D44BEBE7F2E00C94984615980F
:107CA0004698439840980C94FB4CEDEEF7E0949185
:107CB00008C08091C00085FFFCCF9093C60031962C
:107CC00094919923B1F78091C00085FFFCCF8AE0A1
:107CD0008093C60082E394E00E941627EFEDF7E060
:107CE000949108C08091C00085FFFCCF9093C6009E
:107CF000319694919923B1F78091C00085FFFCCF14
:107D00008AE08093C6000C94FB4C82E394E00E94CE
:107D1000A2220C94FB4C82E394E00E94911C0C94F0
:107D2000FB4C8091AA069091AB0604966AE270E043
:107D30000E947BD4FC01009711F031971082609172
:107D4000AA067091AB066C5F7F4F82E394E041E03E
:107D50000E940F1F0C94FB4C82E394E00E94951C40
:107D60000E944A1A609365067093660680936706C0
:107D7000909368060C94FB4C82E394E00E949C1C58
:107D80000C94FB4C80916104882311F40C94FB4CFF
:107D90008091DB05882311F00C94FB4C83E50E9455
:107DA000E933882311F40C94FB4C0E942D34AB0171
:107DB000BC014093240650932506809326067093B9
:107DC000270681E096E00E94B16F0C94FB4C82E3A1
:107DD00094E00E94921E0C94FB4C8091AA06909114
:107DE000AB0604966AE270E00E947BD48C01009797
:107DF00019F12091A0063091A10680E690E0AC0137
:107E0000249FC001259F900D349F900D112484550F
:107E1000994F6EE470E00E947BD460E270E00E94B3
:107E20007BD49C012F5F3F4F3093AB062093AA0673
:107E300001501040F80110826091AA067091AB06C3
:107E40006C5F7F4F82E394E040E00E940F1F0C9430
:107E5000FB4C80916104882311F40C94FB4C8091BD
:107E6000DB05882311F00C94FB4C82E394E00E9424
:107E7000011E8091AA069091AB0604966AE270E01A
:107E80000E947BD48C01009719F12091A0063091BB
:107E9000A10680E690E0AC01249FC001259F900DD3
:107EA000349F900D11248455994F6EE470E00E9428
:107EB0007BD460E270E00E947BD49C012F5F3F4F37
:107EC0003093AB062093AA0601501040F8011082AF
:107ED0006091AA067091AB066C5F7F4F82E394E0DD
:107EE0000E9431210C94FB4C8091AA069091AB0624
:107EF00004966AE270E00E947BD4FC01009711F0C6
:107F0000319710826091AA067091AB066C5F7F4F2B
:107F100082E394E041E00E940F1F82E394E00E941C
:107F2000951C0E944A1A60936506709366068093BA
:107F30006706909368060C94FB4C8091AA0690917A
:107F4000AB0605966AE270E00E947BD48C01009734
:107F500019F12091A0063091A10680E690E0AC01D5
:107F6000249FC001259F900D349F900D11248455AE
:107F7000994F6EE470E00E947BD460E270E00E9452
:107F80007BD49C012F5F3F4F3093AB062093AA0612
:107F900001501040F80110826091AA067091AB0662
:107FA0006B5F7F4F82E394E00E942B210C94FB4C8B
:107FB0000E944A1A6093690670936A0680936B0662
:107FC00090936C0620916506309166064091670695
:107FD00050916806621B730B840B950B28EE33E0FF
:107FE00040E050E00E94A2DCF22EE32ED42EC52EFB
:107FF0002DB73EB7285030400FB6F8943EBF0FBEA5
:108000002DBF0DB71EB70F5F1F4FCE010196EDB705
:10801000FEB79283818380ED97E0F801938382839A
:108020006F2D7E2D842F952F2CE330E040E050E023
:108030000E94A2DCF801358324836F2D7E2D8D2DC7
:108040009C2D2CE330E040E050E00E94A2DCF801DF
:10805000778366830E94CAD4E4EEF5E094912DB74D
:108060003EB7285F3F4F0FB6F8943EBF0FBE2DBFFF
:1080700008C08091C00085FFFCCF9093C600319668
:1080800094919923B1F7FE01319607C08091C00009
:1080900085FFFCCF31969093C60090819923B1F76C
:1080A0008091C00085FFFCCF8AE08093C6000C94CD
:1080B000FB4C83E50E94E933882311F40C94FB4CBC
:1080C0000E9438340E9443D67B018C016B0180E50D
:1080D0000E94E933882369F0F7FC0BC03FEFE316F9
:1080E000F10409F034F40E9438340E9443D68B0125
:1080F00002C008E010E0EEEDF3E08081918180178E
:10810000910711F40C94FB4C329644E0EE34F407E2
:10811000A1F70730110519F4C0925D0604C017FFDE
:1081200002C00C94FB4C802F61E00E94981B802FB2
:108130006C2D0E944B1C802FB6010E94BA1A0C9421
:10814000FB4C88E690E00E944134882311F00C94A7
:10815000FB4C83E50E94E933882379F00E94383490
:1081600020916E06022F10E0000F111F0C581F4EB9
:108170000E9443D6F801718360830E943C870C946F
:10818000FB4C83E50E94E933882311F40C94FB4CEB
:108190000E9438340E9443D6709377106093761013
:1081A0000C94FB4C89E690E00E944134882311F046
:1081B0000C94FB4CEAECF7E0949108C08091C0006D
:1081C00085FFFCCF9093C600319694919923B1F727
:1081D000E0916E06F0E0EE0FFF1FEE0FFF1FE65876
:1081E000FF4E408151816281738180EC98E021E0F3
:1081F00030E00E940D57E7ECF7E0949108C08091C1
:10820000C00085FFFCCF9093C600319694919923CE
:10821000B1F7E0916E06F0E0EE0FFF1FEC58FF4E55
:1082200060817181882777FD8095982F0E9476D68E
:10823000AB01BC0180EC98E021E030E00E940D57DA
:10824000E3ECF7E0949108C08091C00085FFFCCF7B
:108250009093C600319694919923B1F74091801084
:1082600050918110609182107091831080EC98E0A1
:1082700021E030E00E940D57E0ECF7E0949108C057
:108280008091C00085FFFCCF9093C60031969491F9
:108290009923B1F76091761070917710882777FD58
:1082A0008095982F0E9476D6AB01BC0180EC98E0B7
:1082B00021E030E00E940D57ECEBF7E0949108C00C
:1082C0008091C00085FFFCCF9093C60031969491B9
:1082D0009923B1F780916E060E948186BC0180ECE3
:1082E00098E04AE050E00E943A56E7EBF7E09491BC
:1082F00008C08091C00085FFFCCF9093C6003196E6
:1083000094919923B1F78FEF9FEF0E948186BC0172
:1083100080EC98E04AE050E00E943A56E4E9F2E04E
:1083200007C08091C00085FFFCCF31969093C600B6
:1083300090819923B1F78091C00085FFFCCF0C9408
:10834000194C8DE690E00E944134882311F00C9482
:10835000FB4C83E08093640683E50E94E933882325
:1083600079F00E94383420916E06022F10E0000F41
:10837000111F0C581F4E0E9443D6F8017183608371
:108380000E943C870E944A1A4B015C0120916E06B4
:10839000022F10E07724000F111FF801EC58FF4E58
:1083A00060817181882777FD8095982F0E9476D60D
:1083B000000F111F06581F4EF801208131814281A4
:1083C00053810E94D7D7181614F477247394CC24C1
:1083D000CA94DC2C7601E4EBF7E04490E0EBF7E0A4
:1083E0005490ECEAF7E064907AE0372E30C1942D97
:1083F000E4EBF7E008C08091C00085FFFCCF9093CC
:10840000C600319694919923B1F7E0916E06F0E0A1
:10841000EE0FFF1FEE0FFF1FE658FF4E4081518108
:108420006281738180EC98E021E030E00E940D577A
:10843000952DE0EBF7E008C08091C00085FFFCCFF0
:108440009093C600319694919923B1F760916E068E
:1084500080EC98E070E04AE050E00E943A56962D99
:10846000ECEAF7E008C08091C00085FFFCCF909354
:10847000C600319694919923B1F7F7FE03C0E5E960
:10848000F2E028C00E944A1AA70196012854344FEE
:108490004F4F5F4F261B370B480B590BCA01B901D1
:1084A00028EE33E040E050E00E94A2DC80EC98E04F
:1084B000BA01A9012AE030E00E94EB558091C0008A
:1084C00085FFFCCF0EC08091C00085FFFCCF3196A8
:1084D0009093C60090819923B1F78091C00085FFE9
:1084E000FCCF3092C6000E944A1A4B015C010E94E8
:1084F0006D8B0E9470300E94BF94FFEFCF16FFEF8C
:10850000DF06FFEFEF06FFEFFF0609F050C0E09136
:108510006E06772031F1F0E08F01000F111F000F80
:10852000111F06581F4EEE0FFF1FEC58FF4E6081C3
:108530007181882777FD8095982F0E9476D620E05C
:1085400030E040E050E40E94FAD49B01AC01F80115
:1085500060817181828193810E94D7D787FF5AC041
:1085600060C0F0E08F01000F111F000F111F0658AF
:108570001F4EEE0FFF1FEC58FF4E60817181882760
:1085800077FD8095982F0E9476D620E030E040E07D
:1085900050E40E94FBD49B01AC01F8016081718121
:1085A000828193810E94D4D51816A4F53AC0F7FCB5
:1085B00038C0E0916E06F0E08F01000F111F000F30
:1085C000111F06581F4EEE0FFF1FEC58FF4E608123
:1085D0007181882777FD8095982F0E9476D69B0120
:1085E000AC01F80160817181828193810E94FAD48B
:1085F0000E9443D697FF07C090958095709561952E
:108600007F4F8F4F9F4F64307105810591054CF06E
:10861000772039F40E944A1AAC01CB01DA016C01CF
:108620007D01FFEFCF16FFEFDF06FFEFEF06FFEF55
:10863000FF0669F0F7FE02C00C94FE4C0E944A1A35
:108640006C197D09685B7B4010F00C94FE4C0E9415
:108650004A1A681979098A099B09695E7340804042
:10866000904008F0C4CE43CF84E08093640683E555
:108670000E94E933882341F00E9438340E9443D697
:1086800070937710609376100E944A1A7B018C01D8
:10869000E9EAF7E0B490E5EAF7E0C490E1EAF7E050
:1086A000D490BAE0AB2E7DC00E944A1A6E197F09A1
:1086B000800B910B695E73408040904008F46BC062
:1086C000E0915C06F0E0EE0FFF1FEE0FFF1FE65893
:1086D000FF4E40815181628173819B2DE9EAF7E071
:1086E00008C08091C00085FFFCCF9093C6003196F2
:1086F00094919923B1F780EC98E022E030E00E9459
:108700000D579C2DE5EAF7E008C08091C00085FF79
:10871000FCCF9093C600319694919923B1F7609164
:108720005C0680EC98E070E04AE050E00E943A5627
:108730009D2DE1EAF7E008C08091C00085FFFCCFE5
:108740009093C600319694919923B1F7409180108F
:1087500050918110609182107091831080EC98E0AC
:1087600021E030E00E940D57E4E9F2E007C080917B
:10877000C00085FFFCCF31969093C600908199236D
:10878000B1F78091C00085FFFCCFA092C6000E9487
:108790004A1A7B018C010E946D8B0E9470300E94EE
:1087A000BF94609176107091771062507040882766
:1087B00077FD8095982F0E9476D69B01AC01609141
:1087C00080107091811080918210909183100E948E
:1087D000D4D587FD69CF0E944A1A609377067093BB
:1087E00078068093790690937A060C94FB4C83E587
:1087F0000E94E933882309F465C00E9438347B0164
:108800008C0160915C0370E0882777FD8095982F3C
:108810000E9476D69B01AC01C801B7010E94A9D87D
:1088200020E030E048EC52E40E94DBD520E030E06C
:1088300040E050E00E94D4D5882314F460E03EC0AC
:108840000E9438347B018C0160915C0370E08827C2
:1088500077FD8095982F0E9476D69B01AC01C801C8
:10886000B7010E94A9D820E030E048EC52E40E9411
:10887000DBD520E030E04FE753E40E94D7D718164D
:1088800014F46FEF1BC00E9438347B018C0160919F
:108890005C0370E0882777FD8095982F0E9476D63C
:1088A0009B01AC01C801B7010E94A9D820E030E0CB
:1088B00048EC52E40E94DBD50E9448D660935D06E6
:1088C0000C94FB4C80915C039FEF899FC0011124A5
:1088D00064E670E00E948FDC60935D060C94FB4CB4
:1088E00010925D060C94FB4C269A2E980C94FB4C2F
:1088F000269A2E9A0C94FB4C109231060C94FB4C49
:1089000081E0809331060C94FB4C83E50E94E933AF
:108910008823A1F00E94383420E030E04AE754E494
:108920000E94A9D80E9448D660936D0370936E038D
:1089300080936F03909370030C94FB4C88E50E9426
:10894000E933882311F00C94134D89E50E94E93333
:10895000882311F00C94134D8AE50E94E933882393
:1089600011F00C94134D85E40E94E933882311F033
:108970000C94134D0E943D7F409A0E944B7F0C94B3
:10898000FB4C159A89E50E94E9338111469A8AE5E4
:108990000E94E9338111439A85E40E94E9338823D8
:1089A00011F40C94FB4C409A0C94FB4C83E50E9410
:1089B000E933882311F40C94FB4C0E94383420E0F6
:1089C00030E04AE754E40E94A9D80E9448D6609358
:1089D0007B0670937C0680937D0690937E060C94B4
:1089E000FB4CE5ED6E2EE8E07E2E75EC272E78E050
:1089F000372E65E1462E69E0562E88249924F4012D
:108A0000E652FC4F80810E94E933882309F45DC05F
:108A100053E0851609F052C00E9438345B016C01A6
:108A200020E030E040EA51E40E94D4D588230CF0E5
:108A30003FC0F3016081718182819381A60195011C
:108A40000E94DBD57B018C0160910D0970910E09AC
:108A500080910F0990911009A80197010E94A9D84F
:108A600060930D0970930E0980930F09909310097C
:108A7000F1016081718182819381A80197010E9437
:108A8000A9D8F1016083718382839383F2016081AD
:108A90007181828193810E9474D6A80197010E94FE
:108AA000A9D80E9448D6F2016083718382839383A0
:108AB000F301A082B182C282D38207C00E943834FF
:108AC000F30160837183828393830894811C911CDA
:108AD00024E030E0620E731E220E331E420E531E3F
:108AE00034E08316910409F08ACF85C7E1E0F7E00E
:108AF000949108C08091C00085FFFCCF9093C60080
:108B0000319694919923B1F776C78091AA069091F6
:108B1000AB0605966AE270E00E947BD4FC010097E8
:108B200009F469C73197108266C7EEEFF6E09491B9
:108B300008C08091C00085FFFCCF9093C60031969D
:108B400094919923B1F74091340650913506609184
:108B500036067091370680EC98E022E030E00E9403
:108B60000D57EBEFF6E0949108C08091C00085FFAF
:108B7000FCCF9093C600319694919923B1F7409120
:108B800038065091390660913A0670913B0680ECA8
:108B900098E022E030E00E940D57E8EFF6E0949173
:108BA00008C08091C00085FFFCCF9093C60031962D
:108BB00094919923B1F740913C0650913D06609104
:108BC0003E0670913F0680EC98E022E030E00E9483
:108BD0000D57E5EFF6E0949108C08091C00085FF45
:108BE000FCCF9093C600319694919923B1F74091B0
:108BF000400650914106609142067091430680EC18
:108C000098E022E030E00E940D57EAEEF6E0949101
:108C100008C08091C00085FFFCCF9093C6003196BC
:108C200094919923B1F780E00E94277E0E9476D626
:108C30002091D5083091D6084091D7085091D80896
:108C40000E94DBD5AB01BC0180EC98E022E030E073
:108C50000E940D57E7EEF6E0949108C08091C000A5
:108C600085FFFCCF9093C600319694919923B1F77C
:108C700081E00E94277E0E9476D62091D90830910B
:108C8000DA084091DB085091DC080E94DBD5AB018B
:108C9000BC0180EC98E022E030E00E940D57E4EE49
:108CA000F6E0949108C08091C00085FFFCCF9093BE
:108CB000C600319694919923B1F782E00E94277EF5
:108CC0000E9476D62091DD083091DE084091DF08C1
:108CD0005091E0080E94DBD5AB01BC0180EC98E02C
:108CE00022E030E00E940D57E4E9F2E007C08091F5
:108CF000C00085FFFCCF31969093C60090819923E8
:108D0000B1F78091C00085FFFCCF8AE08093C60058
:108D100072C680E00E94D37D6EC681E00E94D37D42
:108D20006AC68091C00085FFFCCF31969093C60043
:108D300090819923B1F78091C00085FFFCCF8AE034
:108D40008093C600ECEDF6E0949108C08091C000DD
:108D500085FFFCCF9093C600319694919923B1F78B
:108D6000009B03C0E7E9F2E00AC0ECE9F2E007C0CB
:108D70008091C00085FFFCCF31969093C600908112
:108D80009923B1F78091C00085FFFCCF8AE08093E2
:108D9000C600E4EDF6E0949108C08091C00085FF24
:108DA000FCCF9093C600319694919923B1F7049B20
:108DB00003C0E7E9F2E00AC0ECE9F2E007C0809105
:108DC000C00085FFFCCF31969093C6009081992317
:108DD000B1F78091C00085FFFCCF8AE08093C60088
:108DE000ECECF6E0949108C08091C00085FFFCCFC8
:108DF0009093C600319694919923B1F7079B03C0D5
:108E0000E7E9F2E00AC0ECE9F2E007C08091C000B7
:108E100085FFFCCF31969093C60090819923B1F7DE
:108E20008091C00085FFFCCF8AE08093C600E3C537
:108E30000AED13E059EEE52E58E0F52EF801808199
:108E40000E94E933882349F00E9438340E9448D6B2
:108E5000F70160837183828393830F5F1F4F24E048
:108E600030E0E20EF31E33E00E3D130739F70E94A7
:108E70009C5AC1C50AED13E045ECE42E48E0F42EFF
:108E8000F80180810E94E933882339F00E94383448
:108E9000F70160837183828393830F5F1F4F24E008
:108EA00030E0E20EF31E33E00E3D130749F7A3C591
:108EB00083E50E94E933882351F00E94383460939F
:108EC000FD087093FE088093FF089093000984E5E5
:108ED0000E94E933882309F48EC50E9438346093D8
:108EE000010970930209809303099093040983C5D3
:108EF00083E50E94E933882351F00E94383460935F
:108F0000F9087093FA088093FB089093FC0884E5B5
:108F10000E94E933882351F00E943834609311098C
:108F200070931209809313099093140982E40E94AC
:108F3000E933882361F00E9438340E9448D6609358
:108F4000C1087093C2088093C3089093C40888E551
:108F50000E94E933882351F00E9438346093050958
:108F60007093060980930709909308098AE50E9487
:108F7000E933882351F00E943834609309097093D3
:108F80000A0980930B0990930C0985E40E94E93348
:108F9000882309F430C50E94383460930D0970931A
:108FA0000E0980930F099093100925C50AED13E06F
:108FB00034E4E32E36E0F32EF80180810E94E93399
:108FC000882339F00E943834F701608371838283EB
:108FD00093830F5F1F4F24E030E0E20EF31E33E077
:108FE0000D3D130749F707C583E50E94E933882340
:108FF00051F00E94383460935D0370935E03809358
:109000005F039093600386E40E94E933882351F064
:109010000E9438346093610370936203809363030A
:10902000909364038AE50E94E933882309F4E3C43A
:109030000E943834609365037093660380936703DE
:1090400090936803D8C483E50E94E933882351F0E4
:109050000E943834609360067093610680936206C4
:109060009093630686E40E94E933882309F4C3C41D
:109070000E9438346093690370936A0380936B0392
:1090800090936C03B8C483E50E94E933882309F404
:10909000B2C40E9438340E9443D6672B21F061305D
:1090A000710561F405C010925E0610925F06A3C4BC
:1090B00081E080935E0610925F069DC4E4EEF5E0C9
:1090C000949108C08091C00085FFFCCF9093C600AA
:1090D000319694919923B1F7E9EBF6E0949108C0A9
:1090E0008091C00085FFFCCF9093C600319694918B
:1090F0009923B1F72091A0063091A10680E690E077
:10910000289FF001299FF00D389FF00D1124E455A0
:10911000F94F07C08091C00085FFFCCF3196909336
:10912000C60090819923B1F7E7EBF6E0949108C06F
:109130008091C00085FFFCCF9093C600319694913A
:109140009923B1F78091C00085FFFCCF8AE080931E
:10915000C60051C483E50E94E933882309F44BC457
:109160000E9438340E9443D670934D0360934C03A1
:1091700042C483E50E94E933882309F43CC480910A
:109180005C06082F10E00E943834000F111F025BAC
:109190001C4F0E9443D6F801718360832CC480E584
:1091A0000E94E933882351F00E943834609385038C
:1091B00070938603809387039093880389E40E94C9
:1091C000E933882361F00E9438340E9460876093FD
:1091D000890370938A0380938B0390938C0384E4B8
:1091E0000E94E933882361F00E9438340E946C8722
:1091F00060938D0370938E0380938F0390939003FD
:1092000083E40E94E933882351F00E94383460934C
:1092100091037093920380939303909394030E941D
:109220005486E6EAF2E007C08091C00085FFFCCFDB
:1092300031969093C60090819923B1F7E9EAF2E064
:1092400007C08091C00085FFFCCF31969093C60087
:1092500090819923B1F740918503509186036091E5
:1092600087037091880380EC98E022E030E00E9450
:109270000D57EDEAF2E007C08091C00085FFFCCFFA
:1092800031969093C60090819923B1F7609189033C
:1092900070918A0380918B0390918C030E94668762
:1092A000AB01BC0180EC98E022E030E00E940D5759
:1092B000E1EBF2E007C08091C00085FFFCCF319662
:1092C0009093C60090819923B1F760918D037091BE
:1092D0008E0380918F03909190030E947287AB015F
:1092E000BC0180EC98E022E030E00E940D57E5EBF5
:1092F000F2E007C08091C00085FFFCCF31969093CB
:10930000C60090819923B1F7409191035091920347
:10931000609193037091940380EC98E022E030E038
:109320000E940D57E4E9F2E007C08091C00085FF7C
:10933000FCCF31969093C60090819923B1F780912C
:10934000C00085FFFCCF8AE08093C60054C380E54F
:109350000E94E933882351F00E94383460939503CA
:1093600070939603809397039093980389E40E94E7
:10937000E933882361F00E9438340E94608760934B
:10938000990370939A0380939B0390939C0384E4C6
:109390000E94E933882361F00E9438340E946C8770
:1093A00060939D0370939E0380939F039093A0030B
:1093B0000E945486E6EAF2E007C08091C00085FF73
:1093C000FCCF31969093C60090819923B1F7E9EADA
:1093D000F2E007C08091C00085FFFCCF31969093EA
:1093E000C60090819923B1F740919503509196035F
:1093F000609197037091980380EC98E022E030E050
:109400000E940D57EDEAF2E007C08091C00085FF91
:10941000FCCF31969093C60090819923B1F760916B
:10942000990370919A0380919B0390919C030E94F1
:109430006687AB01BC0180EC98E022E030E00E943E
:109440000D57E1EBF2E007C08091C00085FFFCCF33
:1094500031969093C60090819923B1F760919D0356
:1094600070919E0380919F039091A0030E94728748
:10947000AB01BC0180EC98E022E030E00E940D5787
:10948000E4E9F2E007C08091C00085FFFCCF31968F
:109490009093C60090819923B1F78091C00085FF19
:1094A000FCCF8AE08093C600A6C283E50E94E93320
:1094B000882329F460E070E080E090E002C00E9420
:1094C00038340E94935A97C285E40E94E933882376
:1094D00019F4CC24DD2412C00E9438340E9443D6F3
:1094E0006B0177FF0BC00F2EF0E0EF2EF0E0FF2EA8
:1094F000FCE80F2FF2E41F2FF02D0AC00F2EF0E032
:10950000EF2EF0E0FF2EF6E10F2FF3E41F2FF02DEA
:1095100083E50E94E933882321F00E9438347B01DF
:109520008C0183E40E94E933882319F425E030E0BC
:1095300005C00E9438340E9443D69B01C801B70180
:10954000A6010E94018E57C20E943D7F54C20E9414
:10955000E62D51C20E94E22C4EC20E94F8274BC257
:109560000E94962948C288E50E94E933882351F079
:109570000E9438340E9443D69B01AC0180E0B901BF
:109580000E945C7E8AE50E94E933882351F00E94A4
:1095900038340E9443D69B01AC0181E0B9010E949E
:1095A0005C7E85E40E94E933882309F424C20E948A
:1095B00038340E9443D69B01AC0182E0B9010E947D
:1095C0005C7E19C210926D068091730690917406AC
:1095D000A0917506B091760680936F069093700601
:1095E000A0937106B09372060E94493204C20E9491
:1095F0003FA501C288E50E94E933882311F400E009
:1096000003C00E942D34062F89E50E94E933882388
:1096100011F410E003C00E942D34162F83E50E9440
:10962000E933882309F4E7C14091AA065091AB06BB
:109630004F5F5F4F802F612F0E94319BDCC188E517
:109640000E94E933882311F400E003C00E942D3406
:10965000062F89E50E94E933882311F410E003C046
:109660000E942D34162F83E50E94E933882309F4E4
:10967000C2C14091AA065091AB064F5F5F4F802F49
:10968000612F0E94139CB7C188E50E94E9338823AB
:1096900011F4FF2403C00E942D34F62E89E50E94A8
:1096A000E933882311F400E003C00E942D34062F13
:1096B00087E50E94E933882311F411E003C00E947A
:1096C0002D34162F88E40E94E933882311F421E019
:1096D00003C00E942D34262F1F0D200F8F2D602FC9
:1096E000412F0E9466A087C188E50E94E933882344
:1096F00011F4FF2403C00E942D34F62E89E50E9448
:10970000E933882311F400E003C00E942D34062FB2
:1097100087E50E94E933882311F411E003C00E9419
:109720002D34162F88E40E94E933882311F421E0B8
:1097300003C00E942D34262F1F0D200F8F2D602F68
:10974000412F0E94699F57C188E50E94E933882311
:1097500011F4FF2403C00E942D34F62E89E50E94E7
:10976000E933882311F400E003C00E942D34062F52
:1097700087E50E94E933882311F411E003C00E94B9
:109780002D34162F88E40E94E933882311F421E058
:1097900003C00E942D34262F1F0D200F8F2D602F08
:1097A000412F0E94699F27C1E1EBF6E0949108C028
:1097B0008091C00085FFFCCF9093C60031969491B4
:1097C0009923B1F7609103157091041580EC98E02E
:1097D0004AE050E00E943A56109204151092031588
:1097E00080910615882399F0ECEAF6E0949108C080
:1097F0008091C00085FFFCCF9093C6003196949174
:109800009923B1F78091C00085FFFCCF12C0E7EA31
:10981000F6E0949108C08091C00085FFFCCF909342
:10982000C600319694919923B1F78091C00085FFCD
:10983000FCCF8AE08093C60001C184E50E94E93331
:10984000882309F48DC00E9438340E9448D6262F00
:1098500060936E066623B9F1E4EEF5E0949108C0DA
:109860008091C00085FFFCCF9093C6003196949103
:109870009923B1F7E9EBF2E007C08091C00085FFC2
:10988000FCCF31969093C60090819923B1F780EC7C
:1098900098E0622F40E050E00E94F655EBEBF2E0DA
:1098A00007C08091C00085FFFCCF31969093C60021
:1098B00090819923B1F78091C00085FFFCCF8AE0A9
:1098C0008093C60098C086E40E94E9338823E1F0C3
:1098D0000E9438347B018C0160939C0670939D0636
:1098E00080939E0690939F0620E030E040E050E099
:1098F0000E94D7D7181644F4E0927103F0927203D5
:109900000093730310937403E4EEF5E0949108C0A0
:109910008091C00085FFFCCF9093C6003196949152
:109920009923B1F7ECECF2E007C08091C00085FF0D
:10993000FCCF31969093C60090819923B1F7609146
:109940005C0680EC98E070E04AE050E00E943A56F5
:109950008091C00085FFFCCF8AE08093C6004BC099
:10996000E4EEF5E0949108C08091C00085FFFCCF43
:109970009093C600319694919923B1F7E4E9F6E00B
:10998000949108C08091C00085FFFCCF9093C600E1
:10999000319694919923B1F72091A0063091A106B8
:1099A00080E690E0289FF001299FF00D389FF00D90
:1099B0001124E455F94F07C08091C00085FFFCCF0A
:1099C00031969093C60090819923B1F7E2E9F6E0D1
:1099D000949108C08091C00085FFFCCF9093C60091
:1099E000319694919923B1F78091C00085FFFCCF07
:1099F0008AE08093C6000E94473020C00E944A1A25
:109A00006093650670936606809367069093680678
:109A10000E944A1A609377067093780680937906BD
:109A200090937A06E8CF0E943D7F88E50E94E93353
:109A3000882311F00C94C1440C94C2446E960FB666
:109A4000F894DEBF0FBECDBFCF91DF911F910F9174
:109A5000FF90EF90DF90CF90BF90AF909F908F904E
:109A60007F906F905F904F903F902F9008952F922E
:109A70003F924F925F926F927F928F929F92AF929E
:109A8000BF92CF92DF92EF92FF920F931F93DF93DB
:109A9000CF93CDB7DEB76E970FB6F894DEBF0FBE8B
:109AA000CDBF90E6A92EB12CE3E6F8E084908AE0E1
:109AB000782EE9EDF8E094906624639440C22D304E
:109AC00071F02A3321F480912D08882341F0809190
:109AD0002E0890912F088F3591050CF40CC2E0915F
:109AE0002E08F0912F08309709F45DC3A09130083B
:109AF000B0913108AA9D7001AB9DF00CBA9DF00C9D
:109B00001124EE0DFF1DE455F94F108280912D08B0
:109B1000882309F0EBC110922D08AE55B94F1C9265
:109B200087010455194FC8016EE470E00E947BD490
:109B30009C01009709F4F5C09093AB068093AA06A8
:109B40002F5F3F4F201B310B2E0D3F1DC901845548
:109B5000994F60E070E04AE050E00E9480D260934C
:109B60003208709333088093340890933508C0907E
:109B70006F06D0907006E0907106F0907206A70113
:109B800096012F5F3F4F4F4F5F4F62177307840758
:109B9000950709F4BAC380913008909131089C016F
:109BA0002A9DC0012B9D900D3A9D900D1124845546
:109BB000994F62E879E00E9440D4892B09F0A5C34F
:109BC000EAEEF5E0949108C08091C00085FFFCCFDB
:109BD0009093C600319694919923B1F7EFE4F9E0A0
:109BE000949108C08091C00085FFFCCF9093C6007F
:109BF000319694919923B1F780EC98E0B701A601D2
:109C00002AE030E00E9407568091C00085FFFCCF1B
:109C100071C0FE264F5FFC01E40FF11DE455F94FC2
:109C2000E081EA32B1F73093AB062093AA06C9016E
:109C3000019660E070E00E941AD10E9443D62F2D59
:109C400030E02617370709F45BC0EAEEF5E094919F
:109C500008C08091C00085FFFCCF9093C60031966C
:109C600094919923B1F7E0E3F9E0949108C08091D1
:109C7000C00085FFFCCF9093C60031969491992344
:109C8000B1F740916F065091700660917106709126
:109C9000720680EC98E02AE030E0B9D78091C000ED
:109CA00085FFFCCF27C0EAEEF5E0949108C08091D3
:109CB000C00085FFFCCF9093C60031969491992304
:109CC000B1F7E6E0F9E0949108C08091C00085FF0B
:109CD000FCCF9093C600319694919923B1F780EC14
:109CE00098E0B701A6012AE030E091D78091C0004A
:109CF00085FFFCCF8AE08093C6000E94493249C0AC
:109D00008091320890913308A0913408B0913508C1
:109D100080936F0690937006A0937106B0937206BD
:109D20003DC0C8016AE270E00E947BD4009709F44C
:109D300035C0EAEEF5E0949108C08091C00085FF3F
:109D4000FCCF9093C600319694919923B1F7ECED36
:109D5000F8E0949108C08091C00085FFFCCF9093FB
:109D6000C600319694919923B1F740916F065091B6
:109D70007006609171067091720680EC98E02AE09E
:109D800030E045D78091C00085FFFCCF8AE080930A
:109D9000C60010922F0810922E08D6C2809130086B
:109DA000909131088A9D70018B9DF00C9A9DF00C6A
:109DB000112487010455194FC80167E470E00E941F
:109DC0007BD49C01009709F445C09093AB06809327
:109DD000AA062F5F3F4F201B310B2E0D3F1DC901DF
:109DE0008455994F60E070E00E941AD10E9443D6DA
:109DF0006430710578F580916D068823B9F48091FF
:109E00003204882339F5992DE9EDF8E008C08091F6
:109E1000C00085FFFCCF9093C600319694919923A2
:109E2000B1F78091C00085FFFCCF12C0982DE3E60A
:109E3000F8E008C08091C00085FFFCCF9093C60079
:109E4000319694919923B1F78091C00085FFFCCFA2
:109E50007092C60080913008909131088A9D7001FF
:109E60008B9DF00C9A9DF00C112487010455194F1D
:109E7000C8016DE470E00E947BD49C019093AB0616
:109E80008093AA062F5F3F4F201B310B2E0D3F1DE5
:109E9000C9018455994F60E070E04AE050E00E94AB
:109EA00080D2693671058105910551F00E944A1AE8
:109EB0006093DF107093E0108093E1109093E210B4
:109EC0008091300890913108019664E070E00E9422
:109ED0008FDC909331088093300880913608909100
:109EE00037080196909337088093360810922F0810
:109EF00010922E0824C02B3311F460922D0880910B
:109F00002D088823E1F420912E0830912F088091AC
:109F10003008909131088A9DF0018B9DF00D9A9D3B
:109F2000F00D1124E20FF31FE455F94F80912C0836
:109F300080832F5F3F4F30932F0820932E0880910E
:109F4000BC089091BD082091BE083091BF08821BCB
:109F5000930B8F779070892B09F4F1C180913608AB
:109F60009091370804970CF0EAC180EC98E075D521
:109F7000282F80932C088A3009F0A1CDB0CD809194
:109F80002E0890912F08892B09F473C1DDC18091AF
:109F90003504882329F482E394E00E94911CF9CED1
:109FA0001092DB0510922F0810922E08409138086D
:109FB0005091390860913A0870913B0880911C06D5
:109FC00090911D06A0911E06B0911F0680509240F0
:109FD000A040B04084179507A607B70718F4109261
:109FE0003404B2C14093240650932506609326069C
:109FF0007093270681E096E00E94B16FA5C1262FDD
:10A0000060932C086A30A1F06D3091F06A3321F42E
:10A0100080912D08882361F080912E0890912F085F
:10A020008F3591052CF43FEF6F3F730709F0FCC0AB
:10A03000209124063091250640912606509127064E
:10A0400080911C0690911D06A0911E06B0911F06DE
:10A05000281739074A075B0720F46F5F7F4F09F025
:10A060009BC0962DE0E5F8E008C08091C00085FF18
:10A07000FCCF9093C600319694919923B1F78091CB
:10A08000C00085FFFCCF3092C6000E944A1A609340
:10A09000690670936A0680936B0690936C06209114
:10A0A0006506309166064091670650916806621B0E
:10A0B000730B840B950B28EE33E040E050E00E94D8
:10A0C000A2DCF22EE32ED42EC52EEDB7FEB73897C4
:10A0D0000FB6F894FEBF0FBEEDBF0DB71EB70F5FF2
:10A0E0001F4FB282A182F80153824282622F732FE6
:10A0F000842F952F20E13EE040E050E00E94A2DC5A
:10A10000F801358324836F2D7E2D8D2D9C2D2CE31E
:10A1100030E040E050E00E94A2DCCA01B9012CE32B
:10A1200030E040E050E00E94A2DCF80177836683D3
:10A130000E94CAD4972DE4EEF5E02DB73EB7285F14
:10A140003F4F0FB6F8943EBF0FBE2DBF08C08091A1
:10A15000C00085FFFCCF9093C6003196949199235F
:10A16000B1F7F50107C08091C00085FFFCCF3196A3
:10A170009093C60090819923B1F78091C00085FF2C
:10A18000FCCF3092C60082E394E00E941C1D82E363
:10A1900094E061E00E94822320912E0830912F08E4
:10A1A0002115310519F410922D08CEC08091300888
:10A1B00090913108889DF001899DF00D989DF00DDA
:10A1C0001124E20FF31FE455F94F1082FC01EE5504
:10A1D000F94F208220913608309137082F5F3F4F8A
:10A1E0003093370820933608019664E070E00E94AF
:10A1F0008FDC909331088093300810922D081092D4
:10A200002F0810922E088091240690912506A09187
:10A210002606B09127068093380890933908A093BA
:10A220003A08B0933B083AC02B3311F420922D0822
:10A2300080912D08882391F520912E0830912F08C8
:10A240008091300890913108889DF001899DF00D32
:10A25000989DF00D1124E20FF31FE455F94F809102
:10A260002C0880832F5F3F4F30932F0820932E08B8
:10A2700015C000E6802E912C22242394E0E5F8E01E
:10A2800064901AE0312E5E010894A11CB11CBCE35D
:10A290004B2EB8E05B2EE4EEF5E07490209124069E
:10A2A00030912506409126065091270680911C0684
:10A2B00090911D06A0911E06B0911F062817390720
:10A2C0004A075B0708F040C0809136089091370834
:10A2D0000497D4F58091090690910A06A0910B0687
:10A2E000B0910C068093240690932506A093260631
:10A2F000B093270681E096E00E944F73BC018091E5
:10A30000DB05882309F47BCE42CE80913008909102
:10A3100031088A9D80018B9D100D9A9D100D11248E
:10A32000C8018455994F6AE270E00E947BD49C0179
:10A33000009709F4B8CCFF2440E0C8016CCC8091B0
:10A340003404882309F01BCE6E960FB6F894DEBF56
:10A350000FBECDBFCF91DF911F910F91FF90EF9076
:10A36000DF90CF90BF90AF909F908F907F906F9035
:10A370005F904F903F902F900895CF93DF938091FF
:10A3800036089091370803970CF471DB82E394E070
:10A3900060E00E9482238091360890913708892BD3
:10A3A00009F469C080913204882309F44CC02091DB
:10A3B000A0063091A10680E690E0289FE001299F49
:10A3C000D00D389FD00D1124C455D94FCE016CE962
:10A3D00079E00E9440D4892BE1F482E394E0BE014D
:10A3E0000E941A1E80913304882369F5E9E9F9E097
:10A3F000949108C08091C00085FFFCCF9093C60067
:10A40000319694919923B1F78091C00085FFFCCFDC
:10A4100016C082E394E00E94011EE7E8F9E09491FF
:10A4200008C08091C00085FFFCCF9093C600319694
:10A4300094919923B1F78091C00085FFFCCF8AE009
:10A440008093C60002C00E945D36809136089091CC
:10A450003708019790933708809336088091A006BB
:10A460009091A106019664E070E00E948FDC9093C9
:10A47000A1068093A0060E946D8B0E9470300E94FE
:10A48000B6850E94BF94DF91CF910895269A2E98A9
:10A4900080EC98E040E950ED63E070E0AAD2E3E799
:10A4A000FAE0949108C08091C00085FFFCCF9093A2
:10A4B000C600319694919923B1F78091C00085FF31
:10A4C000FCCF8AE08093C60044EE55E0FA019491F7
:10A4D00008C08091C00085FFFCCF9093C6003196E4
:10A4E00094919923B1F784B7282F80FF15C0EBE62C
:10A4F000FAE0949108C08091C00085FFFCCF909352
:10A50000C600319694919923B1F78091C00085FFE0
:10A51000FCCF8AE08093C60021FF15C0EBE5FAE08E
:10A52000949108C08091C00085FFFCCF9093C60035
:10A53000319694919923B1F78091C00085FFFCCFAB
:10A540008AE08093C60022FF15C0EAE4FAE0949105
:10A5500008C08091C00085FFFCCF9093C600319663
:10A5600094919923B1F78091C00085FFFCCF8AE0D8
:10A570008093C60023FF15C0EAE3FAE0949108C077
:10A580008091C00085FFFCCF9093C60031969491D6
:10A590009923B1F78091C00085FFFCCF8AE08093BA
:10A5A000C60025FF15C0EAE2FAE0949108C0809148
:10A5B000C00085FFFCCF9093C600319694919923FB
:10A5C000B1F78091C00085FFFCCF8AE08093C60080
:10A5D00014BEE2E2FAE0949108C08091C00085FFC9
:10A5E000FCCF9093C600319694919923B1F7ECE19A
:10A5F000FAE0949108C08091C00085FFFCCF909351
:10A60000C600319694919923B1F78091C00085FFDF
:10A61000FCCF8AE08093C600FA019491E4EEF5E065
:10A6200008C08091C00085FFFCCF9093C600319692
:10A6300094919923B1F7ECE0FAE0949108C08091ED
:10A64000C00085FFFCCF9093C6003196949199236A
:10A65000B1F7E7EFF9E0949108C08091C00085FF61
:10A66000FCCF9093C600319694919923B1F7EBEE0D
:10A67000F9E0949108C08091C00085FFFCCF9093D1
:10A68000C600319694919923B1F7EDEDF9E09491DC
:10A6900008C08091C00085FFFCCF9093C600319622
:10A6A00094919923B1F78091C00085FFFCCF8AE097
:10A6B0008093C600E2EDF9E0949108C08091C0005B
:10A6C00085FFFCCF9093C600319694919923B1F702
:10A6D000E6ECF9E0949108C08091C00085FFFCCFC2
:10A6E0009093C600319694919923B1F78091C00060
:10A6F00085FFFCCF8AE08093C600FA019491E4EED6
:10A70000F5E008C08091C00085FFFCCF9093C600A3
:10A71000319694919923B1F7E7EBF9E0949108C051
:10A720008091C00085FFFCCF9093C6003196949134
:10A730009923B1F70E94E22EBC0180EC98E04AE038
:10A7400050E098D2E0EAF9E0949108C08091C0000E
:10A7500085FFFCCF9093C600319694919923B1F771
:10A7600080EC98E060ED74E04AE050E083D28091A4
:10A77000C00085FFFCCF8AE08093C6001092A2063D
:10A780001092A3061092A4061092A5060E94E22C35
:10A790000E94818A0E94875D0E940CD10E94C67E21
:10A7A0000C946A95BC018091360890913708049703
:10A7B0000CF070C0209130083091310880E690E0B4
:10A7C000AC01249FC001259F900D349F900D112452
:10A7D0008455994F0E94FBD3E4EEF5E0949108C0B4
:10A7E0008091C00085FFFCCF9093C6003196949174
:10A7F0009923B1F7EBE7FAE0949108C08091C0008B
:10A8000085FFFCCF9093C600319694919923B1F7C0
:10A81000209130083091310880E690E0289FF001C7
:10A82000299FF00D389FF00D1124E455F94F07C012
:10A830008091C00085FFFCCF31969093C600908137
:10A840009923B1F7E9E7FAE0949108C08091C0003C
:10A8500085FFFCCF9093C600319694919923B1F770
:10A860008091C00085FFFCCF8AE08093C600C901BB
:10A87000019664E070E00E948FDC90933108809331
:10A8800030088091360890913708019690933708E8
:10A89000809336080895BC0180913608909137085E
:10A8A00004970CF070C0209130083091310880E698
:10A8B00090E0AC01249FC001259F900D349F900D26
:10A8C00011248455994F0E9486D4E4EEF5E09491CA
:10A8D00008C08091C00085FFFCCF9093C6003196E0
:10A8E00094919923B1F7E8E8FAE0949108C0809137
:10A8F000C00085FFFCCF9093C600319694919923B8
:10A90000B1F7209130083091310880E690E0289F1F
:10A91000F001299FF00D389FF00D1124E455F94FF7
:10A9200007C08091C00085FFFCCF31969093C60090
:10A9300090819923B1F7E6E8FAE0949108C08091FC
:10A94000C00085FFFCCF9093C60031969491992367
:10A95000B1F78091C00085FFFCCF8AE08093C600EC
:10A96000C901019664E070E00E948FDC9093310889
:10A970008093300880913608909137080196909323
:10A9800037088093360808951F920F920FB60F92E2
:10A990000BB60F9211242F933F934F938F939F9356
:10A9A000EF93FF934091C600E091BC08F091BD0881
:10A9B00031969F012F77307031978091BE0890912A
:10A9C000BF082817390739F0E45CF74F408330930C
:10A9D000BD082093BC08FF91EF919F918F914F91FB
:10A9E0003F912F910F900BBE0F900FBE0F901F90B5
:10A9F00018959A01AB01203081EE380780E04807B6
:10AA000080E0580729F182E08093C00060E079E09F
:10AA10008DE390E00E94A2DC215030404040504045
:10AA200056954795379527953093C5002093C400D8
:10AA30008091C10080618093C1008091C1008860D5
:10AA40008093C1008091C10080688093C100089507
:10AA50001092C00020E130E0E7CF2091BE08309195
:10AA6000BF088091BC089091BD088217930719F424
:10AA70002FEF3FEF0EC0F901E45CF74F80812F5FAD
:10AA80003F4F2F7730703093BF082093BE08282F98
:10AA900030E0C90108958091BE089091BF0890935D
:10AAA000BD088093BC08089508952F923F924F925D
:10AAB0005F926F927F928F929F92AF92BF92CF924E
:10AAC000DF92EF92FF920F931F93DF93CF93CDB757
:10AAD000DEB7A0970FB6F894DEBF0FBECDBF1C0146
:10AAE0006A017B01411551056105710541F440E39F
:10AAF00050E060E070E020E030E089D053C088246E
:10AB000099245401422E55246624772401E010E054
:10AB10000C0F1D1F080D191DC701B601A3019201DD
:10AB20000E94A2DCF80160830894811C911CA11C86
:10AB3000B11CC701B601A30192010E94A2DCC901A8
:10AB4000DA016C017D01C114D104E104F104F1F6D4
:10AB500091E0E92EF12CEC0EFD1EE80CF91C3E01F3
:10AB60000894611C711CD501C4010197A109B109A8
:10AB70006C01C818D90813C0F601EE0DFF1D408105
:10AB80004A3010F4405D01C0495C50E060E070E084
:10AB9000C10120E030E03BD00894E108F1086E14D8
:10ABA0007F0451F7A0960FB6F894DEBF0FBECDBF5D
:10ABB000CF91DF911F910F91FF90EF90DF90CF9099
:10ABC000BF90AF909F908F907F906F905F904F90CD
:10ABD0003F902F9008952115310539F48091C000E0
:10ABE00085FFFCCF4093C60008955FCFEF92FF92A0
:10ABF0000F931F939A01E62EFF2400E010E0B801A6
:10AC0000A701E9DF1F910F91FF90EF900895EF9258
:10AC1000FF920F931F93CF93DF93EC017A018B0187
:10AC20002115310539F48091C00085FFFCCFE092F9
:10AC3000C60019C02A303105A9F477FF0FC04DE2D4
:10AC400050E060E070E020E030E0E1DF109500953A
:10AC5000F094E094E11CF11C011D111DCE01B8011E
:10AC6000A7012AE022DFDF91CF911F910F91FF9082
:10AC7000EF900895EF92FF920F931F937B019A013B
:10AC80000027F7FC0095102FB801A701C0DF1F9126
:10AC90000F91FF90EF9008950F931F938C014DE05B
:10ACA00050E060E070E020E030E0B1DFC8014AE051
:10ACB00050E060E070E020E030E0A9DF1F910F91EC
:10ACC0000895CF92DF92EF92FF920F931F938C0122
:10ACD0009A016B01EE24FF24B701A6017CDFC801B5
:10ACE000DBDF1F910F91FF90EF90DF90CF900895E1
:10ACF0009F92AF92BF92CF92DF92EF92FF920F930B
:10AD00001F93CF93DF93EC017A018B01922ECB013D
:10AD1000BA0120E030E040E050E00E94D4D5882322
:10AD200064F4CE014DE250E060E070E020E030E0FD
:10AD30006EDF17FB109517F9109520E030E040E02A
:10AD40005FE3AA240BC0CA01B90120E030E040E271
:10AD500051E40E94DBD59B01AC01A394A91498F3A4
:10AD6000C801B7010E94FBD47B018C010E9448D628
:10AD70005B016C010E9474D69B01AC01C801B70154
:10AD80000E94FAD47B018C01CE01B601A5012AE014
:10AD900030E021DF992099F1EEEDF2E007C08091DB
:10ADA000C00085FFFCCF31969093C6009081992317
:10ADB000B1F725C0C801B70120E030E040E251E41E
:10ADC0000E94A9D87B018C010E9443D65B016C01D3
:10ADD000CC24B7FCC094DC2CCE01B601A5012AE03E
:10ADE00030E015DFC601B5010E9476D69B01AC01AB
:10ADF000C801B7010E94FAD47B018C019A94992072
:10AE0000C9F6DF91CF911F910F91FF90EF90DF90E6
:10AE1000CF90BF90AF909F9008956ACF08952F92E2
:10AE20003F924F925F926F927F928F929F92AF92DA
:10AE3000BF92CF92DF92EF92FF920F931F93DF9317
:10AE4000CF93CDB7DEB7CD55D0400FB6F894DEBF67
:10AE50000FBECDBF2F969FAF8EAF2F9761967FAF5E
:10AE60006EAF61972A0162962FAF629763960FAF1C
:10AE700063976496EFAE64976896ACAEBDAECEAE07
:10AE8000DFAE6897E22EFF24EE0CFF1CEE0CFF1CD9
:10AE90009A012E0D3F1D2D963FAF2EAF2D97D90154
:10AEA0006D907D908D909C90FC01EE0DFF1DC40176
:10AEB000B30120813181428153810E94FBD469AF6B
:10AEC0007AAF8BAF9CAF10E0000F111F000F111F66
:10AED000F201E00FF11F2B96FFAFEEAF2B97A08092
:10AEE000B180C280D3802F96EEADFFAD2F97E00FDB
:10AEF000F11FC601B50120813181428153810E9439
:10AF0000FBD46DAB7EAB8FAB98AF64962FAD6497DF
:10AF1000E22FF0E0EE0FFF1FEE0FFF1F2F96AEADFA
:10AF2000BFAD2F97AE0FBF1F4D915D916D917C917D
:10AF300029964CAF5DAF6EAF7FAF299761966EAD2E
:10AF40007FAD6197E60FF71F6081718182819381E8
:10AF500029962CAD3DAD4EAD5FAD29970E94FAD438
:10AF600069AB7AAB8BAB9CAB6196AEADBFAD619775
:10AF70001C968D919D910D90BC91A02D25968CAF26
:10AF80009DAFAEAFBFAF25972F96AEADBFAD2F979C
:10AF90001C962D913D914D915C911F9721962CAF60
:10AFA0003DAF4EAF5FAF2197A401930150582DA73D
:10AFB0003EA74FA758ABB601A501705849A75AA79D
:10AFC0006BA77CA761966EAD7FAD6197E60EF71E0D
:10AFD000D7016D917D918D919C9129AD3AAD4BAD8D
:10AFE0005CAD0E94FAD43B014C016196EEADFFAD21
:10AFF00061970E0F1F1FD8016D917D918D919C91CE
:10B000002DA93EA94FA958AD0E94FAD45B016C014D
:10B010006DA57EA58FA598A9A60195010E94A9D826
:10B020007B018C0169A57AA58BA59CA5A401930140
:10B030000E94A9D89B01AC01C801B7010E94FAD4B3
:10B040001B012C016DA57EA58FA598A9A4019301D4
:10B050000E94A9D87B018C0169A57AA58BA59CA526
:10B06000A60195010E94A9D89B01AC01C801B701B6
:10B070000E94FBD49B01AC01C201B1010E946ED5BC
:10B080005B016C0120E030E040E050E00E94D4D54C
:10B09000882354F4C601B5012BED3FE049EC50E4A0
:10B0A0000E94FBD45B016C01E8968FADE897882382
:10B0B00051F0C601B5012BED3FE049EC50E40E9490
:10B0C000FAD45B016C01C601B501E7962CAD3DAD2C
:10B0D0004EAD5FADE7970E94A9D829A93AA94BA91F
:10B0E0005CA95F770E94E4D77B018C012FE632E1F7
:10B0F00043E85AE30E94D4D587FDF4C1C801B701E3
:10B100000E94B1D60E9448D678A76FA3672B21F47E
:10B11000E1E0F0E0F8A7EFA32FA138A5B90180E0A6
:10B1200090E00E9474D67B018C01C601B501A80194
:10B1300097010E94DBD56BA37CA38DA39EA369A975
:10B140007AA98BA99CA9A80197010E94DBD56F8FD2
:10B1500078A389A39AA325966CAD7DAD8EAD9FADE6
:10B16000259721962CAD3DAD4EAD5FAD21970E9448
:10B17000FAD4A80197010E94DBD56B8F7C8F8D8F4D
:10B180009E8F6BA17CA18DA19EA120E030E040E0CC
:10B190005FEB0E94A9D82BA13CA14DA15EA10E940A
:10B1A000A9D820E030E040E85FE30E94FBD46F8B39
:10B1B000788F898F9A8F64963FAD6497E32FF0E084
:10B1C000EE0FFF1FEE0FFF1F9E012F5F3F4FE20F9D
:10B1D000F31F29964CAD5DAD6EAD7FAD29974083D1
:10B1E0005183628373832F96AEADBFAD2F971C96AC
:10B1F0004D915D916D917C911F974D875E876F8713
:10B20000788B41E050E05A8B498B662462967FAD83
:10B210006297672F70E0660F771F660F771FC9016F
:10B22000860F971F6A969FAF8EAF6A976396BFADE2
:10B230006397AB2FB0E0AA0FBB1FAA0FBB1F21E083
:10B2400030E02C0F3D1F2A0F3B1F6C963FAF2EAFF7
:10B250006C976E96FFAFEEAF6E9719C138E1361559
:10B260000CF446C06DA57EA58FA598A92BA13CA185
:10B270004DA15EA10E94A9D87B018C0169A57AA588
:10B280008BA59CA52F89388D498D5A8D0E94A9D8F0
:10B290009B01AC01C801B7010E94FBD47B018C016A
:10B2A0006DA57EA58FA598A92F89388D498D5A8DBA
:10B2B0000E94A9D85B016C0169A57AA58BA59CA504
:10B2C0002BA13CA14DA15EA10E94A9D89B01AC017C
:10B2D000C601B5010E94FAD46DA77EA78FA798ABCF
:10B2E0006394C701D80189A79AA7ABA7BCA765C07B
:10B2F00049895A89BA0180E090E00E9474D62BA156
:10B300003CA14DA15EA10E94A9D87B018C01C8017E
:10B310000E94D8D56B8B7C8B8D8B9E8BB701C8011F
:10B320000E940CD93B014C012D96AEADBFAD2D97BF
:10B33000ED90FD900D911C9117FB109517F910954C
:10B340002B96EEADFFAD2B9720803180428053804D
:10B35000C801B7012B893C894D895E890E94A9D813
:10B360005B016C01C201B101A40193010E94A9D843
:10B370009B01AC01C601B5010E94FBD46DA77EA75D
:10B380008FA798ABC801B701A40193010E94A9D867
:10B390007B018C01C201B1012B893C894D895E89F9
:10B3A0000E94A9D89B01AC01C801B7010E94FAD440
:10B3B00069A77AA78BA79CA7662469AD7AAD8BADE8
:10B3C0009CAD2DA53EA54FA558A90E94FBD46A9619
:10B3D000AEADBFAD6A976D937D938D939C9313979C
:10B3E0006DA97EA98FA998AD29A53AA54BA55CA505
:10B3F0000E94FBD46C96EEADFFAD6C9760837183B9
:10B40000828393836E96AEADBFAD6E976D917D9145
:10B410008D919C912F8D38A149A15AA10E94FBD4F6
:10B420006E96EEADFFAD6E976083718382839383DA
:10B430006D857E858F8598892B8D3C8D4D8D5E8D9C
:10B440000E94FBD46D877E878F87988BCE010196F3
:10B450000E940A2FCE010196BE016B5F7F4FAE01A5
:10B46000475F5F4F9E01235F3F4F6896ECACFDAC9A
:10B470000EAD1FAD6897F8E7CF2ED12CCC0EDD1E98
:10B480000FD629893A892F5F3F4F3A8B298B4989FB
:10B490005A896FA178A54617570708F4DFCE619641
:10B4A0004EAD5FAD6197485F5F4F61962EAD3FAD8A
:10B4B0006197245F3F4F61968EAD9FAD6197DC0130
:10B4C00014966196BFAFAEAF6197BD016896ECACC4
:10B4D000FDAC0EAD1FAD6897E8E7CE2ED12CCC0E9B
:10B4E000DD1EDED5C35ADF4F0FB6F894DEBF0FBEA8
:10B4F000CDBFCF91DF911F910F91FF90EF90DF9023
:10B50000CF90BF90AF909F908F907F906F905F9003
:10B510004F903F902F9008958091050E9091060EC8
:10B52000891B8F70089560937603709377038093DF
:10B5300078039093790308950F931F93CF93DF932C
:10B54000C0E0D0E08E010B5E164FFE01E751F74FD1
:10B5500060817181828193810E9474D6FE01EB52D9
:10B56000F74F20813181428153810E94A9D80E94E6
:10B5700048D6F80160837183828393832496C03117
:10B58000D10501F7DF91CF911F910F910895FC0133
:10B5900060817181828193812091E1083091E2087C
:10B5A0004091E3085091E4080E94A9D8E0915C061C
:10B5B000F0E0EE0FFF1FEE0FFF1FEB51F74F208162
:10B5C0003181428153810E94A9D80E9479D8609329
:10B5D000310970933209809333099093340981E3E0
:10B5E00099E00C94167E8F929F92AF92BF92CF9269
:10B5F000DF92EF92FF920F931F93FC018B015A0190
:10B60000490160817181828193812091D5083091B7
:10B61000D6084091D7085091D8080E94A9D80E9416
:10B6200079D855E2C52E59E0D52E6093250970933F
:10B6300026098093270990932809F8016081718178
:10B64000828193812091D9083091DA084091DB08FA
:10B650005091DC080E94A9D80E9479D844E0E42ED9
:10B66000F12CEC0CFD1C60932909F7017183828396
:10B670009383F50160817181828193812091DD083E
:10B680003091DE084091DF085091E0080E94A9D86F
:10B690000E9479D88601085F1F4F60932D09F80139
:10B6A000718382839383F4016081718182819381AC
:10B6B0002091E1083091E2084091E3085091E408BC
:10B6C0000E94A9D8E0915C06F0E0EE0FFF1FEE0F9C
:10B6D000FF1FEB51F74F20813181428153810E943E
:10B6E000A9D80E9479D8F6013C96609331097183FC
:10B6F00082839383C601B701A8019F010E94DC7D6C
:10B7000080E090E0A0E0B0E08093070E9093080EF8
:10B71000A093090EB0930A0E80930B0E90930C0E1B
:10B72000A0930D0EB0930E0E80930F0E9093100EFB
:10B73000A093110EB093120E8093130E9093140EDB
:10B74000A093150EB093160E8093170E9093180EBB
:10B75000A093190EB0931A0E1F910F91FF90EF90C6
:10B76000DF90CF90BF90AF909F908F9008958F9271
:10B770009F92AF92BF92CF92DF92EF92FF920F9380
:10B780001F93CF93DF93EC016B01009709F45CC02A
:10B790008FA9882309F058C0EEA0FFA008A519A51D
:10B7A000FB01B6A0A7A090A481A4C801B7012B2DCE
:10B7B0003A2D492D582D0E94D4D588230CF044C031
:10B7C000C801B701A80197010E94A9D87B018C018B
:10B7D0006AA97BA98CA99DA9905820E030E040E09F
:10B7E00050EC0E94A9D82EA53FA548A959A90E94AE
:10B7F000A9D89B01AC01C801B7010E94FBD40E94EB
:10B8000016D97B018C016B2D7A2D892D982D9701EE
:10B81000A8010E94D4D5882324F4EB2CFA2C092DFE
:10B82000182D6B2D7A2D892D982D9701A8010E9436
:10B83000D4D5882349F0C701D801F60186A397A380
:10B84000A0A7B1A781E086ABDF91CF911F910F91A7
:10B85000FF90EF90DF90CF90BF90AF909F908F9030
:10B860000895EF92FF920F931F93CF93DF93F09081
:10B87000060E00E010E020E030E06DE4E62E11C09E
:10B88000FE9CE0011124CB5CD64FC901B801AE018A
:10B890006EDF8F2D8F5F803109F480E0F82E9801E4
:10B8A0008E018091050EF81659F7C901B80140E0E4
:10B8B00050E05DDFDF91CF911F910F91FF90EF90EE
:10B8C0000895AF92BF92CF92DF92EF92FF920F93C3
:10B8D0001F93CF93DF93EB018A016115710509F482
:10B8E00066C04115510509F462C0DAA4CBA4BCA41A
:10B8F000ADA46EA17FA188A599A52D2D3C2D4B2D22
:10B900005A2D0E94D4D5882309F451C08FA98823C9
:10B9100009F043C0F801E6A0F7A000A511A56D2D20
:10B920007C2D8B2D9A2DA80197010E94D7D7181630
:10B93000A4F5C801B701A80197010E94A9D87B010D
:10B940008C016AA97BA98CA99DA9905820E030E0C0
:10B9500040E050EC0E94A9D82EA53FA548A959A9BE
:10B960000E94A9D89B01AC01C801B7010E94FBD479
:10B970000E9416D97B018C016D2D7C2D8B2D9A2D6B
:10B980009701A8010E94D4D5882324F4ED2CFC2C27
:10B990000B2D1A2DC701D80104C08D2D9C2DAB2D68
:10B9A000BA2D8EA39FA3A8A7B9A781E08EABDF9184
:10B9B000CF911F910F91FF90EF90DF90CF90BF90AC
:10B9C000AF900895CF92DF92EF92FF920F93DF93A3
:10B9D000CF930F920F92CDB7DEB78091050E8FB740
:10B9E000F894F090060E8FBF8091050E90E040967F
:10B9F0008F1991098F7090700497FCF00091050EDB
:10BA000003500F70CC24DD2440E050E07DE4E72EAD
:10BA100012C0802F002309F480E1082F01500E9DF1
:10BA2000C00111248B5C964F9A838983B60149DF4C
:10BA3000A601C980DA800F1561F70F900F90CF91A2
:10BA4000DF910F91FF90EF90DF90CF900895DF92FC
:10BA5000EF92FF920F931F93D0905D069091060E88
:10BA60008091050E9817C1F04091060E242F30E00A
:10BA70008DE490E0289FF001299FF00D389FF00D94
:10BA80001124E358F64F608102C04F5F4F708091E0
:10BA9000050E4817D1F7D62EDD2031F1E0901B0EB0
:10BAA000F0901C0E00911D0E10911E0EE114F10479
:10BAB0000105110579F40E944A1A6C597F4F8F4F86
:10BAC0009F4F60931B0E70931C0E80931D0E9093DE
:10BAD0001E0E07C00E944A1A6E157F058007910747
:10BAE00058F4DD24DA9408C010921B0E10921C0E3C
:10BAF00010921D0E10921E0E87E06D2D70E00E94B8
:10BB0000BA1A1F910F91FF90EF90DF900895109255
:10BB1000050E1092060E80E1E5E2F9E0DF011D92CC
:10BB20008A95E9F780E090E0A0E0B0E080930B0E0A
:10BB300090930C0EA0930D0EB0930E0E80930F0EEB
:10BB40009093100EA093110EB093120E8093130ECB
:10BB50009093140EA093150EB093160E8093170EAB
:10BB60009093180EA093190EB0931A0E8093070E9F
:10BB70009093080EA093090EB0930A0E80E090E017
:10BB8000A0E8BFE38093E5089093E608A093E70858
:10BB9000B093E80808952F923F924F925F926F9270
:10BBA0007F928F929F92AF92BF92CF92DF92EF924D
:10BBB000FF920F931F93DF93CF93CDB7DEB76697B6
:10BBC0000FB6F894DEBF0FBECDBF9E8B8D8B6A0182
:10BBD0007B0148015901DC01D8966D917D918D91D1
:10BBE0009C91DB970E9474D6698B7A8B8B8B9C8B94
:10BBF000A70196010E94A9D80E94C1D50E9448D6EB
:10BC00006D837E838F83988769897A898B899C89E4
:10BC1000A50194010E94A9D80E94C1D50E9448D6CE
:10BC200069837A838B839C832D813E814F815885E4
:10BC3000283731054105510540F448E750E060E000
:10BC400070E04D835E836F83788769817A818B8111
:10BC50009C81683771058105910540F488E790E083
:10BC6000A0E0B0E089839A83AB83BC83AD89BE89B1
:10BC7000AC5BBF4FAD90BD90CD90DC901397A454BA
:10BC8000B040BE8BAD8B6D817E818F8198850E9487
:10BC900074D66D877E878F87988BC601B5010E9409
:10BCA00076D61B012C0120E030E040E050E00E94FD
:10BCB000D4D5882321F4E0E070E060E028C06989F1
:10BCC0007A898B899C899B01AC010E94A9D87B0150
:10BCD0008C016D857E858F8598899B01AC010E94C2
:10BCE000A9D89B01AC01C801B7010E94FAD47B011D
:10BCF0008C01C201B101A20191010E94FBD49B0100
:10BD0000AC01C801B7010E94DBD5E62F692F2E2FA9
:10BD1000372F482F562FB901CA010E94C1D50E9462
:10BD200043D63B014C0169817A818B819C810E94C1
:10BD300074D669877A878B879C8766277727CB019C
:10BD40006A197B098C099D090E9476D65B016C01FA
:10BD500020E030E040E050E00E94D4D5882321F478
:10BD6000E0E070E060E028C069857A858B859C857D
:10BD70009B01AC010E94A9D87B018C0169897A8959
:10BD80008B899C899B01AC010E94A9D89B01AC01C5
:10BD9000C801B7010E94FAD47B018C01C601B5012C
:10BDA000A60195010E94FBD49B01AC01C801B7011B
:10BDB0000E94DBD5E62F692F2E2F372F482F562FC5
:10BDC000B901CA010E94B1D6ED89FE89A088B18867
:10BDD000C288D38886017501E618F7080809190991
:10BDE0000E9443D6A8019701261B370B480B590B1D
:10BDF00057FF71C0C201B10120E030E040E050E0E7
:10BE00000E94D4D5882321F4E0E070E060E044C0D3
:10BE1000C201B101A20191010E94FBD47B018C01FE
:10BE2000C601B5010E9474D69B01AC01C801B701DF
:10BE30000E94A9D87B018C016D857E858F859889AC
:10BE40009B01AC010E94A9D89B01AC01C801B701BC
:10BE50000E94FAD47B018C0169857A858B859C854B
:10BE60009B01AC010E94A9D89B01AC01C801B7019C
:10BE70000E94FBD47B018C01C201B10120E030E0C3
:10BE800040E850E40E94A9D89B01AC01C801B70169
:10BE90000E94DBD5E62F692F2E2F372F482F562FE4
:10BEA000B901CA010E94C1D50E9443D6AC01CB01A1
:10BEB000DA013C014D0197FE03C06624772443015B
:10BEC0006A147B048C049D0410F03501460120E0C7
:10BED00030E040E050E09FB7F8946D897E89645B64
:10BEE0007F4FDB018C91AC54B040BE8BAD8B88236F
:10BEF00021F5FD01648A758A868A978A260D371D89
:10BF0000481D591D58962D933D934D935C935B9717
:10BF10002D813E814F815885DC962D933D934D9325
:10BF20005C93DF97A05CBF4F29813A814B815C8194
:10BF30002D933D934D935C9313979FBF66960FB6D9
:10BF4000F894DEBF0FBECDBFCF91DF911F910F914F
:10BF5000FF90EF90DF90CF90BF90AF909F908F9029
:10BF60007F906F905F904F903F902F9008954F92E9
:10BF70005F927F928F929F92AF92BF92CF92DF9209
:10BF8000EF92FF920F931F93CF93DF937090060E63
:10BF9000C0E0D0E0EDE44E2E512C45C02097A9F131
:10BFA0008EA9882361F4849CF001859CF00D949CFB
:10BFB000F00D1124EB5CF64F86A9882331F1EAA03D
:10BFC000FBA00CA11DA16EA17FA188A599A5A80128
:10BFD00097010E94DBD55B016C01849CF001859C7C
:10BFE000F00D949CF00D1124EB5CF64F66A177A147
:10BFF00080A591A5A80197010E94DBD58B019C012A
:10C00000CE01B601A501C7DD1EAA739480E17816A2
:10C0100009F47724849CE001859CD00D949CD00D7C
:10C020001124CB5CD64F872C992487FC9094809167
:10C03000050E90E08816990609F0B0CF2097E9F038
:10C04000EAA0FBA00CA11DA16EA17FA188A599A5C6
:10C05000A80197010E94DBD55B016C016DEC7CECC3
:10C060008CE49DE3A80197010E94DBD58B019C0124
:10C07000CE01B601A5018FDD1EAADF91CF911F91E0
:10C080000F91FF90EF90DF90CF90BF90AF909F9077
:10C090008F907F905F904F90089594DCE2DB67CFA4
:10C0A0002F923F924F925F926F927F928F929F92C8
:10C0B000AF92BF92CF92DF92EF92FF920F931F93B6
:10C0C000DF93CF93CDB7DEB7C659D0400FB6F89403
:10C0D000DEBF0FBECDBF5C014B013A012901CD5639
:10C0E000DF4FE882C359D040CC56DF4FF882C459A5
:10C0F000D040CB56DF4F0883C559D040CA56DF4FDA
:10C100001883C659D040E196DFAECEAEE19780915C
:10C11000050E8F5F803109F480E0282F332727FD3B
:10C1200030953CA72BA706C00E946D8B0E947030F3
:10C130000E94BF948091060E90E04BA55CA58417E9
:10C14000950791F36091D5087091D6088091D70832
:10C150009091D808AF966CAF7DAF8EAF9FAFAF9781
:10C16000D5012D913D914D915C910E94A9D80E94DD
:10C1700079D8EE966FAFEE97EF967FAFEF97C158F5
:10C18000DF4F8883CF57D040C058DF4F9883C058C7
:10C19000D0402091D9083091DA084091DB085091C5
:10C1A000DC08AB962CAF3DAF4EAF5FAFAB97CA018B
:10C1B000B901D4012D913D914D915C910E94A9D876
:10C1C0000E9479D8CF57DF4F6883C158D040CE57EF
:10C1D000DF4F7883C258D040CD57DF4F8883C35894
:10C1E000D040CC57DF4F9883C458D0402091DD0811
:10C1F0003091DE084091DF085091E008A7962CAFFF
:10C200003DAF4EAF5FAFA797CA01B901D3012D91E2
:10C210003D914D915C910E94A9D80E9479D8CB574D
:10C22000DF4F6883C558D040CA57DF4F7883C65860
:10C23000D040C957DF4F8883C758D040C857DF4F19
:10C240009883C858D0402091E1083091E20840918D
:10C25000E3085091E408A3962CAF3DAF4EAF5FAF1B
:10C26000A397E196AEADBFADE1978C91082F10E09A
:10C27000CA01B901F20120813181428153810E94BA
:10C28000A9D8000F111F000F111FF801EB51F74F34
:10C2900020813181428153810E94A9D80E9479D89E
:10C2A000C757DF4F6883C958D040C657DF4F7883E0
:10C2B000CA58D040C557DF4F8883CB58D040C457A9
:10C2C000DF4F9883CC58D04080913109909132094A
:10C2D000A0913309B0913409C757DF4F28813981C4
:10C2E0004A815B81C958D040281739074A075B0744
:10C2F00009F4B2C006581F4ED8016D917D918D9101
:10C300009C9120917603309177034091780350916E
:10C3100079030E94D4D588230CF033C0C757DF4F70
:10C32000288139814A815B81C958D04020933109E5
:10C33000309332094093330950933409E3E9FAE02A
:10C34000949108C08091C00085FFFCCF9093C600F7
:10C35000319694919923B1F7E7EBFAE0949108C0F4
:10C360008091C00085FFFCCF9093C60031969491D8
:10C370009923B1F78091C00085FFFCCF8AE08093BC
:10C38000C6008091310990913209A0913309B09192
:10C390003409C757DF4F288139814A815B81C958E9
:10C3A000D040281B390B4A0B5B0BCA01B90157FF60
:10C3B00007C090958095709561957F4F8F4F9F4FE7
:10C3C0000E9476D67B018C01A3966CAD7DAD8EADBF
:10C3D0009FADA39720E030E046EE53E40E94A9D839
:10C3E0009B01AC01C801B7010E94D7D718160CF009
:10C3F00033C0C757DF4F488159816A817B81C95853
:10C40000D0404093310950933209609333097093BF
:10C410003409E3E9FAE0949108C08091C00085FFF7
:10C42000FCCF9093C600319694919923B1F7E9E936
:10C43000FAE0949108C08091C00085FFFCCF9093F2
:10C44000C600319694919923B1F78091C00085FF81
:10C45000FCCF8AE08093C6008091050E682F70E0C3
:10C460006F967FAF6EAF6F978DE490E0689FF0019D
:10C47000699FF00D789FF00D1124EB5CF64FE45BA3
:10C48000FF4F1082EC54F0408091250990912609CD
:10C49000A0912709B09128096D968CAF9DAFAEAFE2
:10C4A000BFAF6D97C358DF4F288139814A815B81C7
:10C4B000CD57D040281B390B4A0B5B0B69962CAF2C
:10C4C0003DAF4EAF5FAF6997208331834283538383
:10C4D00057FF0DC0DA01C901B095A09590958195DF
:10C4E0009F4FAF4FBF4F80839183A283B38340910F
:10C4F000290950912A0960912B0970912C096596A0
:10C500004CAF5DAF6EAF7FAF6597CF57DF4F888180
:10C510009981AA81BB81C158D040841B950BA60B81
:10C52000B70B61968CAF9DAFAEAFBFAF61978DE497
:10C5300090E06F96AEADBFAD6F97A89FF001A99F39
:10C54000F00DB89FF00D1124EB5CF64F61962CAD09
:10C550003DAD4EAD5FAD61972483358346835783F0
:10C5600057FF0DC0DA01C901B095A095909581954E
:10C570009F4FAF4FBF4F84839583A683B78340916E
:10C580002D0950912E0960912F09709130092D9637
:10C590004CAF5DAF6EAF7FAF2D97CB57DF4F88812C
:10C5A0009981AA81BB81C558D040841B950BA60BED
:10C5B000B70B29968CAF9DAFAEAFBFAF29978DE477
:10C5C00090E06F96AEADBFAD6F97A89FF001A99FA9
:10C5D000F00DB89FF00D1124EB5CF64F29962CADB1
:10C5E0003DAD4EAD5FAD2997208731874287538798
:10C5F00057FF0DC0DA01C901B095A09590958195BE
:10C600009F4FAF4FBF4F80879187A287B3872090FE
:10C610003109309032094090330950903409C7579E
:10C62000DF4F488159816A817B81C958D0404219C6
:10C630005309640975094DA35EA36FA378A79A01F6
:10C64000AB0157FF07C050954095309521953F4F5E
:10C650004F4F5F4F8DE490E06F966EAD7FAD6F975B
:10C66000689F8001699F100D789F100D11240B5C4D
:10C67000164F7CE0E72EF12CE00EF11EE196AEADF8
:10C68000BFADE197EC91F0E0EE0FFF1FE25BFC4FD6
:10C6900060817181882777FD8095982F0E9450DCFA
:10C6A00024E630E040E050E00E94C4DCF80124873A
:10C6B000D70111963C93119712964C9312971396AB
:10C6C0005C936080718082809380A480B580C680F6
:10C6D000D780E084F18402851385C901DA018E15C3
:10C6E0009F05A007B10714F4D801C7018A159B055F
:10C6F000AC05BD0514F4D601C5019C01AD0186153C
:10C700009705A805B90514F4A40193018DE490E000
:10C710006F96EEADFFAD6F97E89FB001E99F700D8A
:10C72000F89F700D11246B5C764FDB0150962D93B2
:10C730003D934D935C935397263031054105510548
:10C7400010F40C948E6CFB01E85BFF4F80915D064A
:10C7500090E0A0E0B0E080839183A283B383FB01EB
:10C7600010A2C358DF4F288139814A815B81CD57A0
:10C77000D0406D968CAD9DADAEADBFAD6D97281719
:10C7800039074A075B0714F481E080A3CF57DF4FD6
:10C79000288139814A815B81C158D04065966CAD52
:10C7A0007DAD8EAD9FAD65972617370748075907B2
:10C7B00094F48DE490E06F96AEADBFAD6F97A89FF7
:10C7C000F001A99FF00DB89FF00D1124EB5CF64F1E
:10C7D00080A1826080A3CB57DF4F288139814A81B5
:10C7E0005B81C558D0402D966CAD7DAD8EAD9FADB3
:10C7F0002D97261737074807590794F48DE490E0E2
:10C800006F96AEADBFAD6F97A89FF001A99FF00DD9
:10C81000B89FF00D1124EB5CF64F80A1846080A3DB
:10C82000C757DF4F288139814A815B81C958D04081
:10C83000221533054405550594F48DE490E06F9678
:10C840004EAD5FAD6F97489FF001499FF00D589F27
:10C85000F00D1124EB5CF64F80A1886080A38DE47D
:10C8600090E06F966EAD7FAD6F97689FF001699F06
:10C87000F00D789FF00D1124EB5CF64FE196AEAD14
:10C88000BFADE1978C9181A3208131814281538199
:10C8900025962CAF3DAF4EAF5FAF259721153105E3
:10C8A0004105510509F015988DE490E06F964EAD65
:10C8B0005FAD6F97489FF001499FF00D589FF00DB5
:10C8C0001124EB5CF64F648075808680978061143C
:10C8D00071048104910409F046988DE490E06F960C
:10C8E0006EAD7FAD6F97689FF001699FF00D789FE7
:10C8F000F00D1124EB5CF64FA084B184C284D38484
:10C90000A114B104C104D10409F043988DE490E06E
:10C910006F96AEADBFAD6F97A89FF001A99FF00DC8
:10C92000B89FF00D1124EB5CF64F84859585A685A4
:10C93000B7850097A105B10551F040982090F908FE
:10C940003090FA084090FB085090FC0808C02090F6
:10C950001109309012094090130950901409CD56D6
:10C96000DF4F6881C359D040CC56DF4F7881C4591E
:10C97000D040CB56DF4F8881C559D040CA56DF4FD3
:10C980009881C659D040A20191010E94D4D587FD5B
:10C9900016C0CD56DF4F8881C359D040CC56DF4FEB
:10C9A0009881C459D040CB56DF4FA881C559D0409B
:10C9B000CA56DF4FB881C659D0401C012D01699677
:10C9C0006CAD7DAD8EAD9FAD69970E9476D6AF966A
:10C9D0002CAD3DAD4EAD5FADAF970E94DBD5EA9675
:10C9E0006FAFEA97EB967FAFEB97EC968FAFEC9734
:10C9F000ED969FAFED97AC01CB01DA0189839A8365
:10CA0000AB83BC8361966CAD7DAD8EAD9FAD619700
:10CA10000E9476D6AB962CAD3DAD4EAD5FADAB97DB
:10CA20000E94DBD5E6966FAFE697E7967FAFE79774
:10CA3000E8968FAFE897E9969FAFE997AC01CB01F5
:10CA4000DA018D839E83AF83B88729966CAD7DAD67
:10CA50008EAD9FAD29970E9476D6A7962CAD3DADA1
:10CA60004EAD5FADA7970E94DBD5E2966FAFE29720
:10CA7000E3967FAFE397E4968FAFE497E5969FAF99
:10CA8000E597AC01CB01DA0189879A87AB87BC8730
:10CA90006DA17EA18FA198A50E9476D6A3962CADFC
:10CAA0003DAD4EAD5FADA3970E94DBD57B018C0100
:10CAB000E196AEADBFADE197EC91F0E0EE0FFF1F58
:10CAC000E25BFC4F60817181882777FD8095982F0C
:10CAD0000E9476D69B01AC01C801B7010E94A9D87B
:10CAE00020E030E048EC52E40E94DBD59B01AC0131
:10CAF0006D877E878F87988B25966CAD7DAD8EADCB
:10CB00009FAD259766307105810591051CF576E08E
:10CB10006716710481049104ECF486E0A816B10450
:10CB2000C104D104BCF48DE490E06F96AEADBFAD0E
:10CB30006F97A89FF001A99FF00DB89FF00D1124E9
:10CB4000EB5CF64FDA01C901BF7786A797A7A0ABC8
:10CB5000B1AB55C0EA962FADEA97EB963FADEB9798
:10CB6000EC964FADEC97ED965FADED97B901CA012C
:10CB70000E9454D93B014C01E6962FADE697E7960B
:10CB80003FADE797E8964FADE897E9965FADE99737
:10CB9000B901CA010E9454D95B016C01E2962FAD24
:10CBA000E297E3963FADE397E4964FADE497E596C1
:10CBB0005FADE597B901CA010E9454D97B018C0190
:10CBC000C401B301A60195010E94FBD4A8019701FD
:10CBD0000E94FBD40E9416D92DE430E06F964EAD32
:10CBE0005FAD6F97429FF001439FF00D529FF00D94
:10CBF0001124EB5CF64F66A777A780AB91AB8DE471
:10CC000090E06F966EAD7FAD6F97689FF001699F62
:10CC1000F00D789FF00D1124EB5CF64F86A597A5DB
:10CC2000A0A9B1A921968CAF9DAFAEAFBFAF2197A0
:10CC300060E070E080E89FE321962CAD3DAD4EAD05
:10CC40005FAD21970E94DBD59B01AC01C201B10110
:10CC50000E94A9D82B013C018091050E9091060EEF
:10CC6000A82FB0E05096A91BB109AF70B070BAA759
:10CC7000A9A7A230B1050CF451C05D01CC24B7FCCA
:10CC8000C094DC2CC601B5010E9476D620E030E0CD
:10CC900040E051E40E94D4D588230CF03FC060E00E
:10CCA00074E284E799E4A30192010E94DBD50E941B
:10CCB00079D87B018C016091C1087091C208809184
:10CCC000C3089091C408E616F7060807190730F55F
:10CCD0006E197F09800B910B660F771F881F991FB4
:10CCE000A60195010E94A2DCCA01B9010E9474D676
:10CCF0000E9479D89B01AC012E0D3F1D401F511F92
:10CD0000CA01B9010E9474D69B01AC0160E074E2D3
:10CD100084E799E40E94DBD52B013C018DE490E08F
:10CD20006F96EEADFFAD6F97E89F8001E99F100D04
:10CD3000F89F100D11240B5C164F21966CAD7DAD44
:10CD40008EAD9FAD2197A30192010E94A9D8D80171
:10CD500092966D937D938D939C93959750966D913C
:10CD60007D918D919C9153970E9474D6A30192015D
:10CD70000E94A9D80E94C1D50E9448D6F80160AF90
:10CD800071AF82AF93AFC357DF4F1882CD58D040F9
:10CD9000C257DF4F1882CE58D04020E8222E9FE3A2
:10CDA000392E88249924E1E0F0E0EC0FFD1FE80D16
:10CDB000F91DC301B20120813181428153810E945A
:10CDC000A9D8E1E1F0E0EC0FFD1FE80DF91D60834B
:10CDD0007183828393835B016C01E894D7F8F4013B
:10CDE000EB53F74FE080F18002811381C601B5015A
:10CDF000A80197010E94D7D71816CCF4C801B70133
:10CE0000A60195010E94DBD56B017C01C357DF4F62
:10CE10006881CD58D040C257DF4F7881CE58D0407E
:10CE2000C101A70196010E94D4D588236CF4C35791
:10CE3000DF4F8881CD58D040C257DF4F9881CE5800
:10CE4000D040D1016C017D0124E030E0820E931EC0
:10CE500030E18316910471F0D701C601C357DF4F4B
:10CE6000C882CD58D040C257DF4F9883CE58D040AB
:10CE70001D0199CFC701B60120E030E040E85FE333
:10CE80000E94D4D588230CF04CC08E010F5E1F4F3A
:10CE900081E2A82EB12CAC0EBD1ED8016D917D9102
:10CEA0008D919C91A70196010E94A9D8F8016193E8
:10CEB0007193819391938F01EA15FB0571F78DE4CE
:10CEC00090E06F962EAD3FAD6F97289F8001299F10
:10CED000100D389F100D11240B5C164FD80192963F
:10CEE0006D917D918D919C919597A70196010E94DE
:10CEF000A9D8F80162A373A384A395A360AD71AD13
:10CF000082AD93AD0E9474D6A70196010E94A9D864
:10CF10000E9448D6D801D8966D937D938D939C93AB
:10CF2000DB978DE490E06F96EEADFFAD6F97E89FD5
:10CF30008001E99F100DF89F100D11240B5C164F16
:10CF4000D80150966D917D918D919C9153970E943F
:10CF500074D6F80126A537A540A951A90E94DBD5B2
:10CF60001B012C01F80180819181A281B38100977E
:10CF7000A105B10549F584819581A681B781009706
:10CF8000A105B10509F580859185A285B385009736
:10CF9000A105B105C9F4C201B10120910109309187
:10CFA000020940910309509104090E94A9D80E94E6
:10CFB000C1D50C5B1F4F0E9448D6D8016D937D935D
:10CFC0008D939C93139771C1C201B1012091FD080B
:10CFD0003091FE084091FF08509100090E94A9D8A5
:10CFE0000E94C1D50E9448D62DE430E06F96EEAD88
:10CFF000FFAD6F97E29F6001E39FD00CF29FD00CD2
:10D00000112425E339E0C20ED31E14E4612E712CE5
:10D010006C0C7D1CD3016D937D938D939C93139722
:10D020008090150990901609A0901709B0901809E2
:10D030000E9474D67B018C01F6016081718182812E
:10D0400093810E9476D69B01AC01C801B7010E9472
:10D05000A9D87B018C01D60150966D917D918D915F
:10D060009C9153970E9474D69B01AC01C801B701F3
:10D070000E94DBD57B018C01C501B4010E9474D6EE
:10D080009B01AC01C801B7010E94D7D718162CF438
:10D09000F30180829182A282B382809019099090DC
:10D0A0001A09A0901B09B0901C098DE490E06F96BE
:10D0B0002EAD3FAD6F97289F6001299FD00C389F00
:10D0C000D00C112445E359E0C40ED51EB4E46B2EF8
:10D0D000712C6C0C7D1CD3016D917D918D919C9177
:10D0E0000E9474D67B018C01F60164817581868172
:10D0F00097810E9476D69B01AC01C801B7010E94BE
:10D10000A9D87B018C01D60150966D917D918D91AE
:10D110009C9153970E9474D69B01AC01C801B70142
:10D120000E94DBD57B018C01C501B4010E9474D63D
:10D130009B01AC01C801B7010E94D7D718162CF487
:10D14000F30180829182A282B38280902109909023
:10D150002209A0902309B09024098DE490E06F96F5
:10D160002EAD3FAD6F97289F6001299FD00C389F4F
:10D17000D00C112445E359E0C40ED51EA4E46A2E58
:10D18000712C6C0C7D1CD3016D917D918D919C91C6
:10D190000E9474D67B018C01F601648575858685B5
:10D1A00097850E9476D69B01AC01C801B7010E9409
:10D1B000A9D87B018C01D60150966D917D918D91FE
:10D1C0009C9153970E9474D69B01AC01C801B70192
:10D1D0000E94DBD57B018C01C501B4010E9474D68D
:10D1E0009B01AC01C801B7010E94D7D718162CF4D7
:10D1F000F30180829182A282B38280901D09909077
:10D200001E09A0901F09B09020098DE490E06F9650
:10D210002EAD3FAD6F97289F6001299FD00C389F9E
:10D22000D00C112445E359E0C40ED51EF4E46F2E52
:10D23000712C6C0C7D1CD3016D917D918D919C9115
:10D240000E9474D67B018C01F60160857185828510
:10D2500093850E9476D69B01AC01C801B7010E945C
:10D26000A9D87B018C01D60150966D917D918D914D
:10D270009C9153970E9474D69B01AC01C801B701E1
:10D280000E94DBD57B018C01C501B4010E9474D6DC
:10D290009B01AC01C801B7010E94D7D718162CF426
:10D2A000F30180829182A282B3828DE490E06F9636
:10D2B0002EAD3FAD6F97289F6001299FD00C389FFE
:10D2C000D00C112445E359E0C40ED51EF601EC5BE9
:10D2D000FF4F60817181828193810E9474D67B01AE
:10D2E0008C01A20191010E94DBD5D601D2966D93EB
:10D2F0007D938D939C93D597C801B7012DEB37E3B0
:10D3000046E051E40E94A9D80E9443D6F601648FFA
:10D31000758F868F978F60900509709006098090B1
:10D32000070990900809C401B30120E030E040E013
:10D330005FE30E94A9D85B016C01298D3A8D4B8D6A
:10D340005C8D29AF3AAF4BAF5CAF4091090950916A
:10D350000A0960910B0970910C094DAB5EAB6FAB84
:10D3600078AFCB01BA0120E030E040E05FE30E94FB
:10D37000A9D87B018C0169AD7AAD8BAD9CAD9F774F
:10D38000A80197010E94D7D7181644F4C601B50129
:10D39000A80197010E94D4D5882314F48601750151
:10D3A0006D8D7E8D8F8D98A169AB7AAB8BAB9CAB6D
:10D3B00080910D0990910E09A0910F09B09110096B
:10D3C0008DA79EA7AFA7B8ABBC01CD0120E030E090
:10D3D00040E05FE30E94A9D81B012C0169A97AA94A
:10D3E0008BA99CA99F77A20191010E94D7D71816FB
:10D3F00044F4C801B701A20191010E94D4D5882349
:10D4000014F4170128018DE490E06F96AEADBFAD26
:10D410006F97A89FF001A99FF00DB89FF00D112400
:10D42000EB5CF64F22A133A144A155A129A33AA355
:10D430004BA35CA3C201B1010E94D4D587FD04C0F7
:10D4400029A03AA04BA05CA049A55AA5423051059D
:10D450000CF401C15091070EC157DF4F5883CF58CC
:10D46000D0406091080EC057DF4F6883C059D0404C
:10D470007091090ECF56DF4F7883C159D04080910B
:10D480000A0ECE56DF4F8883C259D040652FC05751
:10D49000DF4F7881C059D040CF56DF4F8881C159C6
:10D4A000D040CE56DF4F9881C259D04027E137EBAC
:10D4B00041ED58E30E94D7D718160CF0CCC069890B
:10D4C0007A898B899C8920910B0E30910C0E4091AA
:10D4D0000D0E50910E0E0E94FAD40E9454D97B0179
:10D4E0008C016D897E898F89988D20910F0E3091E6
:10D4F000100E4091110E5091120E0E94FAD40E940B
:10D5000054D99B01AC01C801B7010E94FBD40E9411
:10D5100016D97B018C01A40193010E94D7D718165C
:10D520005CF00F2EF0E06F2EF0E07F2EF0E88F2EF3
:10D53000FFE39F2EF02D08C0C401B301A80197019D
:10D540000E94DBD53B014C0169AD7AAD8BAD9CAD42
:10D550002091130E3091140E4091150E5091160E1D
:10D560000E94FAD47B018C01E89417F9C801B70135
:10D570002DA93EA94FA958AD0E94D7D7181694F4EB
:10D580006DA97EA98FA998ADA80197010E94DBD54E
:10D590005B016C01C401B301A60195010E94D4D5C1
:10D5A000882314F46401530169A97AA98BA99CA961
:10D5B0002091170E3091180E4091190E50911A0EAD
:10D5C0000E94FAD47B018C01E89417F9C801B701D5
:10D5D0002DA53EA54FA558A90E94D7D7181694F49B
:10D5E0006DA57EA58FA598A9A80197010E94DBD5FE
:10D5F0007B018C01C601B501A80197010E94D4D519
:10D60000882314F48601750169A17AA18BA19CA1DC
:10D61000A80197010E94A9D87B018C01C157DF4F57
:10D620006881CF58D040C057DF4F7881C059D04073
:10D63000CF56DF4F8881C159D040CE56DF4F9881F9
:10D64000C259D040A80197010E94D4D587FD19C0C6
:10D65000D801C70102C0D201C101C157DF4F888381
:10D66000CF58D040C057DF4F9883C059D040CF56D5
:10D67000DF4FA883C159D040CE56DF4FB883C2597F
:10D68000D0408DE490E06F96AEADBFAD6F97A89F90
:10D690008001A99F100DB89F100D11240B5C164F2F
:10D6A000C157DF4F8881CF58D040C057DF4F988196
:10D6B000C059D040CF56DF4FA881C159D040CE5677
:10D6C000DF4FB881C259D040F80182A793A7A4A721
:10D6D000B5A762A973A984A995A9905820E030E064
:10D6E00040E050EC0E94A9D8D8019E962D913D9122
:10D6F0004D915C91D1970E94A9D82BE037ED43E280
:10D700005BE30E94FBD40E9416D9F62EE72ED82E9A
:10D71000C92EC157DF4F6881CF58D040C057DF4F67
:10D720007881C059D040CF56DF4F8881C159D04051
:10D73000CE56DF4F9881C259D0402F2D3E2D4D2D12
:10D740005C2D0E94D4D587FD14C0C157DF4FF882ED
:10D75000CF58D040C057DF4FE882C059D040CF5695
:10D76000DF4FD882C159D040CE56DF4FC882C25950
:10D77000D0408DE490E06F96EEADFFAD6F97E89FDF
:10D780008001E99F100DF89F100D11240B5C164FBE
:10D79000C157DF4F8881CF58D040C057DF4F9881A5
:10D7A000C059D040CF56DF4FA881C159D040CE5686
:10D7B000DF4FB881C259D040F80186A397A3A0A734
:10D7C000B1A762A173A184A195A12F2D3E2D4D2D4E
:10D7D0005C2D0E94D4D518162CF081E0D801D79684
:10D7E0008C9302C0F80117AA8DE490E06F962EADDD
:10D7F0003FAD6F97289FF001299FF00D389FF00DE6
:10D800001124EB5CF64F81E086ABABE0BEE0FE019D
:10D81000719680E101900D928150E1F78DE490E0E6
:10D820006F964EAD5FAD6F97489F6001499FD00CDA
:10D83000589FD00C112465E379E0C60ED71ED6019F
:10D840009296ED90FD900D911C919597E092070EA8
:10D85000F092080E0093090E10930A0E96966D91A1
:10D860007D918D919C919997A80197010E94DBD59C
:10D870004B015C01C201B101A80197010E94DBD5F7
:10D880008B019C01C601B501A4010E94CB5DBBA523
:10D89000B093050EC757DF4F288139814A815B81DC
:10D8A000C958D0402093310930933209409333094D
:10D8B00050933409CB57DF4F488159816A817B816E
:10D8C000C558D04040932D0950932E0960932F09DD
:10D8D00070933009CF57DF4F688179818A819B81AE
:10D8E000C158D0406093290970932A0980932B096D
:10D8F00090932C09C358DF4F88819981AA81BB81FD
:10D90000CD57D0408093250990932609A0932709ED
:10D91000B09328090E944D600E94D67DCA56DF4F01
:10D920000FB6F894DEBF0FBECDBFCF91DF911F9130
:10D930000F91FF90EF90DF90CF90BF90AF909F90AE
:10D940008F907F906F905F904F903F902F900895B1
:10D95000FF920F931F93CF93DF938B010E944A1A7C
:10D96000EB01FF24FA9409C00E944A1A6C1B7D0B3C
:10D970006017710710F080E008C0FEBC0DB407FE10
:10D98000FDCF8EB58F3F81F781E0DF91CF911F9161
:10D990000F91FF900895FC014281242F30E0C901CE
:10D9A0009595879580658CBD40FF02C080E004C0DE
:10D9B00080E0463009F081E08DBD808160E00C940C
:10D9C0004B1CDF92EF92FF920F931F93CF93DF9345
:10D9D000EC01D62E79018A01DEDFCE016CE271E026
:10D9E000B7DF8D2D80648EBD0DB407FEFDCF28E11D
:10D9F00030E0D801C701022E04C0B695A7959795CF
:10DA000087950A94D2F78EBD0DB407FEFDCF28503E
:10DA100030408FEF283F380761F7DD2011F485E9AA
:10DA200006C088E0D81611F487E801C08FEF8EBDDC
:10DA30000DB407FEFDCF8CE0D81631F48FEF8EBD0C
:10DA40000DB407FEFDCF8EB59FEF2FEF2EBD0DB4A9
:10DA500007FEFDCF8EB587FF04C0992311F09150CA
:10DA6000F5CF8B83DF91CF911F910F91FF90EF90B6
:10DA7000DF900895FC01808161E00C944B1CDC0177
:10DA80006EBDFA0120E030E00DB407FEFDCF8081CD
:10DA90008EBD0DB407FEFDCF81818EBD2E5F3F4F41
:10DAA000329682E02030380779F70DB407FEFDCFBB
:10DAB0008FEF8EBD0DB407FEFDCF8FEF8EBD0DB481
:10DAC00007FEFDCF8FEF8EBD0DB407FEFDCF8EB5E7
:10DAD00013968C9313978F71853011F481E008951C
:10DAE00083E111968C931197CD01C4DF80E00895F6
:10DAF000CF92DF92EF92FF920F931F93CF93DF931A
:10DB0000EC017A018B0169018C81833039F059E095
:10DB1000EE0CFF1C001F111F5A95D1F7CE0168E1D2
:10DB2000A80197014EDF882311F086E020C0CE01C6
:10DB30006EEFA601A4DF8823D9F0CE0168E572E07C
:10DB400007DF882311F487E112C0CE016DE020E0E9
:10DB500030E040E050E035DF882341F48FEF8EBDA8
:10DB60000DB407FEFDCF8EB5882371F086E1898361
:10DB7000CE0180DF80E0DF91CF911F910F91FF9068
:10DB8000EF90DF90CF900895CE0174DF81E0F3CF66
:10DB9000BF92CF92DF92EF92FF920F931F93CF939A
:10DBA000DF93EC016B018A010E944A1A7B01BB24BE
:10DBB000BA9409C00E944A1A6E197F096D527140C9
:10DBC00010F081E15FC0BEBC0DB407FEFDCF8EB585
:10DBD0008B838F3F79F38E3F11F08FE053C0D801D4
:10DBE000119701151105D9F08FEF8EBD20E030E0BF
:10DBF0009FEF0BC00DB407FEFDCF8EB5F601E20F0F
:10DC0000F31F80839EBD2F5F3F4F2A173B0790F382
:10DC10000DB407FEFDCF8EB5AC0DBD1D8C9340E05D
:10DC200050E060E070E016C0272F3327F601E40FC4
:10DC3000F51F808190E028273927220F331F2F52AC
:10DC4000354FF90185919491762F662768277927BA
:10DC50004F5F5F4F4017510738F38FEF8EBD0DB404
:10DC600007FEFDCF3EB58FEF8EBD0DB407FEFDCF95
:10DC70002EB5932F80E030E0822B932B6817790725
:10DC800031F080E28983CE01F5DE80E003C0CE0171
:10DC9000F1DE81E0DF91CF911F910F91FF90EF9026
:10DCA000DF90CF90BF900895AF92BF92CF92DF9256
:10DCB000EF92FF920F931F93CF93DF93EC017A01C2
:10DCC0008B0159018C81833039F029E0EE0CFF1C67
:10DCD000001F111F2A95D1F793E0D92E84E0C82E9A
:10DCE000DA94CE0161E1A80197016BDE882311F07F
:10DCF000C98209C0CE01B50140E052E049DF882366
:10DD000011F081E010C0DD2059F0CE01B3DECE016C
:10DD10006CE020E030E040E050E053DE1982E0CFDC
:10DD2000CE01A8DE80E0DF91CF911F910F91FF908F
:10DD3000EF90DF90CF90BF90AF900895BF92CF92B9
:10DD4000DF92EF92FF920F931F93CF93DF93EC013B
:10DD5000B62E1C82198248830E944A1A6B01888160
:10DD600061E00E94981BCE0185DE82E360E00E94A4
:10DD7000981B83E361E00E94981B84E361E00E94AA
:10DD8000981B85E361E00E94981B85E361E00E9497
:10DD90004B1C85E08A8382E58CBD1DBC80E09FEF33
:10DDA0009EBD0DB407FEFDCF8F5F8A30C9F709C055
:10DDB0000E944A1A6C197D09615D774010F081E07C
:10DDC00059C0CE0160E020E030E040E050E0F9DDF5
:10DDD000182F8B83813061F7CE0168E02AEA31E0A9
:10DDE00040E050E0EEDD82FF02C01C8311C080E005
:10DDF0002FEF2EBD0DB407FEFDCF9EB58F5F843093
:10DE0000C1F79B839A3A11F082E034C082E08C83A0
:10DE10008C81823021F0EE24FF2487010FC0E12C99
:10DE2000F12C012D50E4152F09C00E944A1A6C19DB
:10DE30007D09615D774010F08AE01CC0CE0167E388
:10DE400020E030E040E050E0BCDDCE0169E2A80116
:10DE50009701B7DD8B83882341F78C81823019F5D8
:10DE6000CE016AE320E030E040E050E0AADD882304
:10DE700029F088E08983CE01FDDD20C08FEF8EBDC3
:10DE80000DB407FEFDCF8EB5807C803C11F483E09D
:10DE90008C8380E09FEF9EBD0DB407FEFDCF2EB5B5
:10DEA0008F5F8330C1F7CE01E5DD86E08B1518F476
:10DEB00088E1898303C0BA8281E001C080E0DF91FC
:10DEC000CF911F910F91FF90EF90DF90CF90BF9077
:10DED0000895CF93DF93DC01EB01BA0180E090E07D
:10DEE00020E2FE01E80FF91F208301968B30910597
:10DEF000C1F757E040E022C02E3219F081ED9CE0DE
:10DF000007C05A3049F15AE048E017C0321721F1F2
:10DF1000FC01019634913323C9F75417E8F02132FC
:10DF2000D8F02F37C8F4822F81568A3108F4205256
:10DF3000FE01E40FF11D20834F5F11962C912223E7
:10DF400011F02F32C9F6FB01B183A08390E08881E4
:10DF5000803219F091E001C090E0892FDF91CF91DC
:10DF600008956F927F928F929F92AF92BF92CF92BD
:10DF7000DF92EF92FF920F931F93CF93DF93EC0109
:10DF80007A018B012B81222309F480C089899A8927
:10DF9000AB89BC8984179507A607B70708F476C034
:10DFA00085C0E114F1040105110551F41C821D82A4
:10DFB0001E821F82188619861A861B8681E067C01A
:10DFC000288539854A855B85E98DFA8D858590E0C0
:10DFD0000996215030404040504039014A01082EF6
:10DFE00004C096948794779467940A94D2F72F5F2D
:10DFF0003F4F4F4F5F4F0894E108F10801091109A5
:10E000005701680104C0D694C794B794A7948A9521
:10E01000D2F70894E11CF11C011D111DA614B704D0
:10E02000C804D90428F0211531054105510549F4EA
:10E030008D899E89AF89B88D8C839D83AE83BF8384
:10E0400016C0A618B708C808D90811C04C815D8150
:10E050006E817F81898D9A8D94010E94857B0894C1
:10E06000A108B108C108D108882331F40FC084E0A9
:10E07000882E912C8C0E9D1EA114B104C104D104D4
:10E0800029F7E886F9860A871B8798CF80E0DF9119
:10E09000CF911F910F91FF90EF90DF90CF90BF90A5
:10E0A000AF909F908F907F906F900895223009F0ED
:10E0B00078CFE7CFCF93DF93EC018C859D85AE853C
:10E0C000BF8540E0611141E0BC01CD010E94537960
:10E0D000882319F420E030E00AC08889282F30E036
:10E0E00095E0220F331F9A95E1F72B5D314FC9015F
:10E0F000DF91CF9108950F931F93CF93DF938C01FE
:10E10000FC0183818823E9F1818187FF37C0C80141
:10E1100061E0D0DFEC010097A1F18881853E89F1B3
:10E12000F8018381823040F481899289A389B4897E
:10E130008C8F9D8FAE8FBF8FF801858996899B8FBD
:10E140008A8F85899689A789B08DCD01AA27BB279B
:10E150009D8B8C8BE0911F0EF091200E309751F02B
:10E16000BE016A5E7F4FCE0148961995888D998DC4
:10E170009B8B8A8BF80181818F7781830E9418792C
:10E1800004C081E0F801808380E0DF91CF911F918E
:10E190000F9108950F931F938C01ADDFF801138247
:10E1A0001F910F910895FC018381882311F0CF0105
:10E1B000F1CF08956F927F928F929F92AF92BF920C
:10E1C000CF92DF92EF92FF920F931F93DF93CF9343
:10E1D00000D00F92CDB7DEB77C015A016B01DC0194
:10E1E00013968C911397813009F08EC011968C9103
:10E1F00081FF8AC09DC00097A105B10511F481E09F
:10E2000084C0F7016084718482849384C701B6015D
:10E21000A501A7DE882309F477C0D70159968D910F
:10E220009C915A97A114B104C104D10489F4559664
:10E230004D915D916D917C9158970E94FA7B882356
:10E2400009F462C0F701158A168A178A108E44C035
:10E25000D70114964D915D916D917C9117979E0118
:10E260002F5F3F4F0E94857B882309F44DC0D70163
:10E270005996ED91FC915A9749815A816B817C8125
:10E280008789803149F4483FBFEF5B07B0E06B07F7
:10E29000B0E07B0748F020C0483F8FEF58078FEF72
:10E2A00068078FE07807C0F4CF010E94FA7B8823CB
:10E2B00059F1D70114964D915D916D917C9117970D
:10E2C00059968D919C915A970FEF1FEF2FEF3FE0DA
:10E2D0000E94FF7A8823C1F0F701A18AB28AC38A1B
:10E2E000D48A818180688183C70105DF882361F03A
:10E2F000B601A5016A147B048C049D0410F4B401DA
:10E30000A301C7012EDE01C080E00F900F900F9097
:10E310000F90CF91DF911F910F91FF90EF90DF90C1
:10E32000CF90BF90AF909F908F907F906F90089507
:10E33000F70181899289A389B48984179507A60773
:10E34000B70708F058CFE0CFCF93DF93EC0140E060
:10E3500050E060E070E02EDF882359F0CE0161E0EC
:10E36000A9DEFC01009729F085EE80831B8260D72F
:10E3700001C080E0DF91CF9108952F923F924F929C
:10E380005F926F927F928F929F92AF92BF92CF9245
:10E39000DF92EF92FF920F931F93CF93DF93EC01E5
:10E3A0002A018B81882309F4B5C0898180FFB2C01E
:10E3B000C7C025014E185F083B0174E0272E312CA1
:10E3C0002C0E3D1E4201A0C0288539854A855B85FB
:10E3D0006FEFA62E61E0B62EA222B3228B817901C7
:10E3E0008A0199E016950795F794E7949A95D1F7E5
:10E3F000E98DFA8D823049F4428D538D648D758D8F
:10E400004E0D5F1D601F711F3FC0D480DA94DE2067
:10E41000A114B104D9F4DD20C9F421153105410559
:10E42000510549F48D899E89AF89B88D8C839D8370
:10E43000AE83BF830BC04C815D816E817F81CF0134
:10E4400091010E94857B882309F464C0E98DFA8DCF
:10E450004C815D816E817F814250504060407040B0
:10E46000058404C0440F551F661F771F0A94D2F716
:10E4700086859785A089B189480F591F6A1F7B1F20
:10E480004D0D511D611D711D80E092E08A199B099F
:10E4900084018815990508F48C0182E00030180782
:10E4A00009F066C08091210E9091220EA091230E5A
:10E4B000B091240E481759076A077B0709F458C022
:10E4C00080912510909126109301EEDB882349F46A
:10E4D00021C095012B5D314FC301B901A8010E94F4
:10E4E00067D4600E711E980140E050E088859985E0
:10E4F000AA85BB85820F931FA41FB51F88879987A4
:10E50000AA87BB87801A910A8114910409F05CCF15
:10E51000A20102C04FEF5FEFCA01DF91CF911F91BF
:10E520000F91FF90EF90DF90CF90BF90AF909F90B2
:10E530008F907F906F905F904F903F902F900895B5
:10E54000A988BA88CB88DC88E884F9840A851B8589
:10E550009A0140E050E0D601C5018E199F09A00B39
:10E56000B10B281739074A075B0708F022CF24CFE1
:10E57000CB01BA0140E097D6882309F0AACFCACFD1
:10E58000CF92DF92EF92FF920F931F93CF93DF937F
:10E590007C01EB018A01FC018381823008F46EC0AA
:10E5A00080859185A285B3858F719070A070B070C1
:10E5B0000097A105B10509F061C06CC0F801108297
:10E5C000EDE0CE2ED12CC701BE0140E250E0D5DEF9
:10E5D0009C018032910521F0009709F04FC050C096
:10E5E0004881442309F44CC0453E69F34E3259F347
:10E5F0008B858F738F30E9F501151105D1F18A8D67
:10E600009B8D892BB1F5842F90E08F7190700097CE
:10E6100081F1833091056CF58C9D90018D9D300DBD
:10E620009C9D300D11242D503040F801E20FF31F56
:10E63000898180838B8181838D8182838F81838394
:10E64000898584838E858583888986838A89878363
:10E650008C8980878E898187888D82878C8D83873E
:10E660008E8D8487888186FF04C0F801E20FF31F36
:10E6700015868B8583FDA7CF822F03C08FEF01C046
:10E6800080E0DF91CF911F910F91FF90EF90DF908D
:10E69000CF9008954115510509F090CF91CFDF93A8
:10E6A000CF930F92CDB7DEB7BE016F5F7F4F41E0D2
:10E6B00050E063DE019719F02FEF3FEF03C089812F
:10E6C000282F30E0C9010F90CF91DF910895EF928C
:10E6D000FF920F931F93CF93DF93EC018B818230D6
:10E6E00030F1E884F9840A851B85CE01D8DF97FDD7
:10E6F0001EC088859985AA85BB854F96A11DB11D31
:10E7000088879987AA87BB87A5E016950795F79410
:10E71000E794AA95D1F72E2D30E02F703070F5E0F8
:10E72000220F331FFA95E1F72B5D314F02C020E035
:10E7300030E0C901DF91CF911F910F91FF90EF90D1
:10E7400008950F931F93CF93DF93EC018B018B817F
:10E75000882309F040C0FB018789803109F041C05E
:10E7600082E08B831D8A1E8A1F8A188E808D918D70
:10E77000A0E0B0E045E0880F991FAA1FBB1F4A9593
:10E78000D1F7898B9A8BAB8BBC8B13C083E08B83C7
:10E79000F801428D538D648D758D4D8B5E8B6F8B23
:10E7A000788F9E012F5E3F4FC8010E94567C8823C0
:10E7B00091F01A8F098F81E089831C821D821E824D
:10E7C0001F82188619861A861B861C861D861E8641
:10E7D0001F86188A01C080E0DF91CF911F910F91B1
:10E7E00008958032C1F7D2CF1F93CF93DF93EC010E
:10E7F000142F262F30E0F90175E0EE0FFF1F7A95F8
:10E80000E1F7EB5DF14F8385817121F0842F8271F7
:10E8100009F067C08091210E9091220EA091230EE5
:10E82000B091240E8C879D87AE87BF87688BF901D6
:10E8300065E0EE0FFF1F6A95E1F7EB5DF14F84890C
:10E840009589A0E0B0E0DC01992788278D8B9E8B0D
:10E85000AF8BB88F228D338DA90160E070E0482B1B
:10E86000592B6A2B7B2B4D8B5E8B6F8B788F83851F
:10E8700090E088719070009751F4848D958DA68DED
:10E88000B78D898B9A8BAB8BBC8B81E00CC040978A
:10E8900041F59E012F5E3F4F898D9A8D0E94567CD7
:10E8A0008823F9F084E08B83812F8F7089831C8209
:10E8B0001D821E821F82188619861A861B8614FFE7
:10E8C00016C0CE0140E050E060E070E073DC8823C9
:10E8D00071F409C049895A896B897C89CE0141DB71
:10E8E00002C01B8280E0DF91CF911F91089515FD3A
:10E8F000F1CF81E0F8CF2F923F924F925F926F92CB
:10E900007F928F929F92AF92BF92CF92DF92EF92BF
:10E91000FF920F931F93DF93CF930F92CDB7DEB784
:10E920002C015B013A01490100E010E0EE24EA9479
:10E93000FE2C1E010894211C311C11C00A0D1B1D48
:10E94000F80160838114910419F46A3039F41BC012
:10E95000C40170E00E947BD40097A9F4860168018D
:10E960000894C11CD11CC614D7043CF5C201B101E6
:10E9700041E050E002DD7C0181309105F1F46981D4
:10E980006D30E1F6ECCF8601A00EB11EF5011082CC
:10E99000C8010F90CF91DF911F910F91FF90EF90E1
:10E9A000DF90CF90BF90AF909F908F907F906F90AF
:10E9B0005F904F903F902F900895F7FEE5CF0FEFB7
:10E9C0001FEFE6CFCF93DF93EC019C012C5F3F4F0D
:10E9D000898D9A8D41E050E060E070E0D2D78823C5
:10E9E000A1F08D899E89AF89B88D0097A105B105E9
:10E9F00059F48C819D81AE81BF818D8B9E8BAF8BB5
:10EA0000B88F89818068898381E0DF91CF910895F3
:10EA10002F923F924F925F927F928F929F92AF92EE
:10EA2000BF92CF92DF92EF92FF920F931F93DF93EB
:10EA3000CF9300D000D0CDB7DEB76C01162F072FD3
:10EA40005E834D83DC0113968C911397813009F01E
:10EA500069C111968C9181FF65C182C1F60141891E
:10EA600052896389748980859185A285B3858417CD
:10EA70009507A607B70729F0C60173DA882309F4BA
:10EA800051C1812F902F9C0119014D805E800FC1D3
:10EA9000D6015996ED91FC915A97DA01C90149E0E6
:10EAA000B695A795979587954A95D1F774807A94EE
:10EAB00078228FEF882E81E0982E82229322772071
:10EAC00009F051C08114910409F04DC0D60114968B
:10EAD0004D915D916D917C9117974115510561059F
:10EAE000710581F455968D919D910D90BC91A02D4D
:10EAF0000097A105B10559F1F60184839583A6839A
:10EB0000B78331C0CF019E012F5F3F4FFED58823D1
:10EB100009F408C129813A814B815C81D60159965B
:10EB2000ED91FC915A978789803149F4283FBFEFD6
:10EB30003B07B0E04B07B0E05B0770F008C0283F30
:10EB4000EFEF3E07EFEF4E07EFE05E0728F0C6015C
:10EB500039DF882341F4E6C0D60114962D933D9306
:10EB60004D935C93179780E092E0881999095201C0
:10EB70008415950508F45C01D6015996ED91FC9138
:10EB80005A971496ED90FD900D911C9117978EEF6A
:10EB90009FEFAFEFBFEFE80EF91E0A1F1B1F0584A2
:10EBA00004C0EE0CFF1C001F111F0A94D2F78685CB
:10EBB0009785A089B189E80EF91E0A1F1B1FE70C73
:10EBC000F11C011D111D90E0A91692E0B90639F55E
:10EBD0008091210E9091220EA091230EB091240ECF
:10EBE0008E159F05A007B10771F4109227108FEFC3
:10EBF0009FEFAFEFBFEF8093210E9093220EA09373
:10EC0000230EB093240E8091251090912610B80108
:10EC1000A70191010E94786D8823A9F583C0811412
:10EC2000910411F5D60118962D913D914D915C916D
:10EC30001B9751968D919D910D90BC91A02D2817F9
:10EC400039074A075B0780F0F3D2882309F46AC0CA
:10EC500081E080932710E092210EF092220E009323
:10EC6000230E1093240E07C0C801B70141E01BD347
:10EC7000882309F457C094012B5D314FC901B101BC
:10EC8000A5010E9467D4950140E050E0F60180851F
:10EC90009185A285B385820F931FA41FB51F80871E
:10ECA0009187A287B3872A0C3B1C4A185B08D601C0
:10ECB00018962D913D914D915C911B9741145104F3
:10ECC00009F0E6CE51968D919D910D90BC91A02DAD
:10ECD00082179307A407B50748F4F601218B328BFE
:10ECE000438B548B81818068818311C080911F0E7A
:10ECF0009091200E892B59F08D819E81892B39F0BE
:10ED0000D60111968C911197806811968C93F6011B
:10ED1000818183FF04C0C601EED9882319F04D819B
:10ED20005E8105C081E0D6018C934FEF5FEFCA0191
:10ED300026960FB6F894DEBF0FBECDBFCF91DF9100
:10ED40001F910F91FF90EF90DF90CF90BF90AF9009
:10ED50009F908F907F905F904F903F902F9008955D
:10ED600082FD7CCE8ECEDF92EF92FF920F931F93A7
:10ED7000CF93DF93EC0189899A89AB89BC89805E46
:10ED80009F4FAF41B04008F06FC0CE011BDE88231B
:10ED900009F46AC04DD2882309F466C0E98DFA8D62
:10EDA000EC80FD800E811F818EEF9FEFAFEFBFEFF4
:10EDB000E80EF91E0A1F1B1F058404C0EE0CFF1C81
:10EDC000001F111F0A94D2F786859785A089B18903
:10EDD000E80EF91E0A1F1B1F81E080932710E092A6
:10EDE000210EF092220E0093230E1093240E80E049
:10EDF00092E0E5E2FEE0DF019C011D9221503040EF
:10EE0000E1F7DD24D39411C0B801A7014D0D511DC8
:10EE1000611D711D809125109091261025E23EE024
:10EE20000E94786D882301F1D394E98DFA8D848155
:10EE3000D81650F320E032E040E050E0058404C0F2
:10EE4000220F331F441F551F0A94D2F789899A89CC
:10EE5000AB89BC89820F931FA41FB51F898B9A8B26
:10EE6000AB8BBC8B81E001C080E0DF91CF911F9123
:10EE70000F91FF90EF90DF9008958F929F92AF9245
:10EE8000BF92CF92DF92EF92FF920F931F93CF9397
:10EE9000DF936C01EB01942E852EA22E898D9A8D25
:10EEA000D6015A969C938E935997CB0140E050E03F
:10EEB00060E070E056D8BB2437C0CE0108DCFC010E
:10EEC000009709F48FC055E016950795F794E794DD
:10EED0005A95D1F71E2D1F708081882311F0853E31
:10EEE000C9F4BB2099F42091210E3091220E40915B
:10EEF000230E5091240ED6011C962D933D934D93D5
:10EF00005C931F9750961C93BB24B39480818823F5
:10EF100059F418C0892D982DBF014BE050E00E9494
:10EF20005AD4009709F46CC0E884F9840A851B85DB
:10EF300089899A89AB89BC89E816F9060A071B07F3
:10EF400008F4BBCFA6FE4EC0A1FE4CC0BB2049F0CA
:10EF5000F6011089C60161E0ADD8EC01009761F4BB
:10EF600041C08B81823009F43DC0CE01FCDE882394
:10EF7000C9F110E0C5E2DEE080E2DE011D928A9573
:10EF8000E9F7DE01292D382DC901FC018BE0019044
:10EF90000D928150E1F7E0911F0EF091200E309715
:10EFA00039F0BE01625F7F4FCE014096199508C0CF
:10EFB00081E298E2998B888B80E098E09F878E872A
:10EFC000888999899B8B8A8B998F888F8E859F855D
:10EFD0009F8B8E8B2DD1882329F0C601612F4A2D5E
:10EFE00003DC01C080E0DF91CF911F910F91FF9072
:10EFF000EF90DF90CF90BF90AF909F908F9008954B
:10F00000A7FEEBCFEFCF2F923F924F925F926F927E
:10F010007F928F929F92AF92BF92CF92DF92EF92A8
:10F02000FF920F931F93DF93CF93CDB7DEB7C654F4
:10F03000D0400FB6F894DEBF0FBECDBF3C016B01D0
:10F04000DE01AE5BBF4F11965C934E9325962FAFBA
:10F0500025971C861F861FA21AA66115710509F443
:10F060007CC0FC018381882309F077C0FA0180818C
:10F070008F32F1F08601ECE0EE2EF12CEC0EFD1E4D
:10F0800072E4A72EB12CAC0EBD1E4E010894811C5B
:10F09000911C2796FFAEEEAE279767E2262E312C05
:10F0A0002C0E3D1E270123C01196B183A08301C001
:10F0B000FD01A081B1818C918F32B1F3D6011396FD
:10F0C0008C91139782508230A8F28E01095D1F4FF8
:10F0D00059966D917C915A97C80133DB882359F674
:10F0E0003CC0342D252D8701832F922F7C01F50103
:10F0F00080819181B401A5010E94696F882329F460
:10F100002CC03196D501ED93FC93D501ED91FC9186
:10F1100080818F32B1F38823B9F0C701B801A4010F
:10F1200021E0ABDE8823C9F00C151D0511F0C801E4
:10F1300031D82796EEADFFAD2797EE16FF0689F67C
:10F14000C101322D292FCFCFC301B801A4012596CB
:10F150002FAD259792DE182F01C010E0CE018796C3
:10F1600022D8CE010C961FD8812FCA5BDF4F0FB675
:10F17000F894DEBF0FBECDBFCF91DF911F910F91ED
:10F18000FF90EF90DF90CF90BF90AF909F908F90C7
:10F190007F906F905F904F903F902F9008950F93C6
:10F1A0001F93DF93CF93CDB7DEB76B970FB6F8946D
:10F1B000DEBF0FBECDBF9C01AB0119821C828E0148
:10F1C0000F5F1F4FC801B90122E01DDF882311F432
:10F1D00010E003C0C801B8D8182FCE0101960E94D4
:10F1E000D370812F6B960FB6F894DEBF0FBECDBFE4
:10F1F000CF91DF911F910F910895DB010D900020B9
:10F20000E9F71197A61BB70B0496AD0101CCDF936C
:10F21000CF930F92CDB7DEB769830496BE016F5FBF
:10F220007F4F41E050E0F4DB0F90CF91DF910895E4
:10F2300080912710882399F14091210E5091220E40
:10F240006091230E7091240E8091251090912610CC
:10F2500025E23EE00E94786D882319F14091281044
:10F260005091291060912A1070912B104115510571
:10F270006105710591F0809125109091261025E28D
:10F280003EE00E94786D882361F010922810109261
:10F29000291010922A1010922B101092271081E042
:10F2A000089580E00895DF92EF92FF920F931F93ED
:10F2B0007B018C01D42E8091210E9091220EA09181
:10F2C000230EB091240E8E159F05A007B107B9F04B
:10F2D000AFDF8823E1F08091251090912610B801CE
:10F2E000A70125E23EE00E94546E882381F0E0925F
:10F2F000210EF092220E0093230E1093240EDD2097
:10F3000011F481E011C081E0809327100DC08FEFD0
:10F310009FEFAFEFBFEF8093210E9093220EA0934B
:10F32000230EB093240E80E01F910F91FF90EF9079
:10F33000DF9008958F929F92AF92BF92CF92DF920B
:10F34000EF92FF920F931F93CF93DF936C01142FD3
:10F350007093261060932510FC01178A82E090E0DC
:10F36000A0E0B0E080839183A283B3831092271042
:10F37000109228101092291010922A1010922B101F
:10F380008FEF9FEFAFEFBFEF8093210E9093220E90
:10F39000A093230EB093240E442321F488249924AF
:10F3A00054013FC0453008F01CC160E070E080E0CF
:10F3B00090E040E078DF882309F413C1C12FD0E04A
:10F3C0002197FE0174E0EE0FFF1F7A95E1F7EB5DE8
:10F3D000F14FE254FE4F8081EE5BF14090E08F7779
:10F3E0009070892B09F0FDC0E653FE4F808191811A
:10F3F000A281B38184369105A105B10508F4F1C05D
:10F4000064E0CC0FDD1F6A95E1F7C551D04F8880CD
:10F410009980AA80BB8081149104A104B10409F4ED
:10F42000E0C0C501B40140E03EDF882309F4D9C043
:10F430008091300E9091310E8050924009F0D1C0F1
:10F440002091350E222309F4CCC08091330E909187
:10F45000340E892B09F4C5C08091320E882309F43B
:10F46000C0C0F601228B8091320E8483158661E044
:10F4700070E007C04F5FF60145874150483008F003
:10F48000B0C0F6014585848190E09B01042E02C046
:10F49000220F331F0A94E2F78217930759F720913E
:10F4A0003B0E30913C0E2115310519F040E050E043
:10F4B00008C02091490E30914A0E40914B0E509158
:10F4C0004C0EF6012583368347835087E090330E38
:10F4D000F090340E00E010E0E80CF91C0A1D1B1D32
:10F4E000E38AF48A058B168B8091360E9091370E45
:10F4F000918F808F6091350E70E080E090E00E94E7
:10F5000050DC6E0D7F1D801F911FF601628F738F7F
:10F51000848F958F2091360E3091370E55E0220F53
:10F52000331F5A95E1F721503E4F232F332726955D
:10F5300040E050E0260F371F481F591F26873787A6
:10F54000408B518B8091380E9091390E009719F0B5
:10F55000A0E0B0E008C08091450E9091460EA091C9
:10F56000470EB091480E85017401E21AF30A040BAC
:10F57000150BA8019701280F391F4A1F5B1FF601C1
:10F58000058404C056954795379527950A94D2F778
:10F590002187328743875487253FFFE03F07F0E00C
:10F5A0004F07F0E05F0720F48CE0F601878B19C06D
:10F5B000255F3F4F4040504018F480E1F6010EC0F7
:10F5C0008091510E9091520EA091530EB091540E15
:10F5D000F601828F938FA48FB58F80E2878B81E0B5
:10F5E00001C080E0DF91CF911F910F91FF90EF90CC
:10F5F000DF90CF90BF90AF909F908F9008956F92C3
:10F600007F928F929F92AF92BF92CF92DF92EF92B2
:10F61000FF920F931F93CF93DF93EC015A016B017D
:10F6200038014901423051056105710508F45DC09A
:10F6300089859A85AB85BC850196A11DB11D84176E
:10F640009507A607B70708F450C08F89803129F4C1
:10F65000E52EF62E072F11270CC0803209F045C089
:10F660007A018B0187E016950795F794E7948A95C0
:10F67000D1F78B899C89AD89BE89E80EF91E0A1FD6
:10F680001B1FC801B70141E00EDE882371F18F898D
:10F69000803149F4F501F070EE0FFF1FEB5DF14F83
:10F6A000718260820DC0F501EF77F070EE0FFF1FE1
:10F6B000EE0FFF1FEB5DF14F6082718282829382B9
:10F6C0008A89823080F08D819E81AF81B885E80E75
:10F6D000F91E0A1F1B1FE0922810F09229100093B8
:10F6E0002A1010932B1081E001C080E0DF91CF91B0
:10F6F0001F910F91FF90EF90DF90CF90BF90AF9050
:10F700009F908F907F906F900895CF92DF92EF92AD
:10F71000FF920F931F93CF93DF93EC017A018B013C
:10F72000690189859A85AB85BC850196A11DB11DAE
:10F7300084179507A607B70708F452C08F89803150
:10F7400029F45527412F302F2F2D0CC0803209F07E
:10F7500047C09A01AB0167E05695479537952795C5
:10F760006A95D1F78B899C89AD89BE89280F391F8D
:10F770004A1F5B1F8091210E9091220EA091230EB3
:10F78000B091240E281739074A075B0731F0CA01E8
:10F79000B90140E088DD882319F18F89803159F45F
:10F7A000F701F070EE0FFF1FEB5DF14F808191814B
:10F7B000A0E0B0E00EC0F701EF77F070EE0FFF1F92
:10F7C000EE0FFF1FEB5DF14F80819181A281B3812C
:10F7D000BF70F60180839183A283B38381E001C06F
:10F7E00080E0DF91CF911F910F91FF90EF90DF901C
:10F7F000CF900895AF92BF92CF92DF92EF92FF9297
:10F800000F931F93DF93CF9300D00F92CDB7DEB746
:10F810006C017A018B0182E090E0A0E0B0E0F6019B
:10F8200080839183A283B3835E010894A11CB11CE1
:10F83000C601B801A701950168DF882339F1C60127
:10F84000B801A70100E010E020E030E0D8DE882316
:10F85000E9F0E980FA800B811C81F601878980310B
:10F8600051F4F8EFEF16FFEFFF06F0E00F07F0E0BE
:10F870001F07F0F209C088EFE8168FEFF8068FEF48
:10F8800008078FE01807A0F281E001C080E00F9028
:10F890000F900F900F90CF91DF911F910F91FF90DC
:10F8A000EF90DF90CF90BF90AF9008954F925F920E
:10F8B0006F927F928F929F92AF92BF92CF92DF9280
:10F8C000EF92FF920F931F93DF93CF9300D00F928D
:10F8D000CDB7DEB76C0149835A836B837C833901D2
:10F8E000EE24FF2487012E010894411C511C812C19
:10F8F000E2E09E2EA12CB12C49815A816B817C8142
:10F90000C601920102DF882339F1D501C401F60155
:10F91000058404C0880F991FAA1FBB1F0A94D2F741
:10F92000E80EF91E0A1F1B1F29813A814B815C8159
:10F930008789803131F4285F3F4F40405040E0F2EA
:10F9400005C0285F3F4F4F4F5F40B0F2F301E082A8
:10F95000F1820283138381E00F900F900F900F903C
:10F96000CF91DF911F910F91FF90EF90DF90CF909B
:10F97000BF90AF909F908F907F906F905F904F90CF
:10F9800008952F923F924F925F926F927F928F9243
:10F990009F92AF92BF92CF92DF92EF92FF920F931E
:10F9A0001F93DF93CF93CDB7DEB72F970FB6F894A1
:10F9B000DEBF0FBECDBF1C014A875B876C877D878A
:10F9C0003F872E87DC0119968D919D910D90BC91FA
:10F9D000A02D0196A11DB11D8E839F83A887B98795
:10F9E000F901008111812281338101151105210561
:10F9F000310549F0480159010894811C911CA11C52
:10FA0000B11C1D8210C0D1018D909D90AD90BC9015
:10FA10001D828A859B85AC85BD850197A105B105B1
:10FA200011F491E09D837501640144245524320151
:10FA30008E010F5F1F4FF10181859285A385B485EB
:10FA4000481659066A067B0608F08CC08E819F8195
:10FA5000A885B9858C159D05AE05BF0550F4A2E0BB
:10FA60008A2E912CA12CB12CF2E0CF2ED12CE12C9E
:10FA7000F12CC101B701A601980147DE882309F4E2
:10FA800071C089819A81AB81BC81A70196012F5FEA
:10FA90003F4F4F4F5F4F0097A105B10519F0490146
:10FAA0005A010DC0281939094A095B098A859B85C5
:10FAB000AC85BD85281739074A075B0759F00894BC
:10FAC000411C511C611C711C0894C11CD11CE11CFF
:10FAD000F11CB1CFC101A601B7010FEF1FEF2FEF4E
:10FAE0003FE08DDD882391F43DC026013701089465
:10FAF0004108510861087108C101B301A2019701D1
:10FB000086017DDD882371F1730162018C149D04EF
:10FB1000AE04BF0450F3AE85BF854D915D916D91EC
:10FB20007C91411551056105710531F0C1019501C7
:10FB3000840165DD8823B1F0EE85FF8580829182A6
:10FB4000A282B382FD81FF2359F00894811C911C8D
:10FB5000A11CB11CD1018D929D92AD92BC921397C4
:10FB600081E001C080E02F960FB6F894DEBF0FBE93
:10FB7000CDBFCF91DF911F910F91FF90EF90DF905C
:10FB8000CF90BF90AF909F908F907F906F905F903D
:10FB90004F903F902F900895109260101092621035
:10FBA000109264100895809384030895EFE6F0E0C6
:10FBB00080818260808308951F93FC011FB7F894B1
:10FBC00080819181A281B38180933A1090933B1000
:10FBD000A0933C10B0933D10FB0180819181A281E4
:10FBE000B38180933E1090933F10A0934010B09348
:10FBF0004110FA0180819181A281B38180934210EA
:10FC000090934310A0934410B0934510F901808164
:10FC10009181A281B3818093461090934710A09365
:10FC20004810B09349101FBF1F910895FC012FB7D2
:10FC3000F89480819181A281B38180934610909342
:10FC40004710A0934810B09349102FBF0895E82F94
:10FC50008FB7F894F0E0EE0FFF1FEE0FFF1FE65C8A
:10FC6000FF4E20813181428153818FBFB901CA018A
:10FC7000089580916F008D7F80936F0006C0809102
:10FC8000060E8F5F8F708093060E9091050E809107
:10FC9000060E981751F410922D1010922C1080918E
:10FCA0006F00826080936F0008959091050E80919F
:10FCB000060E981751F3E3CF9B01882399F4B901FD
:10FCC000882777FD8095982F2FEF30E040E050E0B7
:10FCD0000E9450DC20ED37E040E050E00E94C4DCA0
:10FCE0008CE214C08130A9F4B901882777FD809592
:10FCF000982F2FEF30E040E050E00E9450DC20EDE4
:10FD000037E040E050E00E94C4DC8DE2B9010C9481
:10FD1000BA1A8230A9F4B901882777FD8095982F07
:10FD20002FEF30E040E050E00E9450DC20ED37E063
:10FD300040E050E00E94C4DC8EE2B9010C94BA1A93
:10FD400008958CE261E00E94981B8DE261E00E94C0
:10FD5000981B8EE261E00E94981B60917A0370917B
:10FD60007B0380E0A9DF60917C0370917D0381E0DB
:10FD7000A3DF60917E0370917F0382E09DDFE1E26B
:10FD8000F1E08081887F816080830895DADF099ABD
:10FD90003C9A399AEAE0F1E0808180648083808136
:10FDA000846080830D9A159A3E9A469A3B9A439AAC
:10FDB000389A409A8081826080839FB7F894EBE004
:10FDC000F1E08081826080839FBF0898109A0C9830
:10FDD000149A0F98179A0B9A1398159A3D9A45986A
:10FDE000469A3A9A4298439AEAE0F1E08081806824
:10FDF00080839FB7F894EBE0F1E080818F77808378
:10FE00009FBF409AEAE0F1E08081816080839FB7E4
:10FE1000F894EBE0F1E080818E7F80839FBFA1E8C2
:10FE2000B0E08C918F7E8C938C9188608C93E0E80D
:10FE3000F0E080818D7F808380818E7F80838081D0
:10FE40008F73808380818F7C80838C91887F826098
:10FE50008C9380E090E490938900809388001092C6
:10FE6000850010928400EFE6F0E08081826080835C
:10FE700081E080938403789408959091050E809199
:10FE8000060E981739F00E946D8B0E9470300E9408
:10FE9000BF94F3CF0895F1DF159A469A439A409A9A
:10FEA00008951F920F920FB60F920BB60F92112466
:10FEB000AF92BF92CF92DF92EF92FF920F931F9378
:10FEC0002F933F934F935F936F937F938F939F9362
:10FED000AF93BF93CF93DF93EF93FF9380912C1059
:10FEE00090912D10892B09F094C19091050E80916D
:10FEF000060E981719F4E0E0F0E014C08091060EA9
:10FF000090E02DE430E0829FF001839FF00D929FFE
:10FF1000F00D1124EB5CF64FE45BFF4F81E0808332
:10FF2000EC54F040F0932D10E0932C10309709F42E
:10FF30006AC1E45BFF4F81E08083EC54F040109293
:10FF40006C1010926D1010926E1010926F1060ADC8
:10FF500071AD2CE96134720718F060E47CE904C0EB
:10FF60003EE46132730730F0769567957695679534
:10FF700084E007C047E26131740730F076956795F9
:10FF800082E08093651007C0809365106032710530
:10FF900010F460E270E06052704058E06030750725
:10FFA000E8F0472F50E0440F551F440F551F4B5F9B
:10FFB000524F9A012E5F3F4FF901859194919C0118
:10FFC000AA27639FC001629F810D9A1F06948A1F12
:10FFD0009A1F1124FA01459154911EC0CB019695A8
:10FFE00087958C7F8B5F9E4EFC0145915491FC015F
:10FFF000329625913491862F90E087709070FC01A5
:020000021000EC
:100000002E9FC0012F9F900D3E9F900D1124B3E0B5
:1000100096958795BA95E1F7481B590B44365105DB
:10002000A8F4E0EEF2E007C08091C00085FFFCCFAD
:1000300031969093C60090819923B1F780EC98E0B7
:100040004AE050E00E94615644E650E0509371103F
:10005000409370108091651080937210109273100D
:10006000E0912C10F0912D1064AD75AD70936B1074
:1000700060936A10FCE961347F0718F060E47CE962
:1000800004C02EE46132720730F07695679576955C
:10009000679584E007C037E26131730730F07695E9
:1000A000679582E08093651008C081E080936510B9
:1000B0006032710510F460E270E06052704048E018
:1000C00060307407E8F0472F50E0440F551F440F8D
:1000D000551F4B5F524F9A012E5F3F4FF90185919B
:1000E00094919C01AA27639FC001629F810D9A1F72
:1000F00006948A1F9A1F1124FA01459154911EC03B
:10010000CB01969587958C7F8B5F9E4EFC01459128
:100110005491FC01329625913491862F90E087709E
:100120009070FC012E9FC0012F9F900D3E9F900D5F
:10013000112433E0969587953A95E1F7481B590BC2
:1001400044365105A8F4E0EEF2E007C08091C0000B
:1001500085FFFCCF31969093C60090819923B1F72B
:1001600080EC98E04AE050E00E94615644E650E09E
:10017000CA01A0E0B0E08093661090936710A0934E
:100180006810B09369105093890040938800E09103
:100190002C10F0912D1080899189A289B389B69590
:1001A000A79597958795B095A095909581959F4F28
:1001B000AF4FBF4F80934A1090934B10A0934C10B9
:1001C000B0934D1080934E1090934F10A093501009
:1001D000B09351108093521090935310A0935410E9
:1001E000B09355108093561090935710A0935810C9
:1001F000B093591010925A1010925B1010925C102C
:1002000010925D1006C080ED97E090938900809376
:100210008800C0912C10D0912D10209709F489C42A
:1002200088A180935E1080FF03C0119A8FEF02C0F7
:10023000119881E08093800380915E1081FF03C05C
:1002400044988FEF02C0449A81E0809381038091AB
:100250005E1080FF36C080918403882391F120B125
:10026000217031E0232759F180915F10882339F103
:1002700088819981AA81BB81181619061A061B0666
:10028000F4F480913A1090913B10A0913C10B09101
:100290003D1080932E1090932F10A0933010B093A8
:1002A00031103093601088899989AA89BB8980931D
:1002B0005A1090935B10A0935C10B0935D10209344
:1002C0005F1080915E1081FD3AC080918403882385
:1002D000B1F180B182958F708095282F217080FFB9
:1002E0002CC080916110882341F18C819D81AE8169
:1002F000BF81181619061A061B06FCF480913E10E1
:1003000090913F10A0914010B09141108093321015
:1003100090933310A0933410B093351081E0809304
:10032000621088899989AA89BB8980935A10909311
:100330005B10A0935C10B0935D10209361108091CE
:100340005E1082FF05C0419A8FEF8093820339C00F
:10035000419881E08093820380918403882389F10E
:1003600020E007992CC021E080916310882339F1A7
:1003700088859985AA85BB85181619061A061B0655
:10038000F4F48091421090914310A0914410B091E8
:1003900045108093361090933710A0933810B09387
:1003A00039102093641088899989AA89BB89809320
:1003B0005A1090935B10A0935C10B0935D10209343
:1003C000631080915E1083FF0AC08FB7F8949091FC
:1003D0000B019F7B90930B018FBF8FEF09C08FB7ED
:1003E000F89490910B01906490930B018FBF81E082
:1003F0008093830360E070E079C18091C00087FF43
:1004000019C04091C600E091BC08F091BD0831963A
:100410009F012F77307031978091BE089091BF086F
:100420002817390739F0E45CF74F40833093BD0853
:100430002093BC08288139814A815B8180914A10D0
:1004400090914B10A0914C10B0914D10280F391F76
:100450004A1F5B1F20934A1030934B1040934C105F
:1004600050934D1012161306140615066CF5139AC8
:1004700088899989AA89BB89281B390B4A0B5B0B90
:1004800020934A1030934B1040934C1050934D10D2
:1004900020913A1030913B1040913C1050913D100A
:1004A00080918003992787FD9095A92FB92F820FFE
:1004B000931FA41FB51F80933A1090933B10A093F5
:1004C0003C10B0933D1013982C813D814E815F818B
:1004D00080914E1090914F10A0915010B0915110FA
:1004E000280F391F4A1F5B1F20934E1030934F1067
:1004F000409350105093511012161306140615060F
:100500006CF5459A88899989AA89BB89281B390B7A
:100510004A0B5B0B20934E1030934F1040935010BA
:100520005093511020913E1030913F104091401057
:100530005091411080918103992787FD9095A92FB3
:10054000B92F820F931FA41FB51F80933E10909365
:100550003F10A0934010B0934110459828853985ED
:100560004A855B858091521090915310A091541050
:10057000B0915510280F391F4A1F5B1F209352104E
:100580003093531040935410509355101216130685
:10059000140615066CF5429A88899989AA89BB893F
:1005A000281B390B4A0B5B0B2093521030935310CE
:1005B00040935410509355102091421030914310A5
:1005C000409144105091451080918203992787FDF6
:1005D0009095A92FB92F820F931FA41FB51F809349
:1005E000421090934310A0934410B093451042984A
:1005F0002C853D854E855F858091561090915710D2
:10060000A0915810B0915910280F391F4A1F5B1F35
:100610002093561030935710409358105093591010
:100620001216130614061506DCF59FB7F894809190
:100630000B01806880930B019FBF88899989AA89E3
:10064000BB89281B390B4A0B5B0B20935610309348
:1006500057104093581050935910209146103091E4
:100660004710409148105091491080918303992779
:1006700087FD9095A92FB92F820F931FA41FB51F37
:100680008093461090934710A0934810B093491060
:100690009FB7F89480910B018F7780930B019FBFD8
:1006A00080915A1090915B10A0915C10B0915D10F8
:1006B0000196A11DB11D80935A1090935B10A093D9
:1006C0005C10B0935D1020915A1030915B104091F6
:1006D0005C1050915D106F5F7F4F88899989AA895E
:1006E000BB89281739074A075B0738F480916510E2
:1006F00090E0681779070CF480CE20915A10309161
:100700005B1040915C1050915D108C899D89AE8981
:10071000BF8982179307A407B50708F4E3C0E090E8
:100720006610F09067100091681010916910AC8C01
:10073000BD8CCE8CDF8CA8019701C601B501AA271C
:10074000279FB12D389FF001489FF00D479FE00D86
:10075000F11D289FB00DE11DFA1F379FB00DE11D5F
:10076000FA1F469FB00DE11DFA1F369FB10DEA1F1B
:10077000FA1FB695EA1FFA1F11248CAD9DAD8E0F9E
:100780009F1F90936B1080936A1028AD39AD4AADCE
:100790005BADA0E0B0E0281739074A075B0720F4FB
:1007A00030936B1020936A1060916A1070916B10F7
:1007B0008CE96134780718F060E47CE904C09EE4B9
:1007C0006132790730F0769567957695679584E084
:1007D00007C0E7E261317E0730F07695679582E0E9
:1007E0008093651008C081E08093651060327105C8
:1007F00010F460E270E060527040F8E060307F0713
:10080000E8F0472F50E0440F551F440F551F4B5F32
:10081000524F9A012E5F3F4FF901859194919C01AF
:10082000AA27639FC001629F810D9A1F06948A1FA9
:100830009A1F1124FA01459154911EC0CB0196953F
:1008400087958C7F8B5F9E4EFC0145915491FC01F6
:10085000329625913491862F90E087709070FC013C
:100860002E9FC0012F9F900D3E9F900D1124B3E04D
:1008700096958795BA95E1F7481B590B4436510573
:10088000A8F4E0EEF2E007C08091C00085FFFCCF45
:1008900031969093C60090819923B1F780EC98E04F
:1008A0004AE050E00E94615644E650E050938900CF
:1008B000409388009A0140E050E08091661090914A
:1008C0006710A0916810B0916910820F931FA41F48
:1008D000B51F8093661090936710A0936810B09333
:1008E000691002C120915A1030915B1040915C1048
:1008F00050915D10888D998DAA8DBB8D82179307BD
:10090000A407B50708F0E4C060916C1070916D10F9
:1009100080916E1090916F102C8D3D8D4E8D5F8D5E
:10092000AA27639FB12D749FF001849FF00D839FD0
:10093000E00DF11D649FB00DE11DFA1F739FB00D16
:10094000E11DFA1F829FB00DE11DFA1F729FB10DCC
:10095000EA1FFA1FB695EA1FFA1F112480916A1048
:1009600090916B108E179F0738F4C05CDF4F688141
:100970007981C054D04003C0BC016E1B7F0BC05CAA
:10098000DF4F288139814A815B81CB01A0E0B0E053
:1009900082179307A407B50708F4B901FCE961348D
:1009A0007F0718F060E47CE904C02EE4613272072E
:1009B00030F0769567957695679584E007C037E2C5
:1009C0006131730730F07695679582E0809365100A
:1009D00008C081E0809365106032710510F460E218
:1009E00070E06052704048E060307407E8F0472FD4
:1009F00050E0440F551F440F551F4B5F524F9A0153
:100A00002E5F3F4FF901859194919C01AA27639F26
:100A1000C001629F810D9A1F06948A1F9A1F11249C
:100A2000FA01459154911EC0CB01969587958C7F14
:100A30008B5F9E4EFC0145915491FC0132962591AD
:100A40003491862F90E087709070FC012E9FC0013A
:100A50002F9F900D3E9F900D112423E09695879532
:100A60002A95E1F7481B590B44365105A8F4E0EEEE
:100A7000F2E007C08091C00085FFFCCF31969093D3
:100A8000C60090819923B1F780EC98E04AE050E0ED
:100A90000E94615644E650E05093890040938800DC
:100AA0009A0140E050E080916C1090916D10A091FF
:100AB0006E10B0916F10820F931FA41FB51F80930B
:100AC0006C1090936D10A0936E10B0936F100CC0CB
:100AD000809170109091711090938900809388009C
:100AE000809172108093651020915A1030915B10A4
:100AF00040915C1050915D10E0912C10F0912D1000
:100B000080899189A289B389281739074A075B0729
:100B100080F010922D1010922C109091050E809163
:100B2000060E981731F08091060E8F5F8F708093BC
:100B3000060EFF91EF91DF91CF91BF91AF919F9101
:100B40008F917F916F915F914F913F912F911F9165
:100B50000F91FF90EF90DF90CF90BF90AF900F90EC
:100B60000BBE0F900FBE0F901F90189580916010D4
:100B7000882349F480916210882329F480916410BD
:100B8000882309F490C0E5E0F5E1949108C08091D4
:100B9000C00085FFFCCF9093C600319694919923B5
:100BA000B1F7E7E1F5E1949108C08091C00085FFBD
:100BB000FCCF9093C600319694919923B1F7809120
:100BC00060108823D1F060912E1070912F108091C9
:100BD0003010909131100E9476D62091D508309136
:100BE000D6084091D7085091D8080E94DBD5AB01B8
:100BF000BC0183E195E10E94073480916210882353
:100C0000D1F0609132107091331080913410909136
:100C100035100E9476D62091D9083091DA0840919B
:100C2000DB085091DC080E94DBD5AB01BC018FE0F2
:100C300095E10E940734809164108823D1F060917F
:100C400036107091371080913810909139100E94B1
:100C500076D62091DD083091DE084091DF08509172
:100C6000E0080E94DBD5AB01BC018BE095E10E945E
:100C70000734E4EFF2E007C08091C00085FFFCCFAD
:100C800031969093C60090819923B1F78091C0006E
:100C900085FFFCCF8AE08093C6001092601010920E
:100CA000621010926410089560E070E08FE793E4A2
:100CB0002091890330918A0340918B0350918C03DA
:100CC0000E94DBD56093A8107093A9108093AA109E
:100CD0009093AB1060E070E08FE793E4209199036C
:100CE00030919A0340919B0350919C030E94DBD565
:100CF0006093B0107093B1108093B2109093B310C2
:100D00000895FC0197FF03C08091851003C0EC5744
:100D1000FF4E808190E008952F923F924F925F9214
:100D20006F927F928F929F92AF92BF92CF92DF92FB
:100D3000EF92FF920F931F93CF93DF93EC0121E08B
:100D400030E0A901440F551F440F551FFA01E2522C
:100D5000FA4E85919491C817D9070CF059C0B90182
:100D600061507040660F771F660F771FCB0180526E
:100D70009A4EFC010591149162527A4EFB01C59086
:100D8000D490FA01E052FA4EE590F490FA01E25262
:100D9000FA4EA590B490B801882777FD8095982FDA
:100DA0000E9476D61B012C01CC19DD09BE018827D3
:100DB00077FD8095982F0E9476D63B014C01E01A72
:100DC000F10A0027F7FC0095102FC801B7010E9417
:100DD00076D69B01AC01C401B3010E94A9D87B0166
:100DE0008C01AC18BD08CC24B7FCC094DC2CC60127
:100DF000B5010E9476D69B01AC01C801B7010E94E3
:100E0000DBD59B01AC01C201B1010E94FBD419C02A
:100E1000822F8F5F2F5F3F4F2133310509F091CF34
:100E2000813329F0E0E070E080E060E00CC0E0EAAF
:100E3000F6E165917491882777FD8095982F0E943F
:100E400076D6E62F692F2E2F372F482F562FB90130
:100E5000CA01DF91CF911F910F91FF90EF90DF902A
:100E6000CF90BF90AF909F908F907F906F905F904A
:100E70004F903F902F900895089510927510109202
:100E8000741010928410749810927710109276104B
:100E90001092851080E090E0A0E0B0E080939C107C
:100EA00090939D10A0939E10B0939F108093A010DC
:100EB0009093A110A093A210B093A310A5980895A9
:100EC0002DEB37E346E05EE30C94A9D82DEB37E336
:100ED00046E05EE30C94DBD52DEB37E346E05EE3C2
:100EE0000C94DBD52DEB37E346E05EE30C94A9D8F8
:100EF000A5980E949C2F882319F5E6E2F5E19491CC
:100F000008C08091C00085FFFCCF9093C600319649
:100F100094919923B1F7EDE2F5E1949108C08091A5
:100F2000C00085FFFCCF9093C60031969491992321
:100F3000B1F78091C00085FFFCCF8AE08093C600A6
:100F400083E00C94D82F1F93182F97DF0E949C2FBB
:100F5000882391F5E6E2F5E1949108C08091C00004
:100F600085FFFCCF9093C600319694919923B1F7F9
:100F700080EC98E0612F70E04AE050E00E943A5621
:100F80008091C00085FFFCCF8AE08093C600E7E631
:100F9000F5E1949108C08091C00085FFFCCF90934B
:100FA000C600319694919923B1F78091C00085FFD6
:100FB000FCCF8AE08093C60082E00E94D82F1F9168
:100FC00008951F93182F59DF0E949C2F882391F5B5
:100FD000E6E2F5E1949108C08091C00085FFFCCF66
:100FE0009093C600319694919923B1F780EC98E0E4
:100FF000612F70E04AE050E00E943A568091C000B4
:1010000085FFFCCF8AE08093C600E4E9F5E1949186
:1010100008C08091C00085FFFCCF9093C600319638
:1010200094919923B1F78091C00085FFFCCF8AE0AD
:101030008093C60081E00E94D82F1F9108951F92CF
:101040000F920FB60F920BB60F9211242F933F936E
:101050004F935F936F937F938F939F93AF93BF93C0
:10106000EF93FF939091A503992361F480918410ED
:1010700080938A108111749A8091851080938910D1
:101080008111A59A80918A10981708F07498809120
:101090008910981708F0A5989F5F9F779093A503F4
:1010A0008091A603843009F471C0853050F48130FA
:1010B00021F1813098F08230F1F1833009F07AC06B
:1010C00049C0863009F468C0863008F463C08730B0
:1010D00009F466C0883009F06DC06AC088E080936A
:1010E0007B0080E480937C0080917A008064809310
:1010F0007A000E947E9281E01BC0809178009091DE
:101100007900A0E0B0E020919710309198104091C4
:10111000991050919A10280F391F4A1F5B1F209376
:101120009710309398104093991050939A1082E042
:101130008093A6033FC088E080937B0082E4809385
:101140007C0080917A00806480937A000E947E9275
:1011500083E0EECF8091780090917900A0E0B0E03C
:1011600020918B1030918C1040918D1050918E10E9
:10117000280F391F4A1F5B1F20938B1030938C1050
:1011800040938D1050938E1084E0D2CF0E947E92B7
:1011900085E0CECF86E0CCCF0E947E9287E0C8CF9C
:1011A0001092A60380919B108F5F80939B1002C0CA
:1011B0001092A60380919B10803108F463C0809147
:1011C0008610882381F480919710909198109093C5
:1011D00079108093781080918B1090918C1090935F
:1011E0007F1080937E1081E08093861010929B1078
:1011F00010929710109298101092991010929A10C5
:1012000010929310109294101092951010929610C4
:1012100010928F10109290101092911010929210C4
:1012200010928B1010928C1010928D1010928E10C4
:1012300020917810309179108091A1039091A203B0
:101240002817390714F080E0BCDE20917810309127
:10125000791080918710909188108217930714F06D
:1012600080E071DE20917E1030917F108091A30389
:101270009091A403281739072CF010927710109240
:10128000761036DEFF91EF91BF91AF919F918F91D4
:101290007F916F915F914F913F912F910F900BBE76
:1012A0000F900FBE0F901F9018952F926F927F9204
:1012B0008F929F92AF92BF92CF92DF92EF92FF9266
:1012C0000F931F93DF93CF93CDB7DEB729970FB658
:1012D000F894DEBF0FBECDBF8C01E62E662369F108
:1012E000E6E2F5E1949108C08091C00085FFFCCF53
:1012F0009093C600319694919923B1F780EC98E0D1
:101300006E2D70E04AE050E00E943A56E1ECF5E1C3
:10131000949108C08091C00085FFFCCF9093C600D7
:10132000319694919923B1F78091C00085FFFCCF4D
:101330008AE08093C6000E941830AE2DB0E0FD0117
:10134000EE0FFF1FE25EFB4F608171817987688736
:10135000672B09F49FC0A05EBB4F7C917B83222446
:10136000239479C0222D30E0A901440F551F440F6A
:10137000551FE885F985E40FF51F859194910817AD
:1013800019070CF067C0C9010197880F991F880FD2
:10139000991FFC013296A885B985EA0FFB1FC590FD
:1013A000D4908A0F9B1FFC01659174917A836983A5
:1013B000FA013296EA0FFB1FE590F490FD01E40F6D
:1013C000F51FA590B490B601882777FD8095982FDA
:1013D0000E9476D66C837D838E839F8389819A81D8
:1013E000081B190BB801882777FD8095982F0E945C
:1013F00076D63B014C01EC18FD080027F7FC009560
:10140000102FC801B7010E9476D69B01AC01C40120
:10141000B3010E94A9D87B018C01A981BA81AA1AC3
:10142000BB0ACC24B7FCC094DC2CC601B5010E94D9
:1014300076D69B01AC01C801B7010E94DBD59B01A8
:10144000AC016C817D818E819F810E94FBD4E62F4F
:10145000692F09C02394BB812B1608F483CFE0E0E9
:1014600070E080E060E0FB812F1679F5E22DF0E07E
:10147000EE0FFF1FEE0FFF1F329768857985E60F8D
:10148000F71F65917491882777FD8095982F0E94AA
:1014900076D619C0B801882777FD8095982F0E94CD
:1014A00076D620E030E04AEF5EE30E94A9D820E043
:1014B00030E040E85DE30E94A9D820E030E040E061
:1014C00050E00E94FBD4E62F692F2E2F372F482F94
:1014D000562FB901CA0129960FB6F894DEBF0FBE88
:1014E000CDBFCF91DF911F910F91FF90EF90DF90D3
:1014F000CF90BF90AF909F908F907F906F902F90E4
:101500000895EF92FF920F931F93CF93DF930F2EC7
:10151000F0E0EF2EF0E0FF2EF0E00F2FF0E01F2FB5
:10152000F02DE092A410F092A5100093A610109355
:10153000A71060E070E08FE793E420918903309179
:101540008A0340918B0350918C030E94DBD56093FA
:10155000A8107093A9108093AA109093AB10E092FA
:10156000AC10F092AD100093AE101093AF1060E08D
:1015700070E08FE793E42091990330919A034091B2
:101580009B0350919C030E94DBD56093B010709335
:10159000B1108093B2109093B3106C9A6D9A9D9A8B
:1015A0008091010180618093010187ED80937A0031
:1015B00010927E0010927D0080917D00816080936A
:1015C0007D0080917D00826080937D0080917D0010
:1015D000846080937D0080E888BD80916E00846087
:1015E00080936E0085E090E09093B5108093B410E6
:1015F00009C0809187109091881040969093881030
:1016000080938710809187109091881060E04DDE64
:1016100020E030E040EA50E40E94D4D587FDE9CFD5
:1016200083E191E09093A8038093A70309C0809180
:10163000A1039091A20340979093A2038093A103EA
:101640008091A1039091A20360E02FDE20E030E8BA
:1016500049E853E40E94D7D718164CF3C091A3036E
:10166000D091A403EC2E1D2FCE0156DB609720E015
:1016700030E048E453E40E94D7D718169CF3E09278
:10168000A3031093A403DF91CF911F910F91FF90BB
:10169000EF900895809178109091791060E005DEC8
:1016A00060937A1070937B1080937C1090937D10E0
:1016B00080917E1090917F102FDB6093801070934B
:1016C000811080938210909383100E9418D18FB75D
:1016D000F894109286108FBF08952F923F924F92E8
:1016E0005F926F927F928F929F92AF92BF92CF92B2
:1016F000DF92EF92FF920F931F93809186108823C1
:1017000009F46EC2C7DF60907A1070907B108090F1
:101710007C1090907D10C0907410D0907510B60120
:10172000882777FD8095982F0E9476D6A401930193
:101730000E94FAD47B018C016093B6107093B710AD
:101740008093B8109093B91020E030E04AE754E459
:101750000E94D7D7181624F481E08093BA10E9C00C
:10176000C801B70120E030E04AE754EC0E94D4D52C
:1017700087FD02C0CD2821F481E08093BA10C4C057
:101780008091BA10882371F080E090E0A0E0B0E092
:101790008093BB109093BC10A093BD10B093BE106B
:1017A0001092BA10C801B7012091850330918603C9
:1017B00040918703509188030E94A9D81B012C01F6
:1017C0006093BF107093C0108093C1109093C210AB
:1017D000C801B7012091BB103091BC104091BD10E1
:1017E0005091BE100E94FBD45B016C01E090A410EC
:1017F000F090A5100091A6101091A710A8019701D4
:101800000E94D4D587FD12C0E090A810F090A910D6
:101810000091AA101091AB10C601B501A801970163
:101820000E94D7D7181614F086017501E092BB10FC
:10183000F092BC100093BD101093BE10C801B70108
:101840002091890330918A0340918B0350918C033E
:101850000E94A9D85B016C016093C3107093C410FF
:101860008093C5109093C610C401B3012091C71096
:101870003091C8104091C9105091CA100E94FAD4FA
:1018800020918D0330918E0340918F0350919003EE
:101890000E94A9D820E037ED43E25CE30E94A9D87A
:1018A0007B018C016091CB107091CC108091CD1098
:1018B0009091CE1024EA30E74DE75FE30E94A9D86B
:1018C0009B01AC01C801B7010E94FBD47B018C01D4
:1018D0006093CB107093CC108093CD109093CE106A
:1018E000C201B101A60195010E94FBD4A801970194
:1018F0000E94FAD47B018C0120E030E040E050E00F
:101900000E94D4D588235CF40F2EF0E0EF2EF0E097
:10191000FF2EF0E00F2FF0E01F2FF02D14C0C801B4
:10192000B70120E030E04FE753E40E94D7D7181604
:1019300054F40F2EF0E0EF2EF0E0FF2EFFE70F2F14
:10194000F3E41F2FF02D6092C7107092C8108092A0
:10195000C9109092CA106091B4107091B510882788
:1019600077FD8095982F0E9476D69B01AC01C4012B
:10197000B3010E94D7D71816DCF46091A7037091C9
:10198000A803882777FD8095982F0E9476D69B0123
:10199000AC01C401B3010E94D4D588234CF4C80122
:1019A000B7010E9443D6759567956093841002C075
:1019B000109284106090801070908110809082103E
:1019C000909083106091761070917710882777FD42
:1019D0008095982F0E9476D6A40193010E94FAD494
:1019E0007B018C016093CF107093D0108093D11045
:1019F0009093D210209195033091960340919703D4
:101A0000509198030E94A9D81B012C0160939C104F
:101A100070939D1080939E1090939F10C801B70102
:101A20002091D3103091D4104091D5105091D61000
:101A30000E94FBD45B016C01E090AC10F090AD1003
:101A40000091AE101091AF10A80197010E94D4D55B
:101A500087FD12C0E090B010F090B1100091B2106C
:101A60001091B310C601B501A80197010E94D7D704
:101A7000181614F086017501E092D310F092D4107C
:101A80000093D5101093D610C801B7012091990387
:101A900030919A0340919B0350919C030E94A9D8D6
:101AA0005B016C016093A0107093A1108093A21051
:101AB0009093A310C401B3012091D7103091D81096
:101AC0004091D9105091DA100E94FAD420919D03D0
:101AD00030919E0340919F035091A0030E94A9D88A
:101AE00020E037ED43E25CE30E94A9D87B018C0142
:101AF0006091DB107091DC108091DD109091DE1010
:101B000024EA30E74DE75FE30E94A9D89B01AC01CE
:101B1000C801B7010E94FBD47B018C016093DB10EC
:101B20007093DC108093DD109093DE106092D710DC
:101B30007092D8108092D9109092DA10C201B1013F
:101B4000A60195010E94FBD4A80197010E94FAD436
:101B50007B018C0120E030E040E050E00E94D4D5D1
:101B600088235CF40F2EF0E0EF2EF0E0FF2EF0E083
:101B70000F2FF0E01F2FF02D14C0C801B70120E097
:101B800030E04FE753E40E94D7D7181654F40F2ED5
:101B9000F0E0EF2EF0E0FF2EFFE70F2FF3E41F2F12
:101BA000F02DC401B30120E030E040EA50E40E948F
:101BB000D7D718169CF4C401B30120E030E048E404
:101BC00053E40E94D4D588234CF4C801B7010E9485
:101BD00043D6759567956093851002C01092851065
:101BE0001F910F91FF90EF90DF90CF90BF90AF903B
:101BF0009F908F907F906F905F904F903F902F902D
:101C000008952F923F924F925F926F927F928F92A0
